:020000040800F2
:10000000781900209502000823200008F116000846
:1000100021200008CB15000859300008000000001E
:10002000000000000000000000000000D3220008D3
:10003000CD15000800000000D12200088528000826
:10004000AF020008AF020008AF020008AF020008CC
:10005000AF020008AF020008AF020008AF020008BC
:10006000AF020008AF020008AF020008AF020008AC
:10007000AF020008AF020008AF020008AF0200089C
:10008000AF020008AF020008AF020008AF0200088C
:10009000AF020008AF020008AF020008AF0200087C
:1000A000AF020008AF020008AF020008AF0200086C
:1000B00095290008052E000800000000AF02000886
:1000C000AF0200080000000000000000AF020008BE
:1000D00000000000AF020008AF020008AF020008F5
:1000E000AF020008AF02000800000000000000009E
:1000F0000000000000000000000000000000000000
:1001000000000000000000000000000000000000EF
:100110000000000000000000A92E0008AF02000847
:1001200000000000000000000000000000000000CF
:1001300000000000000000000000000000000000BF
:10014000AF020008AF02000800000000000000003D
:10015000000000000000000000000000000000009F
:10016000000000000000000000000000000000008F
:10017000000000000000000000000000000000007F
:1001800000000000AF02000800F002F800F072F872
:100190000AA090E8000C82448344AAF10107DA45E2
:1001A00001D100F067F8AFF2090EBAE80F0013F0C2
:1001B000010F18BFFB1A43F00103184798CB00004A
:1001C000B8CB00000A444FF0000C10F8013B13F0CC
:1001D000070408BF10F8014B1D1108BF10F8015BA0
:1001E000641E05D010F8016B641E01F8016BF9D193
:1001F00013F0080F1EBF10F8014BAD1C0C1B09D1EA
:100200006D1E58BF01F801CBFAD505E014F8016B5B
:1002100001F8016B6D1EF9D59142D6D370470000ED
:100220000023002400250026103A28BF78C1FBD8FF
:10023000520728BF30C148BF0B60704766290AF0DB
:10024000EE87642900F0AA80782900F0E380732902
:1002500000F07584002070471FB50AF0D6FF00F04B
:1002600073FC0400002000210AF07AF9E0601FBD51
:1002700010B510BD00F06CFD1146FFF7EDFF05F065
:10028000FBFB00F08AFD03B4FFF7F2FF03BC00F0B4
:10029000CDFD00000948804709480047FEE7FEE71A
:1002A000FEE7FEE7FEE7FEE7FEE7FEE7FEE7FEE726
:1002B00004480549054A064B704700008529000897
:1002C0008901000878130020781900207815002093
:1002D000781500200FB41CB5074B06AA7B4469466D
:1002E0000090059800F001FC0020694600F010FC29
:1002F0001CBC5DF814FB00003108000070B504461A
:1003000085690068C10601D5302600E02026C007B7
:1003100007D070BDD4E9012130469047206A401CC7
:1003200020626D1EF6D570BD70B5044685690078F3
:10033000C00707D170BDD4E9012120209047206A71
:10034000401C20626D1EF6D570BD70B50C4605468A
:10035000012A05D02878800600D5EA69002302E04A
:10036000012305E05B1C934202D2E05C0028F9D136
:10037000A869E618C01AA861286A184428622846A5
:10038000FFF7BCFF04E0D5E9012114F8010B904709
:10039000B442F8D32846FFF7C7FF70BD2DE9F041FE
:1003A0000646002410687529314616A510D0AFF313
:1003B0000080002802DA404213A507E031688A076E
:1003C00001D512A502E0490704D511A5012401E0D9
:1003D000AFF3008000210A2206F1240709E0B0FBF8
:1003E000F2FCB0FBF2F302FB1C00303078541846EC
:1003F000491C0028F3D123462A463046BDE8F04187
:1004000000F006B9000000002D0000002B000000E5
:100410002000000070B504460D4621461068AFF379
:1004200000802188090502D50F4A7A4402E00E4A6D
:100430007A440E32002104F1240305E000F00F0697
:100440000009965D5E54491C0028F7D120780023EE
:10045000000704D5702D02D009B1022311322046C5
:10046000BDE8704000F0D4B86AC200002DE9F05F2A
:10047000894604464FF0000ADFF874B1FB44C0F827
:1004800020A02046E1688847002874D0252806D09F
:10049000D4E901219047206A401C2062F1E7002640
:1004A0005F462046E16888472028054607DB312D56
:1004B00005D2781910F8200C08B10643F1E7B0070F
:1004C00001D526F00406C4F81CA00027C4F818A023
:1004D0002A2D09D0284604F0D9FB38B304EB87084D
:1004E000303DC8F8185019E059F8041B204604EBB9
:1004F00087029161E1688847012F054618D1E069BC
:10050000002820DA26F020061DE0D8F8180000EBBD
:10051000800005EB40003038C8F818002046E1683C
:100520008847054604F0B2FB0028EED1012F0AD01F
:100530002E2D08D12046E16888477F1C0546022FF2
:1005400046F02006C4DBA069002803DA404246F0EA
:100550000106A061F00701D026F010066C2D0BD02B
:10056000682D09D04C2D39D06A2D35D0742D35D059
:100570007A2D33D016E038E0E1682F4620468847D0
:10058000B842054609D16C2F26D04FF48060E1684F
:10059000064320468847054604E06C2F1AD04FF4E6
:1005A000807006430DB3A5F14100192802D820350B
:1005B00046F400664A462946204626604E46FFF726
:1005C0003DFE80B101280BD0F61D26F0070000F19A
:1005D000080956E74020E4E78020D8E70020D6E766
:1005E00006F104094DE7284652E7206ABDE8F09F6E
:1005F00040C2000070477047704710B500F0A8FA7D
:10060000006810BD10B5044600F0A2FA046010BDE9
:100610002DE9F0470D4699469246044600F124081C
:100620000168880604D5E06921F01001216000E02E
:100630000120A84201DD471B00E00027A1697A19CB
:1006400002EB0900081AA0612078C00602D42046F7
:10065000FFF754FE002608E0D4E901211AF806004D
:100660009047206A401C761C20624E45F4DB2078BF
:10067000C0060AD52046FFF741FE06E0D4E9012175
:1006800030209047206A401C2062381EA7F10107E5
:10069000F4DC07E0D4E9012118F805009047206A4E
:1006A000401C2062281EA5F10105F3DC2046FFF75F
:1006B0003BFE2078000602D50220BDE8F08701202D
:1006C000FBE770472DE9FF4F0C461E464FF0FF3702
:1006D0008BB0D2E90001DDF860800A908A46C1F350
:1006E0000A5505B93D46002108464FF00000BAF111
:1006F000000F00F4400005DA00EB80004FF44001E9
:1007000001EA50004FEA9059B9F1010F00DDB946F6
:100710000A9850EA4A000ED044F61050A5F2FF3570
:1007200045432F14B8F1000F1ED07542291E1EDD5F
:10073000C9F100021CE0B8F1010F4FF0000001D038
:10074000302103E0F24305E02154401CB042FBDBC2
:1007500030460022002121540B99C1F80880C1E9DC
:1007600000200FB0BDE8F08FBD1B6D1CDEE74A46D0
:1007700000DA694206A800F075FA06AB93E80700B4
:1007800003AB83E8070050460A9900F056FB8DE85A
:100790000700A0F500501F3800900398002D0ADDD7
:1007A00042F21F014A460844002303A90390684609
:1007B00000F0BFFD09E0A0F500504A461F380023B5
:1007C00003A90390684600F0C9FD8DE80700000406
:1007D000000C03D04FF0FF30410800E01046B8F1A4
:1007E000000F03D00022009215461EE0751E05D4AE
:1007F00000F0B2F9303262556D1EF9D5B3460122D0
:10080000084302D000227F1C04E02078302801D168
:1008100000227F1E002A099784D01DE0112D07DADF
:1008200000F09AF9303262556D1C50EA0102F5D1A0
:10083000084302D00098C8B10EE00021681E05E010
:10084000235C625C63542254401E491C8142F7DBE6
:10085000AB46A81B401E0990002004F80B000B9823
:10086000099AC0F80880C0E9002B7AE711264FF0FA
:10087000000857E72DE9F04F88460446D21D22F0C4
:10088000070191B0D1E90001CDE90A0102F0D8FCDD
:1008900002460B98C00F01D02D2007E02068810789
:1008A00001D52B2002E0202101EAC000032A099093
:1008B00001D0072A05DB03464146204600F092F9A5
:1008C0000BE12078800601D5E06900E00620B8F150
:1008D000650F814606D0B8F1660F18D0B8F1670FE2
:1008E00070D131E00020B9F1110F009001DB11232C
:1008F00001E009F101030AAA01A90CA8FFF7E2FE31
:10090000DDE90C70002609F10105834647E001206E
:100910004B4600904FF000470AAA01A90CA8FFF728
:10092000D1FEDDE90DB00C995D46002610B909F144
:1009300001000D18B9EB050003D4C0F1FF3609F131
:100940000105A5EB09002BE0B9F1010F01DA4FF029
:1009500001090020B9F1110F0090484601DD112373
:1009600000E003460AAA01A90CA8FFF7ABFEDDE9E7
:100970000C704D4600268346207800070AD4AB450C
:1009800000DA5D4601A8012D04DD411911F8011CB2
:10099000302907D04F4502DA17F1040F04DA01209D
:1009A00082460FE06D1EEEE7002F02DCED1B3E4499
:1009B00003E0781CA84200DD7D1CB81B00F1010A91
:1009C0004FF000472078000703D4AA4501DB4FF021
:1009D000FF3A0021B7F1004F0DF143088DF84310A5
:1009E00024D002202B23002F01DA7F422D230A215D
:1009F000021EA0F1010000DC5FB197FBF1FC97FB48
:100A0000F1F201FB1C7C17460CF1300C08F801CD0B
:100A1000EEE7A8F1010003702188090501D5452101
:100A200000E06521A0F1010800F8011C09980FA958
:100A3000A1EB0807FF1D00B10120411901EBEA708D
:100A4000A1693844081A401EA0612078C00602D46B
:100A50002046FFF753FC099828B1D4E901219047BB
:100A6000206A401C20622078C00622D52046FFF76D
:100A700045FC1EE0002E04DBB34502DD01A8805DCD
:100A800000E03020D4E901219047206A401C206218
:100A9000761CAAF101005FEA000A0AD100F054F8BE
:100AA000C0680168405CD4E901219047206A401C7D
:100AB0002062281EA5F10105DCDC07E0D4E9012154
:100AC00018F8010B9047206A401C2062381EA7F1DD
:100AD0000107F3DC2046FFF727FC032011B041E6B5
:100AE00001694A1C02610878704700B58FB0CDE9F2
:100AF00001310021059105497944CDE903101146E2
:100B00006846FFF7B3FC0FB000BD0000E5FFFFFF34
:100B10000A6802F8010B0A60704710B5436913B107
:100B2000AFF3008001E0FFF710FC012010BD127848
:100B300000F124010A7000224A700122EDE71168D9
:100B40004FF0FF32E9E700000048704738130020FB
:100B5000004870471813002030B5B0F10A024FEA80
:100B6000900E71F100034EEA817EB0EB0E0061EB56
:100B700091014FEA101E4EEA017E10EB0E0041EB90
:100B800011114FEA102E4EEA016E10EB0E0041EBF0
:100B900011214FEA104E4EEA014E10EB0E0041EBD0
:100BA0001141401841F100014FEAD00040EA417084
:100BB0004FEAD10110EB80054FEA810444EA9074BA
:100BC00044EB01046D1944EB0404521BA3414FF0A4
:100BD000000348BF0A3200D530BD401C41F100017E
:100BE00030BD00002DE9F0411F4604460326016890
:100BF000072A01F4006004DB08B116A505E016A57C
:100C000003E008B115A500E015A521F01000206053
:100C1000A069C01EA0610FB1401EA0612046FFF771
:100C20006DFB4FB1D4E9012138469047206A401C42
:100C30002062C01C206206E0206AFAE7D4E90121A4
:100C400015F8010B9047761EF8D22046FFF76CFB93
:100C5000BDE8F0814E414E006E616E00494E460087
:100C6000696E66002DE9F047814616468AB0354820
:100C700078440DC88DE80D0032487844801C03ACE0
:100C80000DC884E80D0041F69B300844372190FBE5
:100C9000F1F290FBF1F5A5F1800501FB12041B3C7C
:100CA00002D56442012000E00020DFF898A08046D1
:100CB0000027FA44AAF1BE0A0EE0E0070AD0324645
:100CC000684607EB470101230AEB810100F046FB70
:100CD0008DE8070064107F1C002CEED1194F7F4473
:100CE000AE3F19E0E80715D007EB04100DF1180A24
:100CF00090E80E008AE80E00C068F04201D1981911
:100D000008903246012306A903A800F027FB03AB95
:100D100083E807006D10641C002DE3D14FF0010340
:100D200032466946B8F1000F03A802D000F001FB7B
:100D300001E000F013FBC9E90001C9F808200AB07E
:100D4000BDE8F08758BD0000004870471813002028
:100D50007546FFF7F9FFAE4605006946534620F099
:100D60000700854618B020B5FFF7A2FABDE820407D
:100D70004FF000064FF000074FF000084FF0000B57
:100D800021F00701AC46ACE8C009ACE8C009ACE80A
:100D9000C009ACE8C0098D46704710B50446AFF3F2
:100DA00000802046BDE81040FFF76DBA4FF0013CCF
:100DB00050F8042B51F8043B9A4221D1A2EB0C03CA
:100DC000934313EACC1317D150F8042B51F8043B8A
:100DD0009A4215D1A2EB0C03934313EACC130BD127
:100DE00050F8042B51F8043B9A4209D1A2EB0C03B2
:100DF000934313EACC13DBD04FF00000704700BFE1
:100E0000D01A01BAB1FA81F101F0180122FA01F009
:100E1000CB40C1F12001DBB2C0B2C01A2CFA01F301
:100E2000D11A914311EAC311E6D170470149182044
:100E3000ABBEFEE72600020070475FEA400C08BF29
:100E400091F0000F4FEA8C234FEAC12243EA51513F
:100E50004FEA1C5018BF00F5F0404FEA300018BFB1
:100E600041F000415FEA6C5C00F02980BCF1FF3F7B
:100E700008BF40F080407047130C06BF12044FF0CB
:100E8000100C4FF0000C130E04BF12020CF1080CF2
:100E9000130F04BF12010CF1040C930F04BF920056
:100EA0000CF1020CD30F04BF52000CF1010C1146DF
:100EB0004FF00002A0F11F00A0EB0C00704711F0F2
:100EC000004F08BF704731F000413FF4D5AF0B0C25
:100ED00006BF09044FF0100C4FF0000C0B0E04BFBE
:100EE00009020CF1080C0B0F04BF09010CF1040CF2
:100EF0008B0F04BF89000CF1020CCB0F04BF49001B
:100F00000CF1010CCCF12003A0EB0C0022FA03F34E
:100F100002FA0CF241EA030100F10100704720F0EF
:100F20007F4C80EA030023F07F47ACEB070303F517
:100F30007C5300F0004003F1FF032DE980494FEAA4
:100F4000154B09B44FEA144325EA0B4E24EA034833
:100F50000FF2042606EB132749083E785FEA3202B7
:100F600003FB0667C7F5000707FB06F64FEA543791
:100F70004FEAD64606F1020607FB066CCCF1005C90
:100F80004FEA1C472CEA074C07FB06F40CFB06F55E
:100F900004EB15464FEA961634BF00204FF0004090
:100FA0004FEAD13706FB07FC4FEA1C4C0CFB0BF752
:100FB000D21B03FB0CF761EB07010CFB0EF7B0EB48
:100FC000074072EB17420CFB08F734BFA2EB074255
:100FD000B2EB074261EB17414FEA0C444FEA91072D
:100FE00006FB07FC4FEA1C4C0CFB0BF7B0EBC740B1
:100FF00072EB573203FB0CF734BFA2EBC742B2EBE4
:10100000C74261EB57310CFB0EF7B0EBC70072EB38
:1010100057720CFB08F734BFA2EBC702B2EBC70252
:1010200061EB5771039F4FEA816141EA921104EB32
:10103000CC044FEAD1374FEA826206FB07FC42EA52
:1010400090124FEA80604FEA1C4C0CFB0BF7D21B4E
:1010500003FB0CF761EB07010CFB0EF7B0EB07404D
:1010600072EB17420CFB08F734BFA2EB0742B2EB5E
:10107000074261EB17414FEA8C554FEA910704EBA9
:101080009C2406FB07FC4FEA1C4C0CFB0BF7B0EB57
:10109000C74072EB573203FB0CF734BFA2EBC742D9
:1010A000B2EBC74261EB57310CFB0EF7B0EBC70058
:1010B00072EB57720CFB08F734BFA2EBC702B2EB1E
:1010C000C70261EB577115EB4C254FEA816141EA8C
:1010D00092114FEA82624FEAD13742EA901206FB40
:1010E00007FC44F100044FEA80604FEA1C4C0CFB03
:1010F0000BF7D21B03FB0CF761EB07010CFB0EF7A0
:10110000B0EB074072EB17420CFB08F734BFA2EBC1
:101110000742B2EB074261EB174115EB1C154FEA92
:10112000813141EA92414FEA823242EA90424FEAEB
:1011300080304FEA0C7644F1000448EA03434EEA5B
:101140000B484FF0000EB2EB080C71EB030724BF05
:10115000624639464EEB0E0E4FF0000B001852411E
:1011600049414BEB0B0BB2EB080C71EB03077BF126
:10117000000B24BF624639464EEB0E0E4FF0000BBB
:101180000018524149414BEB0B0BB2EB080C71EBD1
:1011900003077BF1000B24BF624639464EEB0E0E6F
:1011A00051EA020718BF46F0010616EB0E7655F11C
:1011B000000254F1000103D5BDE88901BDE80088B3
:1011C000BDE88901BDE80048B619524141EB010173
:1011D000A3F10103704780807F7E7D7C7B7A7978E4
:1011E000777676757473727171706F6E6E6D6C6CEC
:1011F0006B6A6A696868676666656464636362618E
:101200006160605F5F5E5E5D5D5C5C5B5B5A5A590E
:10121000595858575756565555555454535352527A
:101220005251515050504F4F4F4E4E4D4D4D4C4CD2
:101230004C4B4B4B4A4A4A4949494848484747471B
:101240004746464645454544444444434343434258
:10125000424242414141002B9C4630D477002BD082
:101260001CB54FEA370703B44FF010004FF01001E0
:10127000BAF1000F06D0BCF1000FDCBF40F008004F
:1012800040F008014FF000000FBCBDE810400BF12A
:10129000010BBBF1010F08BF5FEA170722BF12F174
:1012A000010211F101014FF0004143F1000300F090
:1012B000004043EA00007047F9D35708D0E746EAF8
:1012C000064613F1400F4FEA16461FDD13F1200FBB
:1012D000DFBF16430A46002120335B42BED0C3F174
:1012E000200746EA064602FA07F74FEA164646EA9C
:1012F0000706C3F1200722FA03F201FA07F721FAE1
:1013000003F14FF0000342EA0702A7E746EA0206AC
:1013100046EA06464FEA164646EA0106BCBF46EADA
:101320000646360C4FF000034FF000024FF000016C
:1013300094E72DE9804C9A46934670B491E83800C2
:1013400007C831EA400C48BF34EA430C03D5FFF725
:10135000E6FDFFF780FFF0BCBDE8008C2DE9804C76
:101360009A46934670B491E8380007C810F0804F51
:1013700008BF13F0804F03D100F005F8FFF76BFFB3
:10138000F0BCBDE8008C20F07F4780EA030023F02A
:101390007F4C07EB0C03A3F57C5300F00040A3F156
:1013A000FE0392F0000F00F0B38095F0000F00F004
:1013B00077802DE901494FEA11404FEA144621EAAE
:1013C000004800FB06FC24EA064708FB06F607FB7C
:1013D00008F800FB07F718EB06484CEB164C4FEAF1
:1013E000124B18EB07484FEA15464CEB174022EA20
:1013F0000B4E0BFB06FC25EA06470EFB06F607FB29
:101400000EFE0BFB07F71EEB064E4CEB164C4FF097
:1014100000061EEB074E4CEB174B18EB0B0840F188
:10142000000018EB0E0B58EB000840F100008F1A7B
:101430004FF000013CBFC943661B14BFB5EB040C61
:1014400000213CBFC943F61B4FEA17444EEA8E0EFB
:1014500027EA04454FEA1C4704FB07622CEA074CC5
:1014600005FB07F70CFB05F604FB0CFC16EB074627
:1014700042EB174216EB0C4642EB1C421BEB0606F6
:1014800058EB0202414146EA9E0601D5BDE80189BA
:10149000B619524141EB0101A3F10103BDE80189F5
:1014A0004FEA14454FEA114724EA054621EA074C62
:1014B00005FB07F406FB07F70CFB06F105FB0CFC2C
:1014C00011EB074144EB17444FEA124711EB0C4173
:1014D00044EB1C4422EA074C05FB07F206FB07F726
:1014E0000CFB06F605FB0CFC16EB074642EB17421D
:1014F00016EB0C4642EB1C456A1854F1000148BF3C
:101500007047B619524141EB0101A3F10103704745
:1015100095F0000F37D04FEA11424FEA144721EA05
:10152000024624EA074C02FB07F106FB07F70CFB17
:1015300006F402FB0CFC14EB074441EB17414FEAA5
:10154000154714EB0C4441EB1C4125EA074C02FB08
:1015500007F506FB07F70CFB06F602FB0CFC16EB87
:10156000074645EB174516EB0C4645EB1C42121996
:1015700051F1000148BF7047B619524141EB0101DA
:10158000A3F1010370474FEA14454FEA114724EADB
:10159000054621EA074C05FB07F106FB07F70CFBA4
:1015A00006F24FF0000605FB0CFC12EB074241EB84
:1015B000174112EB0C4251EB1C4148BF7047921887
:1015C00041EB0101A3F101037047FEE77047000002
:1015D000154991F82F20012A04BFD1F80C31C1F828
:1015E000083107D0022A0CBFD1F81031D1F81431DC
:1015F000C1F8083101284FF090434FF0040008BFB4
:1016000098620FD09861D1F80801022A14BF401DDA
:10161000401CC1F80801B0F5B47FC4BFA0F5B47098
:10162000C1F8080100F04CBF00000020264910B4AA
:1016300091F8AC0700234A1C4FF0010C92F8AC273C
:101640000244881C90F8AC070244C81C90F8AC0710
:101650000244081D90F8AC0714181C4A92F8AC0715
:1016600091F8AC172044C01D10F0FF00A2F1020455
:1016700094F8AC470C4492F8AC1704EB01021449FF
:1016800091F8AC170A44134991F8AC170A4412496F
:1016900091F8AC170A44114991F8AC17114401F1C3
:1016A0000901C9B208BF2120002908BF634603D041
:1016B000FF2908BF012200D000221A4318BF4D2085
:1016C00040EA012010BC704700F0FF1F0EF0FF1F22
:1016D00046F0FF1F47F0FF1F50F0FF1F51F0FF1FA4
:1016E00002488168027811448160704758020020E6
:1016F000FEE70000F0B500238027134C134E05468B
:101700005FF0400215F0800F14BF2760376096200D
:1017100003F0F6FB2260962003F0F2FB32606806CD
:10172000050E581CC3B2082BECD3962003F0E8FB3F
:101730002260962003F0E4FB05480068012121EABD
:10174000D0103260F0BD00001804004828040048A2
:10175000100400482DE9F0430024DFF844800646D9
:10176000B3274FF0100900BF4FF40040C8F828001D
:1017700004F15900C5B2384608F0D2FD09EB151046
:1017800008F0CEFD05F00F0008F0CAFDFF2008F0BC
:10179000E3FD601CC4B2B442E6D9BDE8F0830000AA
:1017A000000400482DE9F04100240F4FB3264FF00C
:1017B000100800BF4FF40040B86204F15900C5B2F0
:1017C000304608F0ADFD08EB151008F0A9FD05F056
:1017D0000F0008F0A5FD002008F0BEFD601CC4B29B
:1017E000272CE7D3BDE8F081000400484FF4407196
:1017F00091FAA1F100222048B1FA81F122FA01F117
:1018000000EB81009446016B21F4F86141F4807192
:1018100001634FF0A040D0F8081141F00101C0F879
:1018200008111346D0F8081141F00401C0F808115E
:10183000D0F8001111F0080FFAD0D0F84011521F63
:101840000A44591CCBB2C82BECD3002A12DB0B483C
:1018500090F82F00022806D00948C0FB02C25011A0
:10186000A0EBE27070470748C0FB02C25011A0EB2A
:10187000E27070470022EAE70001005000000020FB
:1018800089888888932449920F49CA6812F0010F09
:10189000FBD1CA6812F0200F4FF0200218BFCA60B7
:1018A0000B6943F002030B614861086940F0400096
:1018B0000861C86810F0200FFBD0CA60086920F0EA
:1018C00002000861704700000020024070B4174B0E
:1018D000D3F80CC01CF0010FFAD1D3F80CC04FF0B4
:1018E00020051CF0200F18BFDD60D3F810C04CF0AD
:1018F000010CC3F810C00024002A10D9061910F8F2
:1019000004C076780CEB062C21F804C0D3F80CC088
:101910001CF0200FFAD0DD60A41CA242EED818699A
:1019200020F00100186170BC7047000000200240E8
:1019300010B44FF0A04C4A68DCF808400023DCF8F3
:1019400008C144EA0C0C1CF0010F18BF012302D09F
:1019500010BC18467047DFF828C052B10C6822430B
:10196000D1E9024121431143826802EA0C0211438A
:1019700004E08268096802EA0C0211438160E7E72B
:10198000E030FCFF8368002213F0010F18BF012232
:1019900001D010467047D1E9003C43EA0C03896846
:1019A000D0F80CC02CF0380C2CF4804C41EA0C011F
:1019B0001943C160EDE7000030B44B68D0F808C0AF
:1019C00000221CF0010F18BF012202D030BC1046CB
:1019D0007047002BDFF848C00B680ED08C6823439B
:1019E000D1E903452C4323434C692343C46804EAEB
:1019F0000C0C43EA0C03C3600BE0CC682343D1E931
:101A000004452C432343C46804EA0C0C43EA0C034A
:101A1000C3604968036B23F00F0319430163D5E7E3
:101A20003CC0F0FF30B401F0100101245368056898
:101A30004FF0000C8C40AC4308BF4FF0010C1BD0A2
:101A40007BB114682343D2E9024222431A4303685C
:101A50008A4040F6FA7404FA01F123EA01011143C5
:101A600009E00368FA248C40A3431468D268224337
:101A700002FA01F11943016030BC60467047000072
:101A80002DE9F0030A6892FAA2F3B3FA83F3DA407D
:101A90007ED001250F244FF0030C00BF0E6805FA1D
:101AA00003F2324075D04E68012E18BF022E22D1AB
:101AB0008E68D0F8088092FAA2F7B7FA87F74FEA53
:101AC00047070CFA07F728EA070792FAA2F8B8FACC
:101AD00088F84FEA480806FA08F647EA06068660DC
:101AE000CF680E68D0F8048028EA060806FB07F6DF
:101AF00048EA060646600E69D0F80C8092FAA2F712
:101B0000B7FA87F74FEA47070CFA07F728EA0707FB
:101B100092FAA2F8B8FA88F84FEA480806FA08F6E6
:101B200047EA0606C6604E68022E36D192FAA2F641
:101B3000B6FA86F6082E15D24E69076A92FAA2F80E
:101B4000B8FA88F84FEA880804FA08F827EA08087B
:101B500092FAA2F7B7FA87F7BF00BE4048EA060636
:101B600006621AE04F69D0F82480160A96FAA6F9A0
:101B7000B9FA89F94FEA890904FA09F996FAA6F639
:101B8000B6FA86F6B60028EA090807FA06F601E072
:101B90001DE017E048EA060646624E68076892FABA
:101BA000A2F8B8FA88F84FEA48080CFA08F892FA4E
:101BB000A2F2B2FA82F2520027EA080706FA02F20B
:101BC0003A4302600A685B1CDA407FF467AFBDE805
:101BD000F003002070474FF47A71B0FBF1F0411E22
:101BE0004FF0E020416100218161052101617047D2
:101BF0000149086070470000640200200A7B8B687E
:101C00001A434B6822F480621A430B6822F4006284
:101C10001A43CB8922F480521A430B6922F40052F2
:101C20001A434B6A22F480421A434B6922F4702211
:101C30001A43A0F18043B3F596330BD10B6A22F41B
:101C400070021A438B6922F080721A43C96922F02C
:101C500000720A43426400207047000070B40268BA
:101C60001D4B1E4E98421CBFB0F1804FB04205D1B3
:101C7000D1F804C022F0700242EA0C02DFF860C022
:101C8000184C194D984218BFB0F1804F07D0B042A0
:101C900018BF604503D0A04218BFA84204D1CE6847
:101CA00022F4407242EA060202608A68C2620A882E
:101CB0008262984218BF604503D0A04218BFA84274
:101CC00001D109690163416941F00101416170BCC1
:101CD0004FF0000070470000002C0140000400405D
:101CE0000040014000440140004801402DE9F0035C
:101CF00001270023DFF8F4C2BD4CBE4DBE4EB1F546
:101D0000805F00F0DB8008DC012910D010294FD063
:101D1000B1F5807F7DD000F065B9B1F5803F00F06E
:101D2000FF80B1F5801F00F02D8100F05BB9016AE2
:101D300021F001010162076A4168D0F81880D2F8E9
:101D4000009028F0730828F4803848EA0908D2F88F
:101D5000109027F0020747EA0907D2F8049027F00D
:101D6000010747EA0907604518BFA04203D0A8420F
:101D700018BFB04215D1546927F0080C4CEA840C06
:101D800094682CF0040C4CEA8407D2F818C021F4B3
:101D9000807141EA0C01D2F81CC021F4007141EAC3
:101DA0004C014160C0F81880D1684163076241E08E
:101DB000016A21F010010162016A4768D0F81880B9
:101DC000D2F8009028F4E64828F0807848EA0928FC
:101DD000D2F8109021F0200141EA0911D2F80490C4
:101DE00021F0100141EA0911604518BFA04203D05B
:101DF000A84218BFB04217D1D2F814C021F0800118
:101E000041EA8C11D2F808C021F0400141EA8C115E
:101E100000E011E0946927F4806C4CEA840CD469EA
:101E20002CF4006C4CEAC4074760C0F81880D268F4
:101E3000826301621F46D5E0016A21F4807101626C
:101E4000076A4168D0F81C80D2F8009028F0730827
:101E500028F4803848EA0908D2F8109027F400776F
:101E600047EA0927D2F8049027F4807747EA092740
:101E7000604518BFA04203D0A84218BFB04215D198
:101E8000546927F4006C4CEA842C94682CF4806C20
:101E90004CEA8427D2F818C021F4805141EA0C1191
:101EA000D2F81CC021F4005141EA4C114160C0F845
:101EB0001C80D168C16307621F4693E0016A21F468
:101EC00080510162076A4168D0F81C80D2F8009006
:101ED00028F4E64828F0807848EA0928D2F81090DB
:101EE00027F4005747EA0937D2F8049027F48057BF
:101EF00047EA0937604518BFA04203D0A84218BF7F
:101F0000B04205D1D2F818C021F4804141EA8C11C9
:101F10004160C0F81C80D168016407621F4661E01F
:101F2000016A21F480310162076A416DD2F80080B4
:101F300021F0700121F4803141EA0801B2F81080EB
:101F400027F4003747EA0847B2F8048027F48037BF
:101F500047EA0847604518BFA04203D0A84218BF0F
:101F6000B04208D1D0F804C094692CF4803C4CEA0B
:101F7000042CC0F804C04165D168826D8165076298
:101F80001F462FE0016A21F480110162076A416D4A
:101F9000D2F8008021F4E04121F0807141EA08216B
:101FA000B2F8108027F4001747EA0857B2F8048007
:101FB00027F4801747EA0857604518BFA04203D0AE
:101FC000A84218BFB04208D1D0F804C094692CF4DC
:101FD000802C4CEA842CC0F804C04165D168C165EE
:101FE00007621F463846BDE8F0037047002C0140E9
:101FF0000040014000440140004801404FF0E02112
:1020000081B00A690092B0F1FF3F18BF401C0A6915
:1020100012F4803F18BF401E0028F8D101B070476D
:10202000FEE7FEE730B4002201256C4903230724B4
:102030004FF0050C05280FD24D708B7081F803C04E
:102040000C714A718A71CA710A724A728A72CA72B2
:102050000A734A7300F0BEB810D14A708D70CB700D
:1020600081F804C04C718A71CA710A724A728A720C
:10207000CA720A734A738A7330BC7047062822D02A
:10208000072831D0082840D009284FD00A285ED030
:102090000B286DD00C287ED00D287BD00E281CBFBD
:1020A00030BC70474A708A70CA700A714A718A716E
:1020B000CA710A724A728A72CD720B7381F80DC0AE
:1020C0008C7330BC70474A708A70CD700B7181F888
:1020D00005C08C71CA710A724A728A72CA720A7316
:1020E0004A738A7330BC70474A708A70CA700D7127
:1020F0004B7181F806C0CC710A724A728A72CA7238
:102100000A734A738A7330BC70474A708A70CA7007
:102110000A714D718B7181F807C00C724A728A7214
:10212000CA720A734A738A7330BC70474A708A70E5
:10213000CA700A714A718D71CB7181F808C04C72F6
:102140008A72CA720A734A738A7330BC70474A70C3
:102150008A70CA700A714A718A71CD710B7281F8E6
:1021600009C08C72CA720A734A738A7330BC704792
:102170004A708A70CA700A714A718A71CA710D7286
:102180004B7281F80AC0CC720A734A738A7330BCEE
:10219000704700E010E04A708A70CA700A714A7194
:1021A0008A71CA710A724D728B7281F80BC00C73FE
:1021B0004A738A7330BC70474A708A70CA700A7159
:1021C0004A718A71CA710A724A728D72CB7281F831
:1021D0000CC04C738A7330BC704700008B02002027
:1021E00030B5092888BF0920062101EB4004C0F161
:1021F0000A05E1B2F62015FB00F040B207F054FFEB
:1022000005EBC500E1B2BDE8304040B207F04CBF7D
:10221000274910B40860274991F82F20022A0CBFE3
:1022200020236023CB72244B401C93FBF0F0CB7A2D
:102230004FF0000C90FBF3F0C1F82C0191F828400E
:1022400000FB03F0022C08D21C4B83FB003043112F
:10225000A3EBE070C1F8840007E0194BC3FB00C09A
:102260004311A3EBE070C1F8840020F01F00C1F817
:102270008400012A0FD0022A14D0DFF848C00022BF
:102280006346E0FB0C32D009C1F888001C20C1F87D
:102290008C0010BC70470C4AA2FB00208009C1F8DA
:1022A0008800F3E7094AA2FB00204009ECE70000A0
:1022B0002C0400400000002000D8B805ED73484D04
:1022C000932449924F09F2941F85EB51DB81B97633
:1022D000704770472DE9F0475C4F2DED028B394672
:1022E00097F82F00D1F80841012808BFC7F80C4122
:1022F00003D0022808BFC7F81041FD7A4FF4B47824
:102300009FED538A002D1CBFDFF84891002621D095
:10231000F87AB8FBF0F000FB0640B0F5B47FA8BF38
:10232000A0F5B47000EE100AB8EEC00A20EE080A5C
:1023300010EE100A08F0F8FE41EC100B01F060FC02
:1023400051EC100B08F02EF949F8040B6D1E06F144
:102350000106DDD1FC7AD7F80891002C1CBF3E4E57
:10236000002521D0F87AB8FBF0F000FB0590B0F51D
:10237000B47FA8BFA0F5B47000EE100AB8EEC00A92
:1023800020EE080A10EE100A08F0CEFE41EC100B09
:1023900001F0EEF951EC100B08F004F946F8040BCB
:1023A000641E05F10105DDD12C4D0024D7F8108104
:1023B000202600BF04EB440000EBC4004044B0F50D
:1023C000B47FA8BFA0F5B47000EE100AB8EEC00A42
:1023D00020EE080A10EE100A08F0A6FE41EC100BE1
:1023E00001F00EFC51EC100B08F0DCF8641C45F811
:1023F000040B761EDED1D7F81071194D002420266B
:1024000004EB440000EBC4003844B0F5B47FA8BF2F
:10241000A0F5B47000EE100AB8EEC00A20EE080A6B
:1024200010EE100A08F080FE41EC100B01F0A0F94C
:1024300051EC100B08F0B6F8641C45F8040B761E3E
:10244000DED1BDEC028BBDE8F0870000000000206B
:102450004BFA8E3C9C0200201C0400209C050020AE
:102460001C070020F0B5403045B20820A0EBD10495
:1024700001F00700802121FA00F608020E49886267
:10248000681EC7B204F1AF00C0B207F049FF1020C8
:1024900000EB171007F044FF07F00F0007F040FFB4
:1024A000064805EB45010144085D3043C0B20855BC
:1024B000BDE8F04007F050BF00040048981100202C
:1024C0002DE9F047A14F4FF4B4792DED028B394639
:1024D00097F82F00CC7A9FED9E8A032873D0D7F807
:1024E0000881002C1CBF9B4E002521D0F87AB9FB37
:1024F000F0F000FB0580B0F5B47FA8BFA0F5B47084
:1025000000EE100AB8EEC00A20EE080A10EE100A1B
:1025100008F00AFE41EC100B01F072FB51EC100BBD
:1025200008F040F846F8040B641E05F10105DDD102
:10253000FC7AD7F80881002C1CBF874E002521D0DB
:10254000F87AB9FBF0F000FB0580B0F5B47FA8BFC6
:10255000A0F5B47000EE100AB8EEC00A20EE080A2A
:1025600010EE100A08F0E0FD41EC100B01F000F94C
:1025700051EC100B08F016F846F8040B641E05F138
:102580000105DDD197F82F009FED740A01287BD05B
:10259000022897F83E004FF0640110FB01F074D060
:1025A00000EE100A97F83D004621F8EE400A10FBB5
:1025B00001F0BDEC028B00EE100ABDE8F047B8EE6A
:1025C000400A07F049BED7F80C81002C1CBF614EB1
:1025D000002521D0F87AB9FBF0F000FB0580B0F5BA
:1025E000B47FA8BFA0F5B47000EE100AB8EEC00A20
:1025F00020EE080A10EE100A08F096FD41EC100BD0
:1026000001F0FEFA51EC100B07F0CCFF46F8040B7A
:10261000641E05F10105DDD1FC7AD7F80C81002C90
:102620001CBF4D4D002621D0F87AB9FBF0F000FB1D
:102630000680B0F5B47FA8BFA0F5B47000EE100A14
:10264000B8EEC00A20EE080A10EE100A08F06CFD81
:1026500041EC100B01F08CF851EC100B07F0A2FFCD
:1026600045F8040B641E06F10106DDD13C4D002443
:10267000D7F81081202600BF04EB440000EBC40013
:102680004044B0F5B47F01E042E054E0A8BFA0F5BB
:10269000B47000EE100AB8EEC00A20EE080A10EE80
:1026A000100A08F041FD41EC100B01F0A9FA51ECC1
:1026B000100B07F077FF641C45F8040B761EDBD186
:1026C000284C0025D7F81081202600BF05EB4500D7
:1026D00000EBC5004044B0F5B47FA8BFA0F5B470CE
:1026E00000EE100AB8EEC00A20EE080A10EE100A3A
:1026F00008F01AFD41EC100B01F03AF851EC100B08
:1027000007F050FF6D1C44F8040B761EDED139E74C
:1027100097F83D00462110FB01F0BDEC028B00EE66
:10272000900ABDE8F047B8EE601AF0EE400AB0EE4D
:10273000410A07F091BDBDEC028B00EE900ABDE8A6
:10274000F047F8EE600A07F087BD000000000020A7
:102750004BFA8E3C9C0200201C040020000000006C
:102760009C0500201C0700202DE9F047082688461C
:102770003E28CCBF0121002110F13E0FB4BF012241
:102780000022114318BFBDE8F08740303B4F4FF4A3
:102790000041C0B2B962441E4FF0B70A04F0FF090D
:1027A000504607F0BDFD102000EB1915284607F034
:1027B000B7FD09F00F0007F0B3FD002007F0CCFDD6
:1027C0007801B8624FF0B609484607F0A9FD2846DF
:1027D00007F0A6FD04F00F0007F0A2FD002007F0AF
:1027E000BBFD7801B862B52007F09AFD284607F0D6
:1027F00097FD04F00F0007F093FD002007F0ACFDFB
:10280000B8F1070F0FD97801B862504607F088FD7C
:10281000284607F085FD04F00F0007F081FDFF203A
:1028200007F09AFD0726B8F10F0F10D94FF40040BA
:10283000B862484607F074FD284607F071FD04F0C1
:102840000F0007F06DFDFF2007F086FD06264FF410
:102850000040B86206F1AF00C0B207F061FD284643
:1028600007F05EFD04F00F0007F05AFD044908F080
:102870000700085CBDE8F04707F06EBD00040048A3
:1028800068020020FEF72CBF70B53A48016821F0BD
:10289000070141F002010160016801F0070102290E
:1028A000FAD1354C206840F480302060206810F464
:1028B000003FFBD0606A40F001006062606A10F087
:1028C000020FFBD02D48016841F480710160206A3D
:1028D00000F44070B0F5007F0DD0206A40F48030E5
:1028E0002062206A20F480302062206A20F4407048
:1028F00040F400702062206A40F40040206260686A
:1029000020F4741141F424114FF480306160E16AC5
:1029100060F30301E162206840F08070206020686D
:1029200010F0007FFBD0606820F0F000606060680D
:1029300020F4E06040F480606060606820F46050E3
:102940006060606820F0030040F002006060606832
:1029500000F00C000828FAD1094D2846FFF73BF992
:102960002846FFF745F9E06A20F4F87040F49070CB
:10297000E06270BD00200240001002400070004084
:1029800000D8B8050248016841F470010160704741
:1029900088ED00E02DE9F0474FF080416FF0010035
:1029A0000861FD4D287A00281CBF401E287295F84A
:1029B00022004FF0010A00281CBF95F82F000328C1
:1029C00040F0FA80DFF8D493EB7A4FF0000709F576
:1029D000C0782BB3A9F10400A8F1040113F0010F92
:1029E00009D090ED010AB8EEC00A81ED010A40F865
:1029F000047F01F104015A0812D000BF90ED010AD2
:102A0000B8EEC00A81ED010A476090ED020AB8EE07
:102A1000C00A81ED020A083140F8087F521EEDD14C
:102A2000FF20AF70002485F82200002B12D900BFD0
:102A300008EB840695F82C1096ED000A204602F06B
:102A4000DFFF86ED000A49F82470601CC4B2E87A02
:102A5000A042EDD89FEDD20A394685ED4C0AC5E972
:102A60002B7795F82F203846032A7DD0EB7A2BB3AD
:102A7000CC4AA2F28474A2F2046C00BF92ED000A68
:102A8000D5ED4C0A5B1E40EE000AC5ED4C0AF2EC97
:102A9000010AB4EC010A20EE800ABDEEC00A10EE75
:102AA000106ABCEC010A304420EE800ABDEEC00A78
:102AB00010EE106A3144E1D1C5E92B01E87AD5ED79
:102AC0004C0A00EE100AB8EE401A80EE810A10EEB1
:102AD000100A08F029FB41EC100B01F0BDF951EC94
:102AE000100B07F05FFD00EE100A85ED4C0AD5EDE6
:102AF000220AF8EE600A80EE201ABCEEC10A85EDCB
:102B00001F0AD5F8AC20C5F8C420D5F8B010C5F818
:102B1000C810E879012803D095F8280002287CD253
:102B2000C5F8B4A0C5F8B8A0D5F8D000D5F8B8302D
:102B30008242CCBF1844C01AC5F8D000D5F8CC00EA
:102B4000D5F8B4308142CCBF1844C01AC5F8CC00C7
:102B500095F8210000281CBF85F82170C5E93312C3
:102B6000D5F8D000101A00E02AE0C5F8C400D5F866
:102B7000CC20891AC5F8C81095F8281001297CD0F6
:102B800000EE100AB8EEC00A02F070FDBDEEC00AF9
:102B900085ED390A95ED320AB8EEC00A02F016FE4C
:102BA000BDEEC00A85ED3A0AD5F8E400C5F8BC00D0
:102BB000D5F8E800C5F8C00085F838A0BDE8F08772
:102BC000EB7A0022002B84BFDFF8DCC10CF5C07467
:102BD0002ED900BF08EB820695ED4C0AD6ED000A0F
:102BE00001EE100A0CEB820600EEA00AB8EEC11A44
:102BF00085ED4C0A96ED000A04EB820600EE801A81
:102C0000BDEEC10A96ED001A10EE100A00EE101A81
:102C1000B8EEC00A00EE810A00E040E0BDEEC00A56
:102C2000921CD2B210EE101A9A42D3D3C5E92B01EE
:102C30005E4A95ED2B0A00EE901A012002F5C07352
:102C400008EB800C00F01F019CED001A08EB810CD2
:102C500095ED4C2ADCED001A02EB810CB8EEC00AAF
:102C600001EE212A03EB810185ED4C2ADCED001AEF
:102C700001EE210ABDEEC00A00E027E0F8EEE00A0E
:102C8000D1ED001A801CC0B241EE210A6028FDEE91
:102C9000E00AD5D385ED2B0AC5ED2C0A0EE7D5F851
:102CA000D000801A48BF404200EBD0700AEB6000B1
:102CB000C5F8B800D5F8CC00401A48BF404200EB38
:102CC000D0700AEB6000C5F8B4002DE795F83B1012
:102CD000012904D0022917D003292AD03DE000EEB3
:102CE000100AB8EEC00A02F0A5FABDEEC00A85EDE2
:102CF000390A95ED320AB8EEC00A02F06FFBBDEE5C
:102D0000C00A85ED3A0A28E000EE100AB8EEC00AC3
:102D100002F0D2FABDEEC00A85ED390A95ED320A0D
:102D2000B8EEC00A02F09CFBBDEEC00A85ED3A0A7F
:102D300013E000EE100AB8EEC00A02F0FFFABDEE92
:102D4000C00A85ED390A95ED320AB8EEC00A02F0E4
:102D5000C9FBBDEEC00A85ED3A0A95F82D0003289F
:102D600026D0022839D001287FF41EAF95ED390A0C
:102D7000B8EEC00A02F0AAFCBDEEC00A85ED390A21
:102D800095ED3A0AB8EEC00A02F050FDBDEEC00A59
:102D900085ED3A0A08E7000000000020A0080020A6
:102DA00000000000200A00209C0200209C0500205A
:102DB00095ED390AB8EEC00A02F008FCBDEEC00A73
:102DC00085ED390A95ED3A0AB8EEC00A02F0AEFC7C
:102DD000BDEEC00A85ED3A0AE6E695ED390AB8EE91
:102DE000C00A02F043FCBDEEC00A85ED390A95ED3C
:102DF0003A0AB8EEC00A02F0E9FCBDEEC00A85ED61
:102E00003A0AD1E6234810B44FF0000CC0F800C0D5
:102E100021498878CA7A401C904228BF00208870D7
:102E20001E4A1F4B32F810201A6091F82F401D4A9D
:102E30009B06032C1CD091F82240002C04BF10BC30
:102E4000704752F820401B6C2344A3F2F17342F800
:102E50002030D1F88000401CC1F88000D1F88420D7
:102E6000904224BF81F822C0C1F880C010BC7047D6
:102E700052F82010D3F840C010F0010F6144A1F2C5
:102E8000F27142F8201014BF40208020186310BC5B
:102E9000704700001004004000000020600C00207B
:102EA00014740040A00800200B496FF00100086175
:102EB0000A48017A002918BF704790F8461011F0AF
:102EC000010F01F1010180F84610054914BF0020EF
:102ED000D0F8A000086070470010004000000020FB
:102EE00008740040424810B4417A1822494202EB6B
:102EF000C12202F1006202F5704292F8002C80F8C3
:102F00003420052202EBC12202F1006202F5704278
:102F100092F8002C80F83020062202EBC12101F14A
:102F2000006101F5704191F8001C80F82C1090F8B8
:102F30002E100A2248F20104002908BFC0F82041DF
:102F40002FD0012904BF48F21F01C0F8201128D05A
:102F500001234FF0040C022926D048F20F04032964
:102F600001BFC0F82041437610BC7047042923D02C
:102F7000052928D0062934D007291CBF10BC70476A
:102F800048F20301C0F820110C214176D0F8081155
:102F90000A29ACBF0A3901F5AF71C0F8081110BC9D
:102FA0007047427610BC7047C0F8204180F819C0C5
:102FB00080F8343010BC704748F25F01C0F820112F
:102FC000427610BC7047C0F8204180F819C0032138
:102FD00080F83B10062180F82C1080F8303010BCAF
:102FE000704749F6DF01C0F82011427610BC7047E7
:102FF000000000204FF4407292FAA2F2144900201F
:10300000B2FA82F2D04000B501EB8000016B21F4EE
:10301000F86141F4407101634FF0A042D2F8080119
:1030200040F00100C2F80801142002F5847201F09A
:1030300067FF106840F0040010601A2001F060FF84
:10304000906B044991F8361090FBF1F000BD000040
:103050000001005000000020FEE7000070B50446AB
:1030600001F0F6FE26A12948FDF734F9274A14217C
:10307000032002F06DF84FF47A7001F0B9FE012CD4
:1030800008BF07F0F9F9224922484160224941600E
:10309000224C2046FEF7F8FB022221462048FEF78C
:1030A00015FC204C204D607A404205EBC020FEF715
:1030B000EBFB607A1022404205EBC02104F2411084
:1030C000FEF704FC607A1949404201EBC02104F28A
:1030D0004115102205F11000FEF7F8FB607A144943
:1030E000404201EBC021082205F12000FEF7EEFB73
:1030F0004FF4FA70FEF782FFBDE8704001F0A8BE01
:1031000020205752495445202120200074020020DD
:103110002301674500200240AB89EFCD00DC0008A9
:10312000090000200000002000FC000810FC00083E
:1031300020FC0008144910B5124A4A60134A4A603C
:10314000012813D1124901F239100A7D4270CA7C5C
:103150008270B1F89420130AC3704271B1F89820BC
:10316000130A0371827191F82610C171094C20462F
:10317000FEF78AFB2146BDE8104008220648FEF70C
:10318000A5BB00002301674500200240AB89EFCDBD
:103190000000002000D40008390100202DE9F04390
:1031A000244E8027884681463760962001F0A8FE8D
:1031B00040243460962001F0A3FE1F4A10681F4D82
:1031C00010F0800F0BD12C60962001F099FE346036
:1031D000962001F095FE106810F0800FF3D02F605C
:1031E000962001F08DFE2C60962001F089FE4FF4B0
:1031F0007A7001F085FE5820FEF77CFA4FF47A7061
:1032000001F07EFE4846FEF775FA4FF47A7001F041
:1032100077FE4046FEF76EFA2F60962001F070FEB2
:103220003460962001F06CFE3760BDE8F0439620D4
:1032300001F066BE18040048100400482804004845
:1032400003B401984100009850EAC12018BF04203F
:103250004A0D18BF40F0010040F2FF72B2EB515F1F
:1032600008BF40F00200012808BF052002B07047E7
:103270004100080218BF04200A0E18BF40F00100E8
:103280004FF07F4232EA010108BF40F002000128FE
:1032900008BF05207047000070B59B482DED020B5C
:1032A0002DED068B079D25F00044A04218DC9748C1
:1032B000844202DC0AD1069840B19DED060BBDECBC
:1032C000068B02B0BDE8704001F0EEBB002DCCBF14
:1032D0009FED8F0B9FED900BBDEC068B02B070BD88
:1032E0008F48A04215DD8F48A042D8BF4FF0FF3471
:1032F00058DD9DED060B51EC100BFFF7A1FF0428E4
:1033000008BF01F0F5FB9DED060BBDEC068B02B08E
:1033100070BD9DED060B51EC100B01F07FFFCDE968
:10332000060181489FED828BA0423CDD8248A0428D
:103330001FDD00249FED82AB9DED060B53EC1A2B95
:1033400051EC100B07F060F99DED060B41EC190BE9
:1033500053EC1A2B51EC100B07F026FC53EC182BF6
:1033600007F0F8FD53EC192B07F002FACDE906013E
:1033700049E09DED060B012453EC182B51EC100B8A
:1033800007F042F99DED060B41EC190B53EC182B9D
:1033900051EC100B07F0DEFD53EC192B07F0E8F9A8
:1033A000CDE906012FE06848A0421FDD02249FED11
:1033B000689B9DED060B53EC192B51EC100B07F09D
:1033C000F3FB53EC182B07F01FF99DED060B41ECB6
:1033D000180B53EC192B51EC100B07F0BBFD53EC01
:1033E000182B07F0C5F9CDE906010CE09DED060BA1
:1033F000032453EC102B9FED580B51EC100B07F0EE
:10340000B7F9CDE906019DED060B53EC102B51ECFD
:10341000100B07F0C9FB41EC180B53EC182B07F00D
:10342000C3FB41EC190B4E480621B0EE490AF0EE01
:10343000690A784401F064F853EC182B51EC100B36
:1034400007F0B2FB41EC180B4648B0EE490AF0EE2B
:10345000690A0521784401F053F853EC192B51EC1B
:10346000100B07F0A1FB41EC100B51EC180B53ECC7
:10347000102B002C0EDA07F0C7F89DED061B53EC5D
:10348000112B07F091FB9DED061B53EC112B07F060
:1034900089FC35E007F0B8F89DED061B53EC112BC5
:1034A00007F082FB41EC100B2F48784400EBC4007E
:1034B00090ED001B51EC100B53EC112B07F04AFD63
:1034C0009DED061B53EC112B07F044FD41EC100B56
:1034D0002648784400EBC40090ED001B51EC100B23
:1034E00053EC112B07F05EFC41EC100B002DA2BF3A
:1034F000BDEC068B02B070BD51EC100B07F046F826
:1035000041EC100B01E70000000010440000F07FC8
:10351000182D4454FB21F93F182D4454FB21F9BFC9
:103520000000DC3F0000203E0000F33F00000000F0
:10353000000000000000F03F0000E63F0000000037
:103540000000000000000040008003400000000078
:10355000000000000000F83F000000000000F0BF85
:1035600042930000F8920000829200003A9200001C
:1035700070B56F4E2DED040B2DED048B82B0DDF890
:1035800024C0DDE907235C422CF000411C4341EAE2
:10359000D474069D22F00040B44205D86C422C43FE
:1035A00040EAD474B4420BD99DED081B9DED060B87
:1035B00002B0BDEC048B04B0BDE8704001F07EBAEF
:1035C000ACF14054A4F17F641C430BD0022404EA04
:1035D000AC7444EAD27405439FED578B9FED582B92
:1035E00007D015E09DED060B51EC100B01F055FBDB
:1035F00042E0002C11BF012C9DED060B02B0BDEC8A
:10360000048B04BF04B070BD022C38D0032C3BD017
:103610000B439FED4D1B9FED4E0B0AD0B14218D1CD
:10362000B04209D121F0804120F0804009910790FB
:103630000FE0002A15DA10E0474B7B44002C08BF4E
:1036400093ED000B0DD0012C10D0022C17D0032CC1
:103650001AD0B0421DD1002A03DAB0EE410AF0EED2
:10366000610A02B0BDEC048B04B070BD93ED000B99
:1036700051EC100B06F08AFF41EC100BF1E7B0EEB5
:10368000480AF0EE680AECE7B0EE420AF0EE620A91
:10369000E7E7401A00159FED329B3C28C8BF8DED2F
:1036A000000B17DCBCF1000FBCBF10F13C0F8DED1F
:1036B000009B0FDB9DED080B53EC102B9DED060BD3
:1036C00051EC100B07F054F801F0A8FD01F0E5FAF9
:1036D000CDE90001B4B1012C10D0022C9FED220BDA
:1036E00053EC102B9DED000B51EC100B19D007F093
:1036F00031FC53EC182B07F02DFCBDE7019880F04E
:10370000004001909DED000B53EC192B51EC100B78
:1037100007F086F904BF0220FCF774FF9DED000B53
:103720009FE707F017FC53EC182B07F03BFBA3E7D0
:103730000000F07F00000000182D4454FB210940D8
:10374000182D4454FB2109C0182D4454FB21F9BF06
:10375000182D4454FB21F93F9A910000000000000D
:103760000000000000000000075C143326A6A13C06
:1037700010B52F499FED2C1B2DED020B84B0059841
:1037800020F000408842D8BF9DED040B2DDD294973
:10379000884209D1049840B94FF00100FCF732FF8C
:1037A00001F096F906B010BD05DB9DED040B01F0AC
:1037B0007BF906B010BD68469DED040B00F0CCFB14
:1037C00010F0030004BF9DED021B9DED000B0CD01B
:1037D00001280ED09DED021B9DED000B022817D095
:1037E000012000F009FF06B010BD00F0D1FD06B0C9
:1037F00010BD9DED021B9DED000B012000F0FCFEB5
:1038000051EC100B06F0C2FE06B041EC100B10BDDF
:1038100000F0BEFD51EC100B06F0B8FE06B041EC16
:10382000100B10BD000000000000000000000000B0
:10383000FB21E93F0000F07F70B5D94B00242DED4E
:10384000020B2DED108BDDE91010984205DA20F007
:1038500000429A4201D809D141B19DED100BBDEC57
:10386000108B02B0BDE8704001F01EB9B0F5801FAA
:1038700026DA11430BD0002813DA0120FCF7C2FE30
:10388000BDEC108B02B0BDE8704001F021B9022000
:10389000FCF7B8FE01F0F0F851EC100B06F076FEE4
:1038A0009EE06FF035049FEDC00B53EC102B9DEDA7
:1038B000100B51EC100B07F077F9CDE91001084619
:1038C00004EB2051C0F31304B948A1F2FF312044A6
:1038D00000F4801080F07F6282F04052224301EBBE
:1038E00020559FEDB50B119253EC102B9DED100B55
:1038F00051EC100B07F02EFB41EC180BA01CC0F391
:1039000013009FEDAFDB9FEDB0EBB14E7E4403287B
:103910006CD296ED000B51EC180B53EC102B07F00A
:103920007FF81DD1002D01BF96ED000BBDEC108B73
:1039300002B070BD284607F00CF941EC180B53ECAF
:103940001D2B07F031F941EC190B53EC1E2B51ECF8
:10395000180B07F029F953EC192B06F055FE3FE040
:103960009FED9D0B51EC180B53EC102B07F01CF93D
:103970009FED9B1B53EC112B07F014FA41EC190B34
:1039800053EC182B51EC180B07F00EF953EC192BD4
:1039900007F00AF941EC190B002D04BF53EC192B69
:1039A00051EC180B1AD0284607F0D3F841EC1A0B4B
:1039B00053EC1D2B07F0F8F853EC192B07F0F2F934
:1039C00053EC182B07F0C6FA41EC180B53EC1E2BE6
:1039D00051EC1A0B07F0E8F853EC182B07F0BAFA81
:1039E000BDEC108B02B041EC100B70BD9FED7E0B57
:1039F00051EC180B53EC102B06F006FE41EC100BAB
:103A000051EC180B53EC102B06F0B2FE41EC190BE5
:103A1000284607F09EF841EC1B0B53EC192B51EC98
:103A2000190B07F0C1F841EC1A0B714853EC1A2B33
:103A3000261851EC1A0B07F0B7F841EC1F0B6D4834
:103A4000C4F1510404F5D724B0EE4F0AF0EE6F0A2A
:103A50000321784400F054FD53EC1F2B51EC100B64
:103A600007F0A2F841EC1C0B6348B0EE4F0AF0EEF1
:103A70006F0A0421784400F043FD53EC1A2B51ECFB
:103A8000100B07F091F8344353EC1C2B06F0BCFDEF
:103A900041EC1C0B002C4CDD9FED510B51EC180B35
:103AA00053EC102B07F080F853EC182B07F07CF840
:103AB00041EC1A0B55B353EC1D2B51EC1B0B07F0CB
:103AC00073F841EC1D0B53EC1C2B51EC1A0B06F058
:103AD0009BFD53EC192B07F067F853EC1D2B06F0F8
:103AE00093FD53EC1A2B07F05DF953EC182B07F0FC
:103AF00031FA41EC180B53EC1E2B51EC1B0B07F069
:103B000053F853EC182B07F025FA69E753EC1C2BFC
:103B100051EC1A0B06F078FD53EC192B07F044F822
:103B200053EC1A2B07F03EF953EC182B07F03AF937
:103B300056E735B353EC1D2B51EC1B0B07F034F853
:103B400041EC1A0B53EC1C2B51EC180B07F002FA4A
:103B500053EC192B07F028F853EC1A2B07F0FAF95D
:103B600053EC182B07F0F6F941EC180B53EC1E2B15
:103B700051EC1B0B07F018F853EC182B07F0EAF97F
:103B80002EE753EC1C2B51EC180B07F0E3F953EC28
:103B9000192B07F009F853EC182B07F003F91FE76E
:103BA0000000F07F00000000000000000000504313
:103BB000645F090000000000000000000000F03F0A
:103BC000763C7935EF39EA3D0000E0FE422EE63FD3
:103BD000C88E000000000000555555555555D53F7D
:103BE000000000000000E03F000000000000004076
:103BF00086EBF9FF828C0000788C0000000000004A
:103C000010B52F499FED2C1B2DED020B84B00598AC
:103C100020F000408842DCBF00209DED040B32DD27
:103C20002849884209D1049840B94FF00100FCF7B7
:103C3000E9FC00F04DFF06B010BD05DB9DED040B67
:103C400000F032FF06B010BD68469DED040B00F099
:103C500083F910F0030011D0012818D09DED021B4C
:103C60009DED000B02281AD000F092FB51EC100BD6
:103C700006F08CFC06B041EC100B10BD9DED021B54
:103C80009DED000B012000F0B7FC06B010BD9DEDCE
:103C9000021B9DED000B00F07BFB06B010BD012068
:103CA00000F0AAFC51EC100B06F070FC06B041ECE1
:103CB000100B10BD0000000000000000000000001C
:103CC000FB21E93F0000F07F00B510EE101A2DED4A
:103CD000028B81B0524A6846B2EB410F2ED94FF0A9
:103CE000E640B0EB410F94BF00204FF0FF30009052
:103CF0000098B0EE408A00286ADB10F0010F4BD02C
:103D000068EE080A9FED471A9FED470A00EE810A08
:103D10009FED461A10F0020F00EE801AB7EE000A6F
:103D200000EE810A02BF01B0BDEC028B00BD00BFF6
:103D300001B0B1EE400ABDEC028B00BD3C4B21F05E
:103D40000042934241D911F0004FDFED3A0A20EED4
:103D5000201ADFED390A19BF31EE601A71EE200A20
:103D600031EE201A71EE600ABDEEE01A11EE100A73
:103D70009FED321A00F0030000EEC10A9FED301AE9
:103D8000009000EEC10A9FED2F1A00EEC10A9FEDD0
:103D90002E1A00EEC10AABE728EE080A9FED2B1A97
:103DA000DFED2B0A10F0020F40EE410A9FED291AB9
:103DB00000EE201A61EE000AB0EE480A08EE200A72
:103DC000B6D101B0BDEC028B00BD00F0B5FE8FE7AF
:103DD00018EE100A4000B0F17F4F0DD218EE100A15
:103DE000FFF746FA042808BF00F09EFEB0EE480A2E
:103DF00001B0BDEC028B00BD09D10120FCF702FC33
:103E000001B0BDEC028B5DF804EB00F085BE01B0A3
:103E1000B0EE480ABDEC028B5DF804EB00F078BE12
:103E2000B61F927EB93AB2BACA9F2A3DDDFFFFBEE5
:103E3000490E494683F9223F0000004B0000C93F6C
:103E400000A0FD390020A2331A61342C336D4C39A7
:103E5000DA82083CA0AA2ABE00B52DED048BB0EE94
:103E6000409AF0EE609A83B051EC190B06F0A6FF71
:103E700041EC180B18EE100A18EE901A8DED008B1D
:103E8000002818BF0120084320F00040C0F17F60E7
:103E900000F1E040C00F14D019EE101A19EE900A8C
:103EA0008DED009B002918BF0121084320F0004040
:103EB000C0F17F6000F1E040C00F04BF0120FCF7BB
:103EC000A1FBB0EE480A03B0F0EE680ABDEC048B2B
:103ED00000BD00000000000010B51D499FED1A1B39
:103EE0002DED020B84B0059820F000408842DCBF25
:103EF00001209DED040B21DD1649884209D104986B
:103F000040B94FF00100FCF77DFB00F0E1FD06B089
:103F100010BD05DB9DED040B00F0C6FD06B010BD25
:103F200068469DED040B00F017F800F00100012138
:103F3000A1EB40009DED021B9DED000B00F0F4FB9A
:103F400006B010BD000000000000000000000000EE
:103F5000FB21E93F0000F07F2DE9F14F04462DEDF4
:103F6000020B2DED088B8AB09FEDE70B80ED020B65
:103F7000139EE74826F0004585420ADC9DED120BB2
:103F8000002084ED000B0AB0BDEC088B03B0BDE847
:103F9000F08FE0489FEDE0AB9FEDE1BBA84247DD2D
:103FA000E14F9FEDE39B9FEDE48B9DED120B53ECF6
:103FB0001A2B51EC100B002E1CDD06F0CBFF41EC50
:103FC000100BBD4208D053EC1B2B51EC100B06F02C
:103FD000C1FFC4E900010BE053EC192B51EC100BAD
:103FE00006F0B8FF53EC182B06F0B4FFC4E900014B
:103FF0000120C8E706F008FB41EC100BBD4208D0D9
:1040000053EC1B2B51EC100B06F0FEFAC4E9000137
:104010000BE053EC192B51EC100B06F0F5FA53ECB6
:10402000182B06F0F1FAC4E900014FF0FF30AAE7BF
:10403000C348A84279DB9DED120B51EC100B01F047
:10404000EDF841EC180B9FEDC00B53EC102B06F074
:10405000ABFD9FEDBF1B53EC112B06F0D5FA06F01C
:104060001BFD074606F075FD41EC190B53EC1A2BAE
:1040700006F09AFD53EC182B06F094FE41EC180B59
:1040800053EC1B2B51EC190B06F08EFDDFF8C8A288
:1040900041EC100B4FEA15580125FA4453EC102B54
:1040A00051EC180B06F056FF032DC4E900013DD07A
:1040B000C1F30A5005EB4511A8EB0000113981420C
:1040C00034DA0AEB051BB0EE48AA9BED000BF0EECC
:1040D00068AA53EC102B51EC190B06F065FD41EC6E
:1040E0001B0B51EC1A0B53EC1B2B06F033FF41EC6E
:1040F000180B51EC1A0B53EC182B06F02BFF53EC5A
:104100001B2B06F027FF9BED020B41EC1A0B53EC27
:10411000102B51EC190B06F047FD53EC1A2B06F04F
:1041200019FF41EC100B6D1CB8E70EE0002EA8BF84
:104130003846BFF628AF94ED000B51EC100B06F09B
:1041400025FAC4E9000178421DE7C6F3130040F4E4
:10415000801EC6F30A50A0F2F530471100F01F058B
:10416000C5F12000DDF848B00890002006900790C7
:104170000520EC467949002D07EB0002794408BF81
:1041800051F8221009D051F8223001EB8201AB40E6
:104190004A68089922FA01F11943A1FB0E26A1FBF6
:1041A0000B131A449A4234BF0123002303EB060881
:1041B0000CEB8003D3E901A60E448E4234BF0121EB
:1041C000002192448A4411B1924502D903E09245FC
:1041D00001D2012100E00021C3E901A641444CF8CD
:1041E0002010011EA0F10100C4DC029800F1005073
:1041F000850F0298DDE903678000DDF8148006F082
:10420000A8FC41EC1A0B304606F0BAFC9FED541B9B
:1042100053EC112B06F0C8FC41EC1B0B384606F0A2
:10422000AFFC9FED511B53EC112B06F0BDFC41EC94
:10423000180B404606F0A4FC9FED4D1B53EC112BD0
:1042400006F0B2FC41EC190B51EC180B53EC192B96
:1042500006F0DAF953EC1B2B06F0D6F953EC1A2BC7
:1042600006F0D2F9CDE90801002008909DED080B79
:1042700053EC1A2B51EC100B06F06CFE53EC1B2B7D
:1042800006F068FE53EC182B06F064FE53EC192B75
:1042900006F088FD9FED381B53EC112B06F084FCD3
:1042A0009FED370B41EC180B53EC102B9DED080BD9
:1042B00051EC100B06F078FC53EC182B06F0A4F927
:1042C0009FED310B41EC180B53EC102B9DED080BBF
:1042D00051EC100B06F068FC53EC182B06F094F927
:1042E00041EC100B139810F0004F06D06D4251ECCA
:1042F000100B06F04BF941EC100B284684ED000B37
:1043000041E6000000000000000000000000000086
:10431000FB21E93F7CD9024000004054FB21F93FDA
:104320003163621A61B4D03DFB21F93F0000000007
:104330000000601A61B4D03D7370032E8A19A33B4C
:10434000FB2139410000000083C8C96D305FE43FA4
:10435000000000000000E03F42870000908600005F
:10436000000000000000103E000000000000103CB3
:10437000000000000000103A182D4454FB21F93DC4
:104380003326A611460B113C00000054FB21F93DD9
:1043900010B52DED040B2DED088B82B0B0EE419AD7
:1043A000F0EE619A0B9820F000449FED4BABB4F116
:1043B000795F11DA9DED0A0B51EC100B06F06CFBE6
:1043C000002801BFB0EE4A0AF0EE6A0A02B0BDEC66
:1043D000088B04BF04B010BD9DED0A0B53EC102BED
:1043E00051EC100B06F0E0FB41EC180B3C480621A9
:1043F000B0EE480AF0EE680A784400F081F853EC19
:10440000182B51EC100B06F0CFFB9DED0A0B41EC85
:104410001B0B53EC192B51EC100B06F0C5FB41ECB8
:10442000190B53EC1B2B51EC180B06F0BDFB53EC96
:10443000192B06F08FFD9FED2C0B41EC190B53EC63
:10444000102B51EC180B06F0AFFB41EC100B284879
:10445000844210DA53EC192B51EC100B06F07AFD64
:1044600053EC1A2B06F09EFC41EC100B02B0BDEC95
:10447000088B04B010BD1F48A042BCBF9FED1E1B9F
:104480008DED001B06DBA4F50010019000200090CC
:104490009DED001B51EC100B53EC112B06F05AFD57
:1044A0009DED000B41EC180B53EC102B51EC1A0B4B
:1044B00006F050FD41EC1A0B53EC192B51EC180B84
:1044C00006F048FD53EC1A2B06F06CFC41EC100B87
:1044D000CCE7000000000000000000000000F03FFA
:1044E000AC83000000000000000000000000E03F7E
:1044F0003333D33F0000E93F000000000000D23F0B
:1045000070B504462DED028B4D1E00EBC500B0EEDC
:10451000408AF0EE608A90ED000B35F0060017D06F
:1045200053EC182B51EC100B06F03EFB41EC100B3A
:104530006D1E04EBC50090ED001B51EC100B53EC0D
:10454000112B06F061F841EC100B35F00600E7D1B5
:10455000022D36D0042D1CD0062D1CBFBDEC028BC5
:1045600070BD53EC182B51EC100B06F01DFB94EDB5
:104570000A1B53EC112B06F047F853EC182B06F0EE
:1045800013FB94ED081B53EC112B06F03DF841ECA6
:10459000100B53EC182B51EC100B06F005FB94EDAF
:1045A000061B53EC112B06F02FF853EC182B06F0DA
:1045B000FBFA94ED040B53EC102B06F025F841ECBC
:1045C000100B53EC182B51EC100B06F0EDFA94ED98
:1045D000021B53EC112B06F017F853EC182B06F0C6
:1045E000E3FA94ED001B53EC112B06F00DF8BDEC33
:1045F000028B41EC100B70BD31B504462DED040B60
:104600002DED0A8BB0EE41BAF0EE61BA0B989DED3C
:104610000A0B20F00040B0F1795F0DDA51EC100B7D
:10462000FEF70EFE042808BF00F062FA9DED0A0BAB
:10463000BDEC0A8B05B030BD53EC102B51EC100BC8
:1046400006F0B2FA41EC180B9DED0A0B53EC182B57
:1046500051EC100B06F0A8FA41EC190B2C48B0EE07
:10466000480AF0EE680A05217844FFF749FF9FEDFC
:104670002ACBB0EE40AAF0EE60AA9CB353EC1C2B00
:1046800051EC190B06F090FA41EC1C0B53EC1A2B71
:1046900051EC190B06F088FA9FED210B41EC190B38
:1046A00053EC102B51EC1B0B06F07EFA53EC192B3C
:1046B00006F050FC53EC182B06F076FA53EC1B2B4B
:1046C00006F048FC53EC1C2B06F044FC9DED0A1B45
:1046D00053EC112B06F066FBBDEC0A8B05B041ECE8
:1046E000100B30BDFFE753EC1A2B51EC180B06F002
:1046F0005BFA53EC1C2B05F087FF53EC192B06F0EB
:1047000053FA9DED0A1B53EC112B05F07DFFE3E7F7
:104710005C82000000000000495555555555C5BF45
:10472000000000000000E03FF1B506462DED040B4F
:10473000BD482DED0C8B8AB0B0EE418AF0EE618A57
:10474000179D25F000449FEDBABB9FEDBBCB844283
:1047500008DA9DED160B51EC100B06F09DF90028C0
:1047600000F0E980B64FA74231DC002D0DDA9DED57
:10477000160B51EC100B05F009FFCDE9160151ECB9
:10478000180B05F003FF41EC180B9FEDAF0B53EC3A
:10479000102B9DED160B51EC100B06F003FB53ECA8
:1047A000182B9FEDAB0BCDE9040151EC100B06F07B
:1047B000D1FB41EC100B53EC102B9DED040B51EC95
:1047C000100B05F021FF9FEDA48BCDE916019DEDA7
:1047D000160B53EC102B51EC100B06F0E5F9CDE95C
:1047E00004019DED040B53EC102B51EC100B06F063
:1047F000DBF941EC190B9A480621B0EE490AF0EEBC
:10480000690A7844FFF77CFE9648B0EE40DAF0EE95
:1048100060DAB0EE490AF0EE690A06217844FFF743
:104820006FFE9DED041B51EC100B53EC112B06F0A9
:10483000BBF99DED040B41EC1A0B53EC102B9DEDD5
:10484000160B51EC100B06F0AFF941EC190B53ECC1
:104850001A2B51EC1D0B05F0D7FE53EC192B06F06B
:10486000A3F953EC182B05F0CFFE9DED041B53EC80
:10487000112B06F099F953EC182B05F0C5FE41EC0D
:10488000180B9FED790B51EC190B53EC102B06F024
:104890008BF953EC182B05F0B7FE41EC190B9DED8D
:1048A000160B53EC192B51EC100B05F0ADFE41EC3F
:1048B000180BA74269DC304606F04BF941EC1A0BA5
:1048C00051EC180B53EC1A2B05F09EFE41EC1B0B20
:1048D00053EC182B51EC180B06F066F953EC1B2B1C
:1048E00005F046FF53EC192B06F034FB9DED161B2B
:1048F00053EC112B06F056FA9FED5D1B53EC112B78
:1049000006F052F953EC1A2B06F04CFA41EC180B56
:10491000022000EAA570C0F1010006F01AF953EC7C
:10492000182B06F041F900BF41EC100B0AB0BDECAA
:104930000C8B05B0F0BD711C1698214308430CD0B8
:104940009DED160B012E1CBF53EC102B51EC1C0BD4
:1049500010D000BF05F00CFFE6E79DED160B51EC03
:10496000100B00F05BFC41EC100B51EC1B0B53ECFB
:10497000102BEFE751EC100BFEF762FC042808BF88
:1049800000F0B6F89DED160BD0E7012E04BFB0EE97
:10499000480AF0EE680AC9D08DED048B0024049417
:1049A0009DED040B53EC102B9DED160B51EC100BF1
:1049B00006F0F8F953EC192B06F0F4F941EC190B59
:1049C00053EC182B51EC1C0B05F0D2FE41EC180BEC
:1049D0008DED008B00949DED040B53EC102B9DEDA1
:1049E000000B51EC100B06F0DFF853EC1B2B05F01D
:1049F0000BFE9DED000B41EC1A0B53EC192B51EC07
:104A0000100B06F0D1F853EC1A2B05F0FDFD53EC1A
:104A1000182B06F0C9F89DED001B53EC112B05F087
:104A2000F3FD81E7000000000000303E00000000C0
:104A3000000000000000F03F000000000000F0BF98
:104A40002894E53F00000000182D4454FB21E93F65
:104A5000075C143326A6813C000000000000000023
:104A6000EA80000000810000635555555555D53F3B
:104A700000000000000000409FED070B10B553EC54
:104A8000102B9FED070B51EC100B05F071FE41EC64
:104A9000100B10BD0000000000000000000000002E
:104AA000000000000000F03F10B553EC102B51EC5B
:104AB000100B05F0A9FD41EC100B10BD10B553EC27
:104AC000112B51EC100B05F09FFD41EC100B10BDAC
:104AD0009FED050B10B553EC102B51EC100B05F0AE
:104AE00047FE41EC100B10BD00000000000000006C
:104AF0009FED050B10B553EC102B51EC100B06F08D
:104B000053F841EC100B10BD000000000000001035
:104B100030EE000A70470000DFED020A80EEA00AC6
:104B200070470000000000009FED020A20EE000A1E
:104B300070470000000000102DE9F0014FF07F42A7
:104B4000B2EB410F9FBF4FF0FF310160BDE8F001B4
:104B500070474FF0004242EA0123C1F3C752783A4E
:104B6000551112F01F0C434CCCF120067C44C1F3CC
:104B7000C752A2F178024FEA621204EB820254F8A3
:104B8000254008BFD2E9015612D0556804FA0CF44A
:104B900025FA06F73C43976805FA0CF527FA06F85C
:104BA000D26807FA0CFCF24045EA08054CEA020616
:104BB000A4FB034CA5FB0352A6FB03631D449D42CB
:104BC00034BF012600261319334416B1934202D98B
:104BD00003E0934201D2012200E00022624402F18C
:104BE000200C9206DC0C42EA443200EE102A5B03F1
:104BF000DFED210AF8EEC01A00EE103A4FEA9C1CD5
:104C000011F0004FB8EE400AC0F800C020EE201AA4
:104C100000EE105ADFED190AB8EE400A20EE200A25
:104C200071EE810A70EE800A10EE902A02F50062A1
:104C30006FF30B0200EE902A70EEE11A31EEC11A0A
:104C4000DFED101A30EE411A9FED0D0A20EE800ABA
:104C500001EE210A9FED0C1A00EE810A04BFBDE8A7
:104C6000F0017047CCF180510160BDE8F001B1EE78
:104C7000400A7047387D0000000000360000802C9C
:104C800022AAFD29DB0FC92F0000C92F30380A28BE
:104C900001D2012070470020704710B541EC100B85
:104CA000FEF7FAFA51EC100B10BD000070B54A4C3B
:104CB0002DED028BE06F64289CBFBDEC028B70BDB4
:104CC0000021084605F076FA00256565A565E06EC9
:104CD000606600F0BDF841494148FBF7FBFA404AE5
:104CE0000A21032000F034FA4FF4FA7000F080F843
:104CF0004FF4FA70FDF782F9DFED3A8AC4F8685094
:104D0000B0EE688AD4E91A0105F054FA3C20FDF7A8
:104D100075F935A13248E26FFBF7DCFA304A3221EF
:104D2000062000F0C9F9E06F00EE100AB8EE400A64
:104D3000B4EEC80AF1EE10FA07D200EE100AA16E26
:104D40002166B8EE408A502834D3A06E401DA0667C
:104D5000B0F5B47FD6DB4FF4FA5000F049F8642088
:104D6000E0660146206E05F025FA3C20FDF746F985
:104D70001DA11B48E26FFBF7ADFA194A322106204C
:104D800000F09AF9E06F00EE100AB8EE400AB4EEB7
:104D9000E80AF1EE10FA07D200EE100AE16E616641
:104DA000F8EE408A502805D3E06E1430E066B0F586
:104DB000FA6FD6DB606E00F10A01206E05F0FAF999
:104DC000606EA065206E60654FF4FA70BDEC028BDA
:104DD000BDE87040FDF712B90000002064A400088F
:104DE0007402002000E87D472D253032642D00003C
:104DF00010B50B490C4C91F839209200C1F8A02055
:104E00000849B1FBF0F0E062206840F0010020604A
:104E10006420FDF7F3F8206820F00100206010BD49
:104E200000000020007C9200001000400020074994
:104E3000024600BF00EB40030B44401CC0B21A60A6
:104E40008128F7D33F2081F8C000704798110020D7
:104E50002DE9F041134E4FF40040B06200200746A8
:104E60004FF01008451C4FF40040B06205F1AF0050
:104E7000C0B205F055FA404605F052FA384605F042
:104E80004FFA0024002005F067FA601CC4B2842C9D
:104E9000F8D3E8B20928E5D34FF40040B061BDE88B
:104EA000F0810000000400482DE9F041134E4FF45A
:104EB0000040B062062500274FF010084FF4004074
:104EC000B06205F1AF00C0B205F02AFA404605F025
:104ED00027FA384605F024FA0024002005F03CFAB1
:104EE000601CC4B2842CF8D3681CC5B2092DE5D36C
:104EF0004FF40040B061BDE8F081000000040048BC
:104F00000146B0F1004F38BF411E15D20029C8BF7D
:104F1000491EFBDC0146B0F1004F38BF411E0ED2E6
:104F20000029C8BF491EFBDC4008B0F1004F09D280
:104F3000401E0028FCDC7047491EFDD1EAE7491EEF
:104F4000FDD1F1E7401EFDD1704700002DE9F74F7C
:104F5000294983464FF400404FF0000988620298C7
:104F60000078002804BF03B0BDE8F08F02980199D3
:104F7000002510F80900A1F101082F38102108F0D0
:104F8000FF0201EB121AC0B21C49C0EB001001EB8A
:104F9000C00700BF184A4FF400410BEB05009162B7
:104FA000AF30C0B205F0BCF9504605F0B9F908F0D1
:104FB0000F0005F0B5F9002405EB450604EBC6002B
:104FC000385C05F0C9F9601CC4B2182CF6D3681C13
:104FD000C5B2052DDED309F1010000F0FF090198EB
:104FE0001830C0B20190029810F809000028BDD115
:104FF00003B0BDE8F08F000000040048E8B20008EC
:105000002DE9F74F2A4983464FF400404FF000093D
:10501000886202980078002804BF03B0BDE8F08FD2
:105020000298002510F809002F38C1B20198A0F1AC
:105030000108102008F0FF0200EB121AC1EB01106A
:105040001C4901EBC00700BF194A4FF400410BEBAC
:1050500005009162AF30C0B205F062F9504605F02C
:105060005FF908F00F0005F05BF9002405EB450639
:1050700004EBC600385CC043C0B205F06DF9601C9B
:10508000C4B2182CF4D3681CC5B2052DDCD309F1C9
:10509000010000F0FF0901981830C0B20190029899
:1050A00010F809000028BBD103B0BDE8F08F000064
:1050B00000040048E8B200082DE9F04FDFF888A0AE
:1050C0000D464FF4004190460026CAF8281011788A
:1050D000802934BF4FF020094FF06109002908BF33
:1050E000BDE8F08F401EC0B200F1B00B18F806000A
:1050F000A0EB0900C7B24FF40040CAF82800681EB0
:10510000C4B20BF0FF0005F00BF9102000EB1410F7
:1051100005F006F904F00F0005F002F90B49002430
:1051200007EB87004718385D05F016F9601CC4B21C
:10513000052CF8D3701CC6B2A81DC5B218F806001D
:105140000028D3D1BDE8F08F0004004878C30008E0
:105150002DE9F74F81B05FEA000B4FF0000704BF65
:1051600004B0BDE8F08F4FF40040DFF8A8A0CAF803
:10517000280003980078802834BF20216121009105
:10518000002804BF04B0BDE8F08F0398C05DA0F113
:105190002001DE2984BF781CC7B234D800990024CE
:1051A000401A0299C0B2A1F10108102108F0FF02D3
:1051B00001EB1219184901EB001600BF4FF4004132
:1051C0000BEB0400CAF82810AF30C0B205F0A8F805
:1051D000484605F0A5F808F00F0005F0A1F80025F5
:1051E00005EBC400305C05F0B7F8681CC5B2082DAB
:1051F000F6D3601CC4B2022CE0D3781CC7B202986C
:105200000830C0B202900398C05D0028BDD104B040
:10521000BDE8F08F0004004878B9000882B0CDE9FD
:10522000000121F0004001909DED000B02B051EC17
:10523000100B7047DFED1D1A00211D48052200BF2D
:10524000C1F1090300EB8303C1F10A0CD3ED000A9D
:1052500000EB8C0CCCED000AC1F1080C00EB8C0CBF
:10526000891CDCED000A521EC3ED000AE8D1114989
:1052700080ED000AB0EE401AD1ED000AB0EE610AEE
:105280005FF0050200EE810AD1ED010A90ED011AEE
:1052900000EE810AD1ED020A90ED021A08300831C1
:1052A000521E00EE810AEFD170470000000000009E
:1052B000E80D002098B20008DFED1D1A00211D48FE
:1052C000042200BFC1F1070300EB8303C1F1080C06
:1052D000D3ED000A00EB8C0CCCED000AC1F1060CFA
:1052E00000EB8C0C891CDCED000A521EC3ED000A99
:1052F000E8D1114980ED000AB0EE401AD1ED000A64
:10530000B0EE610A5FF0040200EE810AD1ED010AFD
:1053100090ED011A00EE810AD1ED020A90ED021A19
:1053200008300831521E00EE810AEFD170470000AC
:10533000000000006C0E0020C4B200089FED211A8E
:1053400000212148032200BFC1F1050300EB8303C4
:10535000C1F1060CD3ED000A00EB8C0CCCED000A79
:10536000C1F1040C00EB8C0C891CDCED000A521E10
:10537000C3ED000AE8D180ED000ADFED140ADFED8D
:10538000141A9FED142A00EE201A90ED010ADFEDA9
:10539000122A00EE211A90ED020A00EE021AB0EE77
:1053A000410A90ED031A01EE220A90ED041A01EE73
:1053B000020A90ED051A01EE210A90ED061A01EE9F
:1053C000200A704700000000D80E002014BEA1BDC6
:1053D0006FEDFCBDDC252FBEE9383F3FDFED1D1A28
:1053E00000211D48052200BFC1F1090300EB830322
:1053F000C1F10A0CD3ED000A00EB8C0CCCED000AD5
:10540000C1F1080C00EB8C0C891CDCED000A521E6B
:10541000C3ED000AE8D1114980ED000AB0EE401A50
:10542000D1ED000AB0EE610A5FF0050200EE810ADC
:10543000D1ED010A90ED011A00EE810AD1ED020AC8
:1054400090ED021A08300831521E00EE810AEFD1A9
:105450007047000000000000140E002098B2000801
:10546000DFED1D1A00211D48042200BFC1F1070312
:1054700000EB8303C1F1080CD3ED000A00EB8C0CA8
:10548000CCED000AC1F1060C00EB8C0C891CDCEDA4
:10549000000A521EC3ED000AE8D1114980ED000A4E
:1054A000B0EE401AD1ED000AB0EE610A5FF00402DE
:1054B00000EE810AD1ED010A90ED011A00EE810A99
:1054C000D1ED020A90ED021A08300831521E00EEAA
:1054D000810AEFD17047000000000000900E00200C
:1054E000C4B200089FED211A00212148032200BF09
:1054F000C1F1050300EB8303C1F1060CD3ED000AF3
:1055000000EB8C0CCCED000AC1F1040C00EB8C0C10
:10551000891CDCED000A521EC3ED000AE8D180EDC3
:10552000000ADFED140ADFED141A9FED142A00EED5
:10553000201A90ED010ADFED122A00EE211A90EDFB
:10554000020A00EE021AB0EE410A90ED031A01EED3
:10555000220A90ED041A01EE020A90ED051A01EEFE
:10556000210A90ED061A01EE200A704700000000A3
:10557000F40E002014BEA1BD6FEDFCBDDC252FBED6
:10558000E9383F3F70B501260F4B0C46F20306EB9E
:10559000D4019A62401EC5B201F1AF00C0B204F05E
:1055A000BFFE102000EB151004F0BAFE05F00F004E
:1055B00004F0B6FE04F0070006FA00F0BDE8704003
:1055C000C0B204F0C9BE000000040048214B032112
:1055D000A3F1100003EB810252ED010AC2ED000AB3
:1055E00000EB8102491E52ED010A11F0FF01C2EDEC
:1055F000000AEFD183ED000ADFED170AD3ED011A9F
:1056000090ED012A20EE201A9FED140ADFED142AF6
:1056100061EE801A42EE621A9FED122A31EE811A73
:10562000D3ED021A21EE800AD0ED021A01EEC20A71
:10563000DFED0D1A30EE010A93ED031A61EE200A38
:1056400090ED031A41EE610A30EE800A80ED000A07
:1056500070470000C01000205BC0FF3C45D0BF3D3C
:10566000D417A5BFF8782A3FE66401BE1449032089
:10567000A1F1100301EB800252ED010AC2ED000A14
:1056800003EB8002401E52ED010A10F0FF00C2ED54
:10569000000AEFD181ED000ADFED0A0A91ED011A4F
:1056A000DFED091A20EE200A61EE200A93ED011ABF
:1056B00041EE610A30EE800A83ED000A7047000077
:1056C00000110020D315003F589B2E3A14490320A7
:1056D000A1F1100301EB800252ED010AC2ED000AB4
:1056E00003EB8002401E52ED010A10F0FF00C2EDF4
:1056F000000AEFD181ED000ADFED0A0A91ED011AEF
:10570000DFED091A20EE200A61EE200A93ED011A5E
:1057100041EE610A30EE800A83ED000A7047000016
:1057200040110020ADAD5B3FDD5B373F214B0321D6
:10573000A3F1100003EB810252ED010AC2ED000A51
:1057400000EB8102491E52ED010A11F0FF01C2ED8A
:10575000000AEFD183ED000ADFED170AD3ED011A3D
:1057600090ED012A20EE201A9FED140ADFED142A95
:1057700061EE801A42EE621A9FED122A31EE811A12
:10578000D3ED021A21EE800AD0ED021A01EEC20A10
:10579000DFED0D1A30EE010A93ED031A61EE200AD7
:1057A00090ED031A41EE610A30EE800A80ED000AA6
:1057B00070470000E01000205BC0FF3C45D0BF3DBB
:1057C000D417A5BFF8782A3FE66401BE1449032028
:1057D000A1F1100301EB800252ED010AC2ED000AB3
:1057E00003EB8002401E52ED010A10F0FF00C2EDF3
:1057F000000AEFD181ED000ADFED0A0A91ED011AEE
:10580000DFED091A20EE200A61EE200A93ED011A5D
:1058100041EE610A30EE800A83ED000A7047000015
:1058200020110020D315003F589B2E3A1449032025
:10583000A1F1100301EB800252ED010AC2ED000A52
:1058400003EB8002401E52ED010A10F0FF00C2ED92
:10585000000AEFD181ED000ADFED0A0A91ED011A8D
:10586000DFED091A20EE200A61EE200A93ED011AFD
:1058700041EE610A30EE800A83ED000A70470000B5
:1058800060110020ADAD5B3FDD5B373F10B5254CAF
:105890004FF09042204694F82F30416F4FF0A040D7
:1058A000012B15D0022B18BF21671CD0816841F055
:1058B00001018160206FFCF7ABFC94F83000FBF72E
:1058C00087FE6420FCF79AFB012084F8210010BDBC
:1058D0004FF400739361402202632167A521C4F84D
:1058E000A4106E211BE04FF40071916280210163CE
:1058F0004FF4407292FAA2F20021B2FA82F2D14041
:1059000000EB81010A6B22F4F86242F080020A6324
:10591000A16F216740F22B11C4F8A4107721C4F8BD
:10592000A810C3E70000002010B5344C4FF400402D
:10593000A0624FF09043C0119862642200210220BF
:10594000401C6E28FCD3491C9142F8D34FF4807060
:105950009861142200210220401C6E28FCD3491CAF
:105960009142F8D3E22004F0DBFC0A22002102205D
:10597000401C6E28FCD3491C9142F8D32C2004F023
:10598000CFFC0A2200210220401C6E28FCD3491CB7
:105990009142F8D32E2004F0C3FC0A2200210220F9
:1059A000401C6E28FCD3491C9142F8D32F2004F0F0
:1059B000B7FC0A2200210220401C6E28FCD3491C9F
:1059C0009142F8D3252004F0ABFC812004F0A8FC20
:1059D000282004F0A5FCA22004F0A2FCC82004F0BA
:1059E0009FFCA02004F09CFC402004F099FCAF2018
:1059F00004F096FC4FF40040A06110BD0004004884
:105A0000C1F10B0100EE901A9FED0C1A0C49F8EE53
:105A1000E00A01EB8000D0ED001A20EE811AF7EECB
:105A2000000A70EEC10A60EEA10A41EE000AC0ED64
:105A3000000ABDEEE00AB8EEC00A70470000003D63
:105A40002C0F00200A4B10B54FF400429A62491EF9
:105A5000AF30CCB2C0B204F063FC102000EB1410E5
:105A600004F05EFC04F00F00BDE8104004F058BCE8
:105A700000040048000000002DED088BA2B0FCF7E8
:105A800003FF0024FF4D0294039404940594686975
:105A900040F400206861686900F40020069068699D
:105AA00040F480006861686900F4800006906869CD
:105AB00040F400306861686900F40030069068695D
:105AC00040F4802068616869EF4900F48020069006
:105AD0004FF4005088624FF0904148F20C308862D9
:105AE000EA4E4CF2F800B0624FF400504FF001095A
:105AF000CDE900096946E448FBF7C2FF48F20C30E3
:105B00000090CDE90194039469464FF090400494CD
:105B1000FBF7B6FF43F60340CDE900046946CDF834
:105B200010903046FBF7ACFF4CF2F8000090CDE946
:105B300001940394694630460494FBF7A1FF2815AD
:105B4000CDE900046946CDF810904FF09040FBF786
:105B500097FF6815CDE90004694630460494FBF7C9
:105B60008FFF1294139414940794089409940A9440
:105B700006940C940D940E940F940B940294039439
:105B800004940594686940F080506861686900F089
:105B900080501590686940F40030686168694FF082
:105BA000030800F40030CDF804801590CDF8008093
:105BB00069464FF09040FBF763FF1294139412A9CB
:105BC0004FF0A0401494FBF7DDFE06940794089470
:105BD000CDE909494FF4805906A94FF0A040CDF80E
:105BE0002C90FBF7E9FE0C940CA9A9480D94FBF747
:105BF0009FFE4FF0A045A86820F04050A860A8681C
:105C000020F03F0020F0004040F08050A860A14804
:105C1000DFF884B20068B0FBFBF000EB80004100CD
:105C20009E48A0FB0110C008002843F3738700BF03
:105C30004FF4407191FAA1F1B1FA81F14FF0A04017
:105C400024FA01F100EB8100016B21F4F86141F0CD
:105C5000400101634FF0007191FAA1F1B1FA81F1B5
:105C60004FF0A04024FA01F100EB810148694FF0A8
:105C7000F87393FAA3F34FF44012B3FA83F322FAC2
:105C800003F307229A404FF0F873904393FAA3F37B
:105C90004FF44012B3FA83F3DA4004FA02F21043ED
:105CA0004861D5F8B0004FF0A04120F00200C1F8E3
:105CB000B0000C940D940E947248069407940894C6
:105CC00009940A940B9402940394049405944169F2
:105CD00041F080514161416901F080510F9141696A
:105CE00041F400314161416901F400310F91416992
:105CF00041F4802141614069694600F480200F90A1
:105D00008020CDE900084FF09040FBF7B9FE4FF03E
:105D1000040A0320CDE900A0694604945B48FBF720
:105D2000AFFE5F4E0C940D940CA930460E94FBF719
:105D300029FE069407940120CDF82C900894CDE913
:105D4000094006A93046FBF737FEB06820F0405006
:105D5000B060B06820F03F0020F0004040F080507C
:105D6000B0604C480068B0FBFBF000EB80004100E5
:105D70004A48A0FB0110C008002843F3D28600BFA8
:105D80004FF4407090FAA0F0B0FA80F024FA00F0DE
:105D900006EB8000016B21F4F86141F4807101632E
:105DA0004FF0007090FAA0F0B0FA80F024FA00F002
:105DB00006EB8001D1F814C04FF0F87292FAA2F30A
:105DC0004FF44000B3FA83F320FA03F9072303FAF0
:105DD00009F392FAA2F2B2FA82F2D0402CEA03035B
:105DE00004FA00F018434861D6F8B00020F0100023
:105DF000C6F8B000DFF88C900794089409940694D4
:105E00000294039404940594D9F81C0040F00050C7
:105E1000C9F81C00D9F81C0000F000500A90D9F80D
:105E2000140040F40030C9F81400D9F81400694691
:105E300000F400300A903020CDE900084FF0904087
:105E4000FBF71EFEDFF85CA0DAF80000C0F30220CA
:105E5000011D072934BF0020C01E04FA00F01249BA
:105E6000000181F80004DFF844B04FF48000CBF863
:105E700000013820CDE906040E4E06AA0C49304632
:105E8000099419E00010024000080048000400488E
:105E90000003005064020020400D0300CDCCCCCCA8
:105EA000000100500CED00E036E000E004E000E00E
:105EB0000100100200740040FBF7B4FD306820F0D0
:105EC000040030600220099006AAFE493046FBF724
:105ED000A9FD306820F4802030600794089409946C
:105EE00006940294039404940594D9F81C0040F09D
:105EF0008060C9F81C00D9F81C0000F080600A908E
:105F0000D9F8140040F40030C9F81400D9F814008E
:105F1000694600F400300A90402000900320019070
:105F20004FF09040FBF7ACFD3820CDE9060402208D
:105F3000099006AAE449E548FBF774FDE3480068C8
:105F4000E24920F004000860E1484CF6CC410160D1
:105F5000DF4945F2555008600620486040F6FF7062
:105F600088600846C16811F0070FFBD1D8484AF68F
:105F7000AA21016000940194029403940494D9F836
:105F80001C0040F00100C9F81C00D9F81C0000F00A
:105F900001000590DAF80000C0F30220C0F107010B
:105FA000042988BF0421021D072A34BF0020C01E17
:105FB000012606FA01F1491E01F00201814006FAAC
:105FC00000F0401E00F002000843C249000181F8C1
:105FD00000044FF0E0283007C8F8000145F6BF5034
:105FE000ADF80000272002906946B007FBF736FEA7
:105FF000B007016821F080010160816821F007018C
:1060000021F4A0318160416821F070014160816814
:1060100021F080018160009401940294039404941F
:10602000D9F81C0040F00200C9F81C00D9F81C0087
:1060300000F002000590DAF80000C0F30220011D14
:10604000072934BF0020C01E04FA00F0A249000155
:1060500081F800044FF00050C8F80001E020DFF89C
:106060007C820290ADF8004069464046FBF7F6FDA1
:10607000D8F8000020F08000C8F80000D8F8080028
:1060800020F0070020F4A030C8F80800D8F8040079
:1060900020F07000C8F80400D8F8080020F0800054
:1060A000C8F8080000940194029403940494D9F869
:1060B0001C0040F01000C9F81C00D9F81C0000F0CA
:1060C00010000590DAF80000C0F30220C0F10701CB
:1060D000042988BF0421021D072A34BF0020C01EE6
:1060E00006FA01F1491E01F00101814006FA00F0B3
:1060F000401E00F0010008437949000181F80004C6
:106100004FF48000CBF800010920ADF8000040F208
:10611000DC50DFF8D081029069464046FBF79EFDD7
:10612000D8F8000020F08000C8F80000D8F804007B
:1061300020F07000C8F80400D8F8080020F08000B3
:10614000C8F80800159416940094129413940194BE
:106150000294059403940494069407941994189453
:106160001A941B941C941E941D941F9420942194A3
:106170000A940B940C940D940E940F94D9F8180073
:10618000594940F400308861886912A900F4003050
:10619000089040F22B10ADF84800401C1490534872
:1061A000FBF75CFD51480068504940F080000860F2
:1061B0004F4801784F4801EB0009D9F80000DFF89B
:1061C00038A108229AF8001002FA01F10843C9F830
:1061D00000006020CDE90004029403940494059427
:1061E00006946A46012141480794FBF77FFDD9F8E0
:1061F00000209AF800100420884022EA0000C9F824
:10620000000018944FF40050CDE91C0440008DF8B4
:106210006C40219019941A94ADF86E4018A9334837
:10622000FBF7ECFC304840692F4940F4802048617E
:10623000486900F48020089088150A900220CDE972
:106240000B04CDE90E460AA92C480D94FBF718FC67
:10625000FFF76AFBFEF7FCFDA86840F00040A8606D
:10626000A86810F0004FFBD1D5F8080140F00040BD
:10627000C5F80801D5F8080110F0004FFAD14FF029
:10628000A042D06820F47C60D060D06840F4807078
:10629000D060D06840F48060D060906840F0010029
:1062A0009060C820FEF72CFED2F8080140F00100F3
:1062B000C2F80801C820FEF723FE906840F00400F1
:1062C00090601DE01200431501001002009800408C
:1062D000003000401CE000E01DE000E00004004051
:1062E00036E000E000100040001002400044014091
:1062F00022B20008184401402BB2000800040048F4
:10630000FD48016841F001010160016841F48031FC
:106310000160FA48016841F001010160F848016834
:1063200021F002010160C16841F00101C160F5493D
:106330000A6842F060020A60F3490A6842F001020A
:106340000A60011D0A6822F070020A600A6842F0C1
:1063500030020A60ED4A69211160016841F00101D3
:1063600001600005016821F002010160C16841F08F
:106370000101C160016841F001010160E448016868
:1063800021F002010160C16841F00101C160E148F2
:10639000016A41F00101016264214163016841F039
:1063A00001010160C820FBF729FEDFF86C830020A3
:1063B00098F80910494200EBC12000F1006000F597
:1063C000704090F8000CDFF85493D54DFF280DD0A5
:1063D000286810F4806F04BF286810F0010F25D1E1
:1063E0004FF09040006910F4806F1FD188F8094089
:1063F0004FF00000FCF732FE98F80900401CC0B2D4
:1064000088F809000428F3D388F809404846FBF7C8
:106410003BFA02224946C348FBF758FAC248D8F86B
:106420007410A0FB01104008C8F8780099F800002B
:1064300088F80900032884BF032088F8090003F0C6
:10644000A5FB98F82F00FFF721FAFCF74BFDD8E9E0
:10645000150103F0AFFE98F8351001EBC10000EB19
:106460000110AC494863012088F82800002088F812
:10647000270098F81C009FEDAEAB01287BD0AE49F9
:106480004FF4804088614FF090410820C1F8280007
:106490004FF4FA70FBF7B2FDFEF7DAFCA7A1A948AA
:1064A000F9F718FF0521A8A20120FEF751FE40F6DA
:1064B000B830FEF79DFC1521A4A20220FEF748FE8D
:1064C0004FF4FA60FEF794FC2521A1A20120FEF70B
:1064D0003FFE4FF47A70FEF78BFC35219DA202201F
:1064E000FEF736FE6420FBF789FD42219AA20120C7
:1064F000FEF72EFE40F2DC50FEF77AFC3220FBF76E
:106500007DFD40F2DC50FEF773FC96A298A18D4809
:10651000F9F7E0FE8B4A41210320FEF7CDFD98F804
:1065200009100120494200EBC12000F1006000F594
:10653000704090F8000C88F839004FF4FA70FBF7BF
:106540005DFD00241C212046FFF71CF8601CC4B22E
:10655000802CF7D398F8010098F82E1000EB410139
:10656000844850F8212084A17648F9F7B3FE192118
:10657000744A052000E006E0FEF7EAFD98F81C00EA
:1065800001283BD12FE06C484FF4804181624FF0ED
:106590009041082088616420FBF730FD98F81B00CB
:1065A0004C3804F0EDFA53EC1A2B04F0E1F804F047
:1065B000A3FAC4B280210020FCF7F0FD4FF47A70FA
:1065C000FEF79EFC31210020FCF7E8FDB9210220F6
:1065D000FCF7E4FD4B211020FCF7E0FD21460120F3
:1065E000FCF7DCFD54E798F81B2064A15548F9F747
:1065F00071FE544A0F210720FEF7AAFD4FF4FA70EE
:10660000FBF7FCFC0C2088F81F00B8F89400C0F3DE
:106610000721C0B211FB0011091A133101FB00124E
:10662000101A3B304FF47F42C0B202EA0121084405
:10663000D8F8981088420CD1FAF7F8FFD8F89410DF
:10664000884206D1042088F84100022088F84000E2
:106650001FE0042088F84100012088F84000FFF77F
:1066600063F9FEF7F5FB49A13648F9F733FE354AE1
:1066700018210120FEF76CFD47A13248F9F72AFEE8
:10668000304A0A210320FEF763FD4FF4FA60FBF75E
:10669000B5FC98F8140055281ED098F84000022840
:1066A0001ED1FBF7A3F898F87C10484300F00700D0
:1066B000062811D1FEF7CCFB3BA12248F9F70AFED0
:1066C000204A0A210320FEF743FD41F28830FBF700
:1066D00095FC19492020886298F84000022806D0CD
:1066E00098F83100142884BF142088F8310000265F
:1066F000304661E000000000007400400098004057
:10670000000400401804004020040040340400400D
:1067100000100040004401400000002000DC0008A0
:106720001004004809000020ABAAAAAA000000003B
:106730009A9999999999A93F000400484B504F5450
:106740002D000000740200204B00000050000000EB
:106750004F000000540000002053544D5F46333278
:1067600020000000762E31372F30372F32360000D0
:10677000257320001802002025730000464D202DAF
:10678000202564206D487A20000000002A2A2A442F
:10679000454D4F2A2A2A0000726164696F646F6D4B
:1067A00040692E7561000000204B4559204552522A
:1067B0004F522120000000004FF000610958001DD9
:1067C0000E44B0F5E04F94D3FB48C06C864224D011
:1067D000FEF73EFB6420FEF70BFBF8A1FB48F9F740
:1067E00079FDFA4A0A210320FEF7B2FC4FF47A70D1
:1067F000FBF704FC286810F4805F04BF286810F4DD
:10680000005F09D13246F2A1F048F9F763FDEF4A83
:1068100023210620FEF750FCFEE7EE48006810F446
:10682000806F05D14FF09040006910F4806F06D062
:10683000E848006810F4006F2FD000F0F4B8DE4D87
:10684000FF2068710F2085F827000120A871FEF74E
:10685000FFFAE1A1DD48F9F73DFD0121DB4A0846D9
:10686000FEF776FCFCF7C6FBC5F89C0040F6B83096
:10687000FEF7BEFAFCF7BEFBC5F89C004FF4FA60C9
:10688000FEF7B6FAFCF7B6FBD249C5F89C000868DB
:1068900010F4805FFBD000F02AB9C74D012085F8C5
:1068A0002300FEF7D5FA0A2085F83E0085F83D0062
:1068B000FBF706FE40F6E4466420FBF79FFBD5E9B4
:1068C0002980804588BFDFF824B30FD9CBF800803A
:1068D0001420FBF793FBE86FB04201D206468146D5
:1068E000D5F8A800A8F105088045EFD895F8300044
:1068F000A0EBC00000EB800009EB80099FEDBC8B92
:106900009FEDBD9B4FF000086420FBF777FBD5E9B6
:106910002960864255D3B54806601420FBF76EFB0C
:10692000E86F404506D9B6498046A1FB00213746AD
:106930004FEA111A95F83010A0EB09004901B0FB9D
:10694000F1FBBBF13C0F03F2F38000BFD5F8A400CC
:10695000801B04F015F9B0EE481AF0EE681A53ECFB
:10696000112B03F005FFB0EE491AF0EE691A53EC53
:10697000112B04F0EFFA04F08FF840B20BF0FF0196
:10698000FBF770FD9F484AF6AA2101609C48EB6F17
:10699000EA7AA0FB03109C490009B1FBF2F1721CDA
:1069A00091FBF2F2009099A18848F9F793FC874A8D
:1069B00002210120FEF780FBD5F8A800761E864252
:1069C000A9D2E97A9048CDF800A0B0FBF1F0791C8B
:1069D00090FBF1F395F8302091A17C48F9F77AFC0F
:1069E0007A4A02210120FEF767FB86494AF6AA206F
:1069F00008607848016811F4006F08D0016811F44C
:106A0000805F3FF47FAF016811F4006FF6D103F0AF
:106A1000BDF895F82F00FEF739FFFCF763FAD5E9CA
:106A2000150103F0C7FBDFF8AC81D8F8000010F0C7
:106A3000010F40D14FF4FA70FEF7DAF9FEF708FAC9
:106A4000FAF7D4FE5C4DDFF8BC91834640F6E4468D
:106A50004AF6AA2AC820FBF7D1FAC9F800A0E86FC5
:106A6000B04203F269805B4672A15848D5F82C21E8
:106A7000F9F730FC554A03210120FEF769FB71A1AB
:106A80005248EA6FF9F726FC504A03210420FEF72A
:106A90005DFA6DA14D48F9F71DFC4C4A64210720B1
:106AA000FEF756FBD8F8000010F4006FD2D14FF477
:106AB000C870FEF79DF96420FBF7A0FAFAF796FE7E
:106AC000052814DAFEF7C4F960A14048F9F702FC82
:106AD0003E4A14210320FEF73BFB3220FEF788F9E3
:106AE0003C20FEF785F94FF47A70FBF787FADFF860
:106AF000C89001254FF47A7089F82150FBF77EFA8F
:106B0000FEF7A6F999F84000401D89F81D00FCF732
:106B100071FAC9F89C006420FBF770FAFCF76AFA76
:106B2000C9F89C006420FBF769FAFCF763FAC9F81E
:106B30009C0000BF99F83100C0F11E0089F83200B6
:106B4000D9ED2F0AC9ED350A99ED300A89ED370ADA
:106B500099F8370000282ED0D9F85C0004F0E4FA48
:106B600041EC100BFDF74CF8B0EE408AF0EE608A75
:106B7000D9F8DC0003F0EDFF53EC182B04F014F807
:106B800041EC190BD9F85C0004F0CEFA41EC100B83
:106B9000FCF7EEFDB0EE408AF0EE608AD9F8D40042
:106BA00003F0D7FF53EC182B03F0FEFF53EC192B27
:106BB00003F02AFD52E0EDE00000002020474C4F9A
:106BC00042414C204552524F522120007402002075
:106BD000256C640010040048466163746F7279206C
:106BE00073657474696E6773000000002C040040C4
:106BF00000000000000012400000000000005040B3
:106C0000898888880030004000D8B8052564487A13
:106C10002025646D42204B553D2564202000000056
:106C2000472564204D41583D2564487A204B553D09
:106C3000256420002564487A202A2025646D41209F
:106C40000000000025642F006D562000205475724E
:106C50006E20636F696C21200000000003F01CFFB0
:106C6000C9F8EC00D9F85C0004F05EFA41EC100BB6
:106C7000FCF7C6FFB0EE408AF0EE608AD9F8D40087
:106C800003F067FFB0EE480AF0EE680A53EC102BF1
:106C900003F08AFF41EC180BD9F85C0004F044FAC9
:106CA00041EC100BFCF764FDB0EE409AF0EE609AF8
:106CB000D9F8DC0003F04DFF53EC192B03F074FFFF
:106CC00053EC182B04F046F903F0E6FEC9F8F00087
:106CD000C9F8F40099F82E00042806BFD9F8D400AA
:106CE00040106420C9F81801D9F8F400C01C03F062
:106CF00030FF41EC100BFCF79FFD51EC100B03F043
:106D0000CBFEC9F800010028C2F21987D9F8F400B7
:106D1000C11700EB917085104AF6E030854228DDFE
:106D2000C320FD4A99F83A10B2FBF0F0490001EB9C
:106D30004101FA4B4900C9F8A010D862186840F028
:106D40000100186049F64040FEF7DAF8C32099F8D0
:106D50003A10B2FBF0F0490001EB41014900C9F8DB
:106D6000A010D862186840F001001860002089F86F
:106D7000380099F94810D9F800010144C8B289F8DF
:106D8000240099F83820012A18BF4FF4967012D0C9
:106D900000F068BAB8EEC01AF8EEE01A99ED172ABA
:106DA00001EEC21ABDEEC11A89ED3D1AC9ED3B0ACA
:106DB00089ED3C0A8EE74FF0000A89F838A099F86F
:106DC0002820012A76D0022A00F0BC81401C99F8C4
:106DD0003A204FF4FA71C0B2520012FB00F0DFF813
:106DE0003883C9F8A000B8FBF1F0CC4EF0623068EF
:106DF00040F00100306099F83200D9F8F410814277
:106E0000C4BFD9F81821B2EB400F40F32F82B1F57F
:106E1000AF7FC4BF012089F8160089F829A099F82E
:106E20002A00401CC0B289F82A00322884BF012001
:106E300089F82100D9F8D810D9F8EC00411AC9F81E
:106E4000EC10D9F8E020D9F8F000801A00EE100A12
:106E5000C9F8F000F8EEC00A00EE101AB8EEC00A49
:106E600003F096FA41B289F80D10D9F81C010844D4
:106E7000C9F81C01D9F8F400109A904204DD89F891
:106E80000F10C9F82451109099F90F1089F81110BA
:106E900089F80D1099F83B3099F82A209B1C9A42EA
:106EA00040F2508299F82E20042A40F0AB8100F085
:106EB000A7B9FFE799F83210D9F8F420481C8242AC
:106EC000C4BFD9F8180188427BDD89F82BA089F866
:106ED00029A099F82A00401CC0B289F82A00142879
:106EE00084BF012089F82100D9F8D810D9F8EC0026
:106EF000401AC9F8EC00D9F8E020D9F8F010891A46
:106F000000EE101AC9F8F010F8EEC00A00EE100AF0
:106F1000B8EEC00A03F03CFA40B289F80D0089F8D7
:106F20001200D9F8F410109A914204DD89F80F008C
:106F3000C9F82451109199F911209042B8BF89F8ED
:106F4000100099F8100089F8110099F90F3089F8AC
:106F50000D3099F8392089F83A2099F82500012850
:106F600030D93229C2BF99F9471008290A2B29DDE7
:106F70004FF4FA61032820D0501CC6B26648DFF8EF
:106F80009C81B0FBF1F0C8F82C00D8F8000040F06C
:106F90000100C8F80000092506FB05F0C9F8A000AB
:106FA0001E20FBF72BF8681E10F0FF05F4D1D8F86F
:106FB000000020F00100C8F8000089F847A000F0A8
:106FC000C1B903E002F098FF00F0BCB900201090B6
:106FD000642089F8100099F82900401C89F82900DC
:106FE00089F82AA0D9F8EC00C9F8D800D9F8F0003F
:106FF000C9F8E00099F82500022879D999F82B0002
:10700000401C89F82B0099F83700E8B3D9F85C00E8
:1070100004F08AF841EC100BFCF7F2FDB0EE408A68
:10702000F0EE608AD9F8C40003F093FD53EC182BFE
:1070300003F0BAFD41EC180BD9F85C0004F074F8C9
:1070400041EC100BFCF794FBB0EE409AF0EE609A26
:10705000D9F8C80003F07DFD53EC192B03F0A4FD13
:1070600053EC182B03F076FF03F016FDC9F8F80077
:10707000C01C03F06EFD41EC100BFCF7DDFB9FED37
:10708000281B53EC112B00E033E051EC100B03F004
:107090006FFB03F001FDC9F80401D9E93E128B1A18
:1070A000214981FB0331A1EBE1711144C9F8F810CA
:1070B000C9F8FC1099F83220914237DD99F82B106D
:1070C000052933D999F848204FF4FA71104499F8FA
:1070D0003A20C0B2520012FB00F0C9F8A0000E48DE
:1070E000B0FBF1F10D48C162016841F0010121E0FE
:1070F00022E099ED320AD9ED310A99ED171AB8EE6E
:10710000C00AF8EEE00A00EEC10ABDEEC00A89ED41
:107110003E0A10EE100AABE7007C9200001000401F
:10712000000000C0CCCCF43F56555555FE480168D0
:1071300021F00101016005E1FB48016821F0010136
:107140000160FFE099F83200D9F8F4208242C4BF10
:10715000D9F81821B2EB400F3EDD89F829A099F843
:107160002A00401CC0B289F82A0099F83B20921CE2
:1071700090421ED9C8B299F83A104FF4FA724900F9
:1071800011FB00F0C9F8A000E848B0FBF2F1E648B6
:10719000C162016841F00101016099ED370AF8EE22
:1071A000C00A99ED350AB8EEC00A03F0F1F889F883
:1071B0000D00D9F8F4001099884206DD99F80D10F9
:1071C00089F80F10C9F82451109099F80F0089F828
:1071D000110089F80D00B5E0D9F8C400C9F8D8004D
:1071E000D9F8C800C9F8E00000201090C9F824A11F
:1071F00089F82AA099F82900401C89F82900A1E003
:1072000014292EDB002901DA012A2AD001F14602D5
:107210009D2A26D2002912DD00F5FA7199F83A204C
:1072200099F82400520012FB00F0C9F8A000B8FB46
:10723000F1F0F062306840F00100306011E0C0F51C
:10724000FA7199F83A2099F82400520012FB00F0E4
:10725000C9F8A000B8FBF1F0F062306840F001001E
:1072600030606420FDF74CFE6CE000BFD9F8EC0004
:10727000C9F8D800D9F8F000C9F824A1C9F8E0008D
:107280000020109099F82900401C89F8290099F8ED
:107290001600012850D199F82A000A284CD9D9F8AB
:1072A0001C1191FBF0F20A2A1FDD99F825104FF40A
:1072B000FA60032940D0B8FBF0F099F83910F06279
:1072C000491CCDB2306840F0010030604FF0090831
:1072D00005FB08F0C9F8A0001E20FAF78FFEA8F100
:1072E000010010F0FF08F3D122E091FBF0F010F163
:1072F000140F21DA99F82510C82003291CD0B8FBF7
:10730000F0F099F83910F062491CCDB2306840F0C5
:10731000010030604FF0090805FB08F0C9F8A00033
:107320001E20FAF76BFEA8F1010010F0FF08F3D160
:10733000306820F001003060C9F81CA189F816A05F
:1073400089F82AA099F82900FA280CBF0122002206
:1073500099F82A10FA290CBF0121002111430DD000
:107360000021C9F8241189F80E1089F80D1089F848
:107370001210012289F8212089F84710C22808BF7D
:10738000FDF754FD99F82900FA2808BFFDF78CFD98
:1073900099F80500002899F8900006D000F01F0029
:1073A000032800F02B8200F02DBAC0B289F8430008
:1073B00000F00F0189F844100A2803D1FBF71AFEE8
:1073C000C9F89C00B9F89000C0F30B00B0F5167F27
:1073D00004D1FDF769FD002089F8120099F84400F6
:1073E000012878D1D9F8240199F90D50C01C03F077
:1073F000B0FB41EC100BFCF71FFA9FED4D1B51EC5D
:10740000100B53EC112B03F0A5FD03F045FB0646D2
:10741000D9F82401C9F82801D9F8F40032285ADD36
:1074200095FBF6F000EBD07089F80E50401089F80B
:10743000470099F90F0099F91110401AC01C03F088
:1074400088FB41EC100BFCF7F7F951EC100B03F043
:1074500023FB99F94710074691FBF7F040B289F8F2
:107460004700552D03DC99F91110002904DA00EBCF
:10747000D070401089F8470099F83F0000F13401BE
:107480008D42A4BF4030A84206DB99F9470000EBCB
:10749000D070401089F84700002EA6BF99F9470028
:1074A0000028002003DB0A28C8BF0A2001DD89F874
:1074B000470099F9471099F90C00091A01EBD171AD
:1074C00000EB610089F8470089F80C00F54204BF21
:1074D000002089F8470099F8440002280CD1FAF7F7
:1074E00061F915A253210420FDF7E6FD99F8470044
:1074F0008006000EFAF72EF999F8440003280CD103
:1075000099F830200DA11048D9F87C30F8F7E2FE48
:107510000D4A3A210320FDF7CFFD99F81D000728F9
:1075200024D00AA1084815E000100040007C920019
:10753000000000000000F03F520000004725643CBE
:1075400025646D563E2000007402002044454D4FD6
:1075500000000000F8F7BEFEFE4A55210720FDF7A7
:10756000ABFDFC4A14210720FDF7A6FD99F8440065
:10757000042841D1F849D9F89C00A1FB0021C90891
:107580004A4202EB820200EB4200CDE9001099F87A
:107590003B3099F83120F1A1EE48F8F79BFEED4A17
:1075A0003A210120FDF788FDD9F82C01009099F8C7
:1075B000090099F82F30421CEDA1E648F8F78AFE41
:1075C00099F82F30032B12D1D9F82C0140F24D112C
:1075D00090FBF1F24FF47A7190FBF1F0CDE90002EB
:1075E00099F80900E6A1421CDA48F8F773FED94A77
:1075F0003A210220FDF760FD99F8440005280BD1DF
:10760000D9F8580020B3E3A1D248F8F763FED14A75
:1076100070210320FDF750FD99F8440006281AD187
:1076200099F84500042816D099F90E20002AB8BF11
:107630005242DAA1C748F8F74DFE99F90E00C54A43
:1076400000284FF002014FF0010002DBFDF77EFC45
:1076500001E0FDF7D5FC99F8430032280BD199F8E9
:107660003700E8B3CFA1BB48F8F734FEB94A3A2156
:107670000420FDF721FD99F8280001283AD099F857
:1076800044000B2808BFFDF70FFCD9F800010028C3
:10769000C4BFC0B2FAF7A4FD99F82800022873D03D
:1076A000C2A1AC48F8F716FEAA4A02210620FDF74F
:1076B0004FFD40212046FEF7C5F9AA2002F04CFEFE
:1076C00099F84500042800F006850624402120464C
:1076D000FEF7B8F9AA2002F03FFE601CC4B200E039
:1076E00003E0082CF2D300F0F6BCB2A19948F8F7F9
:1076F000F1FDBBE799F84500012829D0022844D0C4
:107700000328DDD1AD48D9F8F41099ED370A80FB94
:107710000110F8EEC00A99ED350AA0EBE070C5B291
:10772000B8EEC00A02F034FEA549C0EBC00081FBF0
:1077300000108110A1EBE07040B22946FBF714F86D
:1077400040210820FEF77EF9AA2002F005FEB7E7E7
:1077500099F844000728B8D1D9F82801C01048BFCB
:107760004042C9F82801172802F3EE8199F8281140
:1077700099F9120002F098FC40212046FEF762F9C8
:10778000AA2002F0E9FD9BE732E099F83010D9F821
:10779000D400091D084140B289F81700D9F8DC204F
:1077A00042FA01F149B201F1160289F818102C2AA7
:1077B0009CBF00F13F027E2A87D899F90D20002A4C
:1077C00008DB0029B8BF4942C9B20028B8BF40420F
:1077D00040B20AE00028C4BF404289F817000029DF
:1077E000B8BF4942C9B299F91700FAF73BFE67E7FB
:1077F00074A15848F8F76EFD56E700BFF9F7F6FF99
:1078000089F81A0099F8060038B1012800F034828E
:10781000022800F0B98300F05EBC6B4D99F80100BE
:107820006AA155F820204B48F8F754FD684C0A210E
:10783000A4F117026078FDF78BFC99F8392065A157
:10784000A4F11700F8F746FD6078A4F117025F2154
:10785000FDF77EFC99F801005CA105EB80008268D1
:10786000A4F11700F8F736FDA078A4F117020A2159
:10787000FDF76EFC99F8252056A1A4F11700F8F742
:1078800029FDA078A4F117025F21FDF761FC99F8AA
:1078900001004EA105EB80000269A4F11700F8F782
:1078A00019FDE078A4F117020A21FDF751FC99F9BE
:1078B0004820012A05DA49A1A4F11700F8F70AFDCA
:1078C00003E048A12348F8F705FDE078214A582154
:1078D000FDF73EFC99F801003CA105EB80008269B0
:1078E0001C48F8F7F7FC20791A4A0A21FDF730FC0A
:1078F00099F833003EA1C0F106021648F8F7EAFCF9
:107900002079144A5F21FDF723FC99F801002FA18B
:1079100005EB8000026A0F48F8F7DCFC60790D4A3D
:107920000A21FDF715FC344999F83C000A5C30A1A6
:107930000848F8F7CFFC6079064A5F21FDF708FC9C
:1079400099F8010021A105EB8000826A0148F8F74F
:10795000C1FC53E074020020CDCCCCCC5325303296
:1079600064202046256425202064762564000000DC
:10797000502564282564292564487A2000000000E9
:107980005025642825642925642B25646B487A20BA
:1079900000000000432E422E00000000253032641B
:1079A000000000004742462E00000000446570744D
:1079B000680000004742562E0000000056555555FD
:1079C0006766666650696E00AC0100202573000092
:1079D0008B0200202D202564200000002D28256426
:1079E000292020002D282B256429202000000000BC
:1079F0002D2025642020000034010020A079FE4ABB
:107A00000A21FDF7A5FB99F82F0001287DD0022857
:107A10007CD099F83D0099F83E1099F81A30421838
:107A2000F6A1F548F8F756FCA079F34A2821FDF7AE
:107A30008FFB99F8010005EB8000AFF27001026B3B
:107A4000ED48F8F747FCE079EB4A0A21FDF780FBA7
:107A500099F82C20AFF26801E748F8F73BFCE07991
:107A6000E54A6021FDF774FB99F8010005EB800001
:107A7000AFF2A801826BE048F8F72CFC207ADE4ACE
:107A80000A21FDF765FB99F82D20AFF29C01DA4839
:107A9000F8F720FC207AD84A6021FDF759FB99F8C5
:107AA000010005EB8000AFF2DC01026CD248F8F770
:107AB00011FC607AD04A0A21FDF74AFB99F80110BF
:107AC00099F82E0001EB4000D04951F82020AFF288
:107AD0000411C948F8F7FEFB607AC74A3221FDF766
:107AE00037FB99F8010005EB8000AFF22011826CA2
:107AF000C148F8F7EFFBA07ABF4A0A21FDF728FB3F
:107B000099F83400C0F1090201E095E09EE0AFF27F
:107B10002011B948F8F7DEFBA07AB74A5F21FDF7DC
:107B200017FB99F8010005EB8000AFF26011026DC0
:107B3000B148F8F7CFFBE07AAF4A0A21FDF708FB1E
:107B400099F83520AFF25811AB48F8F7C3FBE07A4B
:107B5000A94A5F21FDF7FCFA99F8010005EB8000C6
:107B6000AFF29811826DA448F8F7B4FB207BA24ACB
:107B70000A21FDF7EDFA99F84520AFF2A8119E48C9
:107B8000F8F7A8FB207B9C4A5F21FDF7E1FA99F802
:107B9000010005EB8000AFF2CC11026E9648F8F7B9
:107BA00099FB607B944A0A21FDF7D2FA99F81E20CE
:107BB000AFF2E0119048F8F78DFB607B8E4A5F21B1
:107BC000FDF7C6FA99F81B2091A18B48F8F782FBC4
:107BD000A07B894A0A21FDF7BBFA99F81C00A0B3E3
:107BE0008FA18548F8F776FBA07B834A1E21FDF71D
:107BF000AFFA01248BA201212046FDF7A9FAA01CAF
:107C0000C4B2082CF6D399F827004FF0FF3101EBEE
:107C1000400189F82010042884BF072089F820003B
:107C200081A2012199F82000FDF792FA99F8270026
:107C30000E2840F0508217E099F81A3099F83D204C
:107C40007AA16D48F8F746FBEEE608E099F81A309D
:107C500099F83E2079A16848F8F73CFBE4E67BA15F
:107C60006548F8F737FBBFE77AA2012199F82000B1
:107C7000FDF76EFA00F02FBA99F827000E3889F850
:107C8000200099F8900000F00700012803D1F9F7CF
:107C9000ADFD89F81A00704C99F8010054F82020C5
:107CA000AFF2D8215448F8F715FB534A0A210120B6
:107CB000FDF702FA99F8090068A1421C4E48F8F74E
:107CC00009FB4D4A4B210120FDF7F6F999F8010017
:107CD00004EB8000AFF20C3182684748F8F7FAFAFB
:107CE000454A0A210220FDF7E7F95E49D9F89C00D0
:107CF000A1FB0021CA08514201EB810100EB4103C5
:107D000059A13D48F8F7E6FA3B4A4B210220FDF71E
:107D1000D3F999F8010004EB8000AFF25031026909
:107D20003548F8F7D7FA344A0A210320FDF7C4F999
:107D300099F83020AFF264312F48F8F7CBFA2E4A89
:107D40004B210320FDF7B8F999F8010004EB8000FE
:107D5000AFF2883182692848F8F7BCFA264A0A212E
:107D60000420FDF7A9F999F82F20D9F82C01032A4E
:107D700040D0009099F81A303EA11F48F8F7AAFAAF
:107D80001D4A28210420FDF797F999F8010004EB1A
:107D90008000AFF2C831026A1748F8F79BFA164A1A
:107DA0000A210520FDF788F936A11348D9F80821E2
:107DB000F8F790FA104A4B210520FDF77DF999F864
:107DC000010004EB8000AFF2FC31826A0A48F8F748
:107DD00081FA094A0A210620FDF76EF999F8010097
:107DE00004EB8000AFF21C41026B0348F8F772FA13
:107DF000014A4DE0A0E00000740200203328256411
:107E000029202D20256420200000000018020020D9
:107E1000464D20202020202D2025646D487A20000A
:107E2000284F4E29200000003E0000003128256424
:107E300029202D2025642020000000003228256400
:107E400029202D202564202000000000284F4646D0
:107E5000290000006F000000740100202D2025641F
:107E600000000000CDCCCCCC2D2025642E25642034
:107E7000560000002564282564292D202564487AB1
:107E8000202000002D2025642067722020000000A3
:107E90000A210720FDF710F999F83700F0B3FCA18B
:107EA000FD48F8F717FAFC4A4B210720FDF704F9C3
:107EB00099F8010004EB8000AFF2F041026BF64844
:107EC000F8F708FAF44A0A210720FDF7F5F899F8BF
:107ED0001D00072846D0F1A1EF48F8F7FBF9EE4A5C
:107EE0000A210820FDF7E8F80124AFF2C8020121B9
:107EF0002046FDF7E1F8601CC4B2092CF5D399F8CF
:107F00002700122808BF012204D00022132808BF2E
:107F1000012100D000211143162800E01DE00CBF14
:107F200001200020084322D0AFF2D802012199F8A5
:107F30002000FDF7C1F821E040F24D1190FBF1F176
:107F40004FF47A7390FBF3F0CDE9000199F81A3001
:107F5000D7A1D148F8F7BEF912E7DAA1CE48F8F771
:107F6000B9F9A0E7D9A1CC48F8F7B4F9B7E7AFF26F
:107F70004812012199F82000FDF79EF84FF6E850CD
:107F8000FCF7BEFFA7E000BF99F8400002287DD0B3
:107F9000D14C94F80004FF280CBF0121002194F873
:107FA000000400280CBF01200020084325D0CB4846
:107FB00090F80014FF290CBF0121002190F8000463
:107FC00000280CBF01200020084316D0F9F72EFB33
:107FD000C3496622030A4A7000228A7089F8132076
:107FE000CB7048710A718A71C9F8982099F80B0012
:107FF0003730C8711046FBF79DF8B84890F8000478
:1080000094F8001440EA0120C9F89400B5A1A248F0
:10801000F8F760F90121A04A0846FDF799F8D9F868
:108020009420B2A102F500539B48F8F753F99A4AFD
:1080300059210120FDF78CF8AEA19748D9F8982076
:10804000F8F748F9944A02210320FDF781F899F8DE
:10805000900000F00300022812D999A18E48F8F789
:1080600039F999F81F006FF0050101EBC000C1B2AA
:10807000894A0320FDF76CF84FF49670F9F7BEFFBC
:1080800000242B212046FDF77DFA00E04CE0601C27
:10809000C4B27F2CF5D39CA29EA17F48F8F71AF9B1
:1080A0007D4A02210520FDF707F89EA17A48F8F7DE
:1080B00011F9794A05210720FCF7FEFF9FA17648B8
:1080C000F8F708F9744A05210820FCF7F5FF4FF688
:1080D000E850FCF715FF9E4D002089F81500286830
:1080E00010F4006F5DD0286810F0010F7ED0286872
:1080F00010F4806F00F0EF83286810F0020F00F09A
:10810000BB864FF09046306910F4806F00F03387E3
:10811000286810F4005F01F04C80286810F4805F3C
:1081200001F0968201F0D4BCFCF792FE89A15A4876
:10813000F8F7D0F8584A05210220FDF709F872A295
:1081400088A15548F8F7C6F8534A1E210420FCF7C9
:10815000B3FF85A15048D9F89420F8F7BBF84E4AF0
:108160001D210620FCF7A8FF99F91400009099F949
:10817000133080A14848D9F89820F8F7ABF8464A60
:108180001D210720FCF798FF41F28830F9F736FFF0
:10819000FCF75EFE012089F80600152089F827000B
:1081A00099E77949086820F00100086099F82700EC
:1081B000F9F738FF002689F8086099F803000128CC
:1081C00004D0286810F4006F13D04BE040F6B830AC
:1081D000FCF70EFE286810F4006FFBD0C82089F869
:1081E0002A0089F8290089F8036000E013E101F012
:1081F00072BC1E20F9F702FF99F81500401CC1B2AD
:1082000089F81510D9F88C00814227D999F8050012
:10821000C04389F80500FCF71BFE012089F8030024
:1082200089F80A6099F8050090B199F8040089F876
:108230002700F9F7DBFA89F81A0099F82700F9F70F
:10824000F1FE00BF89F806604FF4FA6000F088BBC9
:1082500089F827606420F9F7D1FEF3E7286810F465
:10826000006FC6D099F8050070B199F80600012892
:108270000BD0022899F8270000F10100C0B289F85C
:10828000270003D00E2881E092E0B5E0C0E00000B6
:108290002D2047424620000074020020456E747273
:1082A00079204B45592020202D2C2B200000000048
:1082B000256428256429202D25642B25646B487AA4
:1082C000200000002D204742562000004B45592039
:1082D0004F4B21202020000003D0000805D00008CB
:1082E00039010020436F6465202D3E002558255834
:1082F000000000004B65792028417070292020255E
:108300003034582000000000762E31372F30372FC0
:10831000323600003C53544D33324633323E202532
:10832000732000006D61696C3A20726164696F644A
:108330006F6D40692E7561202000000068747470B4
:108340003A20726164696F646F6D2E6F726700000E
:10835000100400482020204B455920204F4B20215D
:1083600020000000257320004B6F64653A20253003
:10837000345820004B65793A202025303458202885
:1083800025642D25782900000010004084BF0120BD
:1083900089F82700C0B2F9F745FE00BF99F8270019
:1083A0000F2838BF89F8040040F6C41000F0D8BA8E
:1083B000FCF74EFD40F2DC50FCF71AFD99F828005E
:1083C000401CC0B289F82800032884BF012089F826
:1083D0002800D9F87000F9F71BFF642089F808001D
:1083E000012089F82100C820F9F708FEF02089F85B
:1083F0002A0089F82900D7E799F82700401CC0B265
:1084000089F827001628C9D9162089F82700CBE754
:108410001628F9D8C2E7FE48016821F00101016081
:10842000FCF716FD6420F9F7E9FD012689F80760DD
:10843000286810F0010F10D12320F9F7DFFD99F81B
:108440001500401CC0B289F81500D9F88C1088427C
:108450009CBF286810F0010FEED099F81510D9F8DC
:108460008C0081427CD93220F9F7C8FD99ED310AA0
:10847000B8EEC09A99ED320AB8EEC00A10EE100AB2
:1084800002F052FE41EC180B19EE100A02F04CFEFD
:1084900041EC100BB0EE481AF0EE681AFBF768F8E2
:1084A0009FEDDD1B51EC100B53EC112B02F07CFB0C
:1084B00002F0F2FA99F82E10072908BF0A3089F85D
:1084C0000D00D9F8C40000FB00F1D9F8C80000FB8A
:1084D000001002F03EFB41EC100BFBF7BDFC51EC31
:1084E000100B02F0D9FA801002F033FB41EC100BB4
:1084F000FBF7A2F951EC100B02F0FEFAC4B20C2CFF
:1085000088BF0C2499F8370058B3C5A1C748F7F7BE
:10851000E1FE0121C54A0846FCF71AFE99F90D0053
:1085200010F15A0FB4BF0121002110F13C0FCCBF54
:108530000120002008431AD0BDA1BC48F7F7CAFEAD
:10854000BA4A53210120FCF703FE4FF49670FCF762
:108550004FFCC820FCF74CFCBE20FCF749FC53E064
:10856000F4E0FFE7B4A1B148F7F7B4FED1E7092C76
:1085700088BF032005D8062C8CBF022089F83B60F9
:1085800001D989F83B00AFA1A848F7F7A3FEA74A95
:1085900053210120FCF7DCFD4FF49670FCF728FC1A
:1085A0004FF4C870F9F72AFD4FF41670FCF720FC61
:1085B0004FF4FA70FCF71CFC99F80D00401E40B215
:1085C00089F80D0002F0C5FA9FED9F1B53EC112BAB
:1085D00002F0CEF841EC100BFBF77EFC53EC102BB5
:1085E0009FED9B0B51EC100B02F0C2F801F0DAFF8B
:1085F000C9F85C0099F83700002814BF99F80D00FD
:108600006FF0590089F8000093A18848F7F762FEDF
:10861000864A02210620FCF74FFD4FF44870FCF714
:10862000E7FB286810F0010F7ED19FED898B9FED4D
:10863000869B8F4E6FF0590A4AF6AA2899F83B009C
:10864000009099F90D3022468AA17848F7F742FE4A
:10865000764A01210420FCF77BFDD9F85C0002F08A
:1086600063FD41EC100B88A153EC102B6F48F7F71A
:1086700031FE6E4A1E210820FCF71EFD286810F40A
:10868000005F0DD0286810F4805F33D06420F9F7C4
:10869000B5FCC6F80080286810F0010FCED012E1BA
:1086A00099F80D00401C89F80D004FF4FA70FCF7A2
:1086B0009FFB99F90D0002F04CFA53EC192B02F0D4
:1086C00057F841EC100BFBF707FC53EC102B51EC67
:1086D000180B02F04DF801F065FFC9F85C0099F83D
:1086E000370000281ABF99F80D0089F8000089F8B2
:1086F00000A0C7E799F80D00401E89F80D004FF45F
:108700001670FCF775FB99F90D0002F022FA53EC94
:10871000192B02F02DF841EC100BFBF7DDFB53ECAD
:10872000102B51EC180B00E06EE002F021F801F084
:1087300039FFC9F85C0099F8370000281ABF99F88A
:108740000D0089F8000089F800A09FE70020D9F803
:108750007C8089F8150089F82A0089F8290089F8B1
:10876000216040F6E4464645C1F2F481424649A103
:108770002E48F7F7AFFD2D4A0A210320FCF7E8FC4D
:108780004FF47A70FCF734FBB8F1C80F3CDD46A11A
:108790002648F7F79FFD254A05210720FCF78CFCAA
:1087A00099F81500401CC0B289F815001E282BD27C
:1087B0004CF25030FCF7A4FB286810F0020F1CD1DB
:1087C0004FF4FA60FCF714FB0020FCF76FFA4FF44B
:1087D0007A70FCF70DFB42F21070FCF791FBD9F8B0
:1087E0007C20B24201F3C8812AA11048F7F772FD3C
:1087F0000E4A0A210320FCF7ABFC99F81500401C37
:10880000C0B289F815005BE05DE0000000000000E8
:1088100000100040000000000000006066A64C4010
:10882000477261756E642042462D0000740200207C
:108830004572726F72210000477261756E6420424A
:10884000562D00004F4B20006666666666A64C40BB
:10885000000000000000F03F416D706C69742E2034
:108860005068617365202046696C747200000000D6
:10887000003000403C253032643E203C25643E20E0
:108880003C4625643E200000203C25302E33663EC9
:10889000202000002A2A2A202564206D56202A2A1A
:1088A0002A20202020000000436F696C20626C2E7B
:1088B000707265737320274D656E75270000000088
:1088C0001E28FFF475AF4FF49670F9F797FBFCF78D
:1088D000BFFA01F0FDB8FE48016821F00101016016
:1088E000286810F4806F10D12820F9F787FB99F8D9
:1088F0001500401CC0B289F81500D9F88C108842C8
:108900009CBF286810F4806FEED099F81510D9F844
:108910008C00814228D9FCF79BFA99F81D000728A2
:1089200010D0ECA1EE48F7F7D5FCED4A1E2103204C
:10893000FCF70EFCC820FCF75BFA4FF4C870F9F79F
:108940005DFBDFE04FF41670FCF752FA0120FAF7F6
:1089500085FB4FF4FA70F9F751FB4FF4C87000BF74
:10896000FCF746FA01F0B4B899F80500002801F0C8
:10897000AF8099F827000B2819D041F3A98011285E
:1089800015D005DCA0F10C01042901F2A1800EE054
:1089900015280CD005DC12285CD013287ED001F0FD
:1089A00097B8162803D04D2879D001F091B80E2839
:1089B00041F08E8040F6B830FCF71AFA99F81C00A6
:1089C00098B10020C74989F81C004FF480408861A5
:1089D0004FF09041082088624FF4FA60FCF708FAE3
:1089E0006420F9F70BFB01F073B8012089F81C0033
:1089F0008103BC4881624FF0904108208861322099
:108A0000F9F7FCFA99F81B004C3802F0B9F853EC6E
:108A10001A2B01F0ADFE02F06FF8C5B280210020E4
:108A2000FAF7BCFB4FF47A70FCF76AFA31210020A8
:108A3000FAF7B4FBB9210220FAF7B0FB4B21102062
:108A4000FAF7ACFB29460120FAF7A8FB3220F9F728
:108A5000D5FAC1E799F82F00032808BFC8203FF4D2
:108A60007FAF0120002689F82300FCF7F1F99E4929
:108A70009B48F7F72FFC9A4A0A210320FCF768FB72
:108A80004FF4FA70FCF7B4F9D9E929783D46474527
:108A9000C4BFDFF858A2DFF858B201E036E075E154
:108AA0001EDD00BFCAF800501920F9F7A7FAF8F741
:108AB0009DFEB042C4BF0646C9F870509BFBF5F05E
:108AC00099F80B1090FBF1F28AA18548F7F702FCA8
:108AD000834A10210520FCF73BFB6D1E4545E1DC78
:108AE00099F82F000228D9F870000CBFC9F8780057
:108AF000C9F87400D9F87000F9F78AFB4FF4FA60EE
:108B0000FCF776F9FCF7A4F900F0E2BFFCF7A0F956
:108B10000120F8F75DFD012689F8236089F80760D8
:108B200099F82F00032808D00020C9F80801F9F7A8
:108B3000D1FB4CF25030FCF7E3F989F8216070A1C9
:108B40006748F7F7C7FB664A0A210320FCF700FBDA
:108B500040F6B830FCF74CF989F82160D9F88C0060
:108B6000C0EB00108000F9F749FA68A15C48F7F7FC
:108B7000B1FB5B4A0A210320FCF7EAFA40F6B83061
:108B8000FCF736F9D9F88C0000EB8000C000F9F74B
:108B900035FA00252C461FEDE0BB00BF99ED310AE8
:108BA000B8EEC08A99ED320AB8EEC00A10EE100A8B
:108BB00002F0BAFA41EC190B18EE100A02F0B4FAFE
:108BC00041EC100BB0EE491AF0EE691AFAF7D0FC3E
:108BD00053EC1B2B51EC100B01F0E6FF01F05CFF96
:108BE00099F82E10072908BF0A300544C820F9F764
:108BF00005FA601CC4B2082CD0D3E81705EB5070FE
:108C000099F82F10C010032943D05A304042C9F8B8
:108C10000801B0F5B47FC4BFA0F5B470C9F808016D
:108C20000028BCBF00F5B470C9F80801F9F752FB81
:108C300089F82160D9F88C0032214843F9F7DEF930
:108C400099ED310AB8EEC08A99ED320AB8EEC00A41
:108C500010EE100A02F068FA41EC190B18EE100A37
:108C600002F062FA41EC100BB0EE491AF0EE691A0C
:108C7000FAF77EFC53EC1B2B51EC100B01F094FF28
:108C800001F00AFF99F82E10072908BF0A3007469D
:108C900006E06FF0580189F82160081AC9F8080148
:108CA000002FACBF3846784257283FDA99F82F009A
:108CB00003283BD019A10A48F7F70CFB084A0A2100
:108CC0000520FCF745FAC820FCF792F8962029E029
:108CD000001000402A2044454D4F202A000000008B
:108CE000740200200004004864A400082C04004022
:108CF00000D8B8052A20256420487A202A202000A0
:108D0000204E6F2046657272697465002054616B55
:108D100065204665727269746500000020457272B4
:108D20006F722100FCF764F864200EE0FCA1FE489D
:108D3000F7F7D0FAFC4A0A210520FCF709FA4FF4AC
:108D4000FA60FCF755F840F6C410FCF751F84FF400
:108D50007A70F9F753F9FCF77BF899F82F0001289E
:108D600004BFD9F80801C9F80C0106D0022804BFD5
:108D7000D9F80801C9F8100103D0D9F80801C9F8D9
:108D80001401002089F8070000F0A2BEB9F8940091
:108D9000C0F30721C0B211FB0011091A133101FB06
:108DA0000012101A3B304FF47F42C0B202EA012198
:108DB0000844D9F8981088423CD1F8F737FCD9F824
:108DC0009410884236D1D9A1D748F7F783FAD64A0A
:108DD0001E210320FCF7BCF94FF4FA70FCF708F8E9
:108DE0004FF47A70FCF704F8B9F89810D54B552277
:108DF000D24889F81420D24C4FEA112C5C60D24C36
:108E00005C60427099F813208270B9F89420CF4CBE
:108E1000130AC370427180F804C0817199F826105A
:108E2000C1712046F8F730FD08222146C348F8F703
:108E30004DFDFEE7C6A1BC48F7F74CFABA4A00213F
:108E40000120FCF785F9C7A1B748F7F743FAB64AFE
:108E500000210320FCF77CF96420FBF7C9FF5020B8
:108E6000FBF7C6FF6420FBF7C3FF99F81300401C13
:108E700089F81300FEE700BF99F827004D282AD093
:108E80004FF47A70FBF7B4FF99F80500E8B399F84E
:108E90002700401E10F0FF0089F8270004BF0E20B5
:108EA00089F8270001D00F2801D289F8040099F829
:108EB0000600012801BF99F827000E28162089F81E
:108EC000270040F6C410FBF793FF99F82700F9F745
:108ED000A9F8C8204BE099F9130006281FDAA64824
:108EE00099F81F10014411F80C2C521C02F00F02CB
:108EF00001F80C2CC178027841EA0231427880787E
:108F0000120242EA0010084300E01AE0C9F8980093
:108F10004FF44870FBF76CFF4FF4967027E097A171
:108F20008148F7F7D7F9804A00210320FCF710F9B0
:108F30006420FBF75DFF5020FBF75AFF4FF4FA6007
:108F400015E099F83000012814BF0120022089F8AB
:108F50003000C0B2F8F73CFB012089F82100C8209E
:108F6000F9F74CF8642089F8080000F0B1BDF9F772
:108F700045F800F0ADBDDFF81882D8F8000020F009
:108F80000100C8F80000306910F4806F47D14FF03D
:108F9000FF0B4FF0320A01253C20F9F72FF899F822
:108FA0001500401CC0B289F81500D9F88C10884211
:108FB00031D989F82350D8F8000020F00100C8F812
:108FC0000000FBF745FF99F8060001282CD089F82E
:108FD00005B00F2089F8270089F806506D495248DE
:108FE000F7F778F94FF4FA60FBF702FF01214E4AD8
:108FF0000846FCF7ADF8306910F4806FFBD04FF4F1
:109000007A70FBF7F5FEF9F7F5FFC9F89C00FBF75E
:109010001FFF89F808A0306910F4806FBCD099F860
:10902000230078B100F054BD002089F8050089F8CC
:10903000270089F8060058A13B48F7F74BF94FF491
:10904000FA70D1E74FF47A70FBF7D2FE99F82F004F
:10905000401CC0B289F82F00042804BF012089F801
:109060002F00C0B201282AD002281CBFD9F87400F2
:10907000C9F8700033D000BF4FF0A040816841F0C4
:1090800001018160D9F87000F9F7C2F899F8300051
:10909000F8F79EFA6420F8F7B1FF012589F821500E
:1090A0006420F8F7ABFF4FF49660FBF7A1FE89F858
:1090B0002150502089F808004FF4FA7057E74FF418
:1090C0000070B0614FF0A04140200863D9F87400EF
:1090D000C9F87000A520C9F8A4006E201FE04FF465
:1090E0000070B0624FF0A040802101634FF44072E5
:1090F00092FAA2F20021B2FA82F2D14000EB810092
:10910000016B21F4F86141F080010163D9F8780026
:10911000C9F8700040F22B10C9F8A400772045E090
:10912000204F4B210000000074020020204F4B21F3
:1091300020202020202020202000000039010020B5
:109140002301674500200240AB89EFCD00D4000821
:1091500020726164696F646F6D40692E75612020B3
:109160002000000020202020204552524F52212074
:109170002020202020000000500000202020455208
:10918000524F5221204E3E3D35202120200000002C
:1091900000100040D86B0008202A2A2A20204558B9
:1091A000495420202A2A2A2000000000C9F8A800DB
:1091B00062E7FC4E306820F00100306099F827002B
:1091C0000C2877D009DC0C2873D2DFE800F01F757B
:1091D00081929EAAB6D4E0EFEDEC12286BD008DCA9
:1091E000A0F10D00052864D2DFE800F0F2F1F0EF05
:1091F000EE00152878D004DC132876D0142875D01A
:109200001EE2162873D04D2872D019E2286810F497
:10921000005F3BD11420F8F7F1FE99F81500401CCF
:10922000C0B289F81500D9F88C1088422AD90125D6
:1092300089F82350306820F00100306099F8300040
:10924000012806BF022089F8300089F8305099F8CB
:109250003000F8F7BDF90021084600F0ABFF4FF4ED
:109260007A70FBF7C5FD962089F808000020C9F840
:109270009050C9F8580089F82150C820F8F7BEFE70
:1092800000F029BC286810F4005FC3D099F82300CF
:1092900078B999F81D00072814BF1C201E2099F8E2
:1092A0003110491CC9B289F831108142C8BF89F810
:1092B0003100C5E1ACE035E199F83900401CC0B29D
:1092C00089F83900192884BF192089F83900B7E1D5
:1092D00099F82500401CC0B289F82500032884BFF6
:1092E000032089F82500ABE183E13EE15EE18CE1FA
:1092F00096E199F84800401C40B289F848000528DA
:10930000C4BF052089F848009AE199F83300401E4F
:10931000C0B289F83300FF2804BF002089F8330069
:109320008EE199F83C00401CC0B289F83C0004284A
:1093300084BF042089F83C0082E199F82F000128BD
:109340000DD099F83E00401CC0B289F83E001428A8
:1093500084BF142089F83E00F9F7B2F870E199F85B
:109360003D00401CC0B289F83D00142884BF142081
:1093700089F83D00F0E799F82C00401CC0B289F84C
:109380002C000A2884BF0A2089F82C0058E199F89B
:109390002D00401CC0B289F82D00032884BF032093
:1093A00089F82D004CE120E013E0FFE799F82E004A
:1093B000401CC0B289F82E00072884BF072089F816
:1093C0002E00F9F78FFD3BE19DE084E06BE037E094
:1093D0002AE099F83400401EC0B289F83400FF2812
:1093E00004BF002089F834002AE199F83500401CB8
:1093F000C0B289F83500062884BF062089F83500F8
:10940000C0B200EBC00101EB00106749486317E1EF
:1094100099F84500401CC0B289F84500032884BF74
:10942000032089F845000BE199F81E00401CC0B2EA
:1094300089F81E005A2884BF5A2089F81E00FFE0D0
:1094400099F81C00012845D199F81B00401CC0B2B6
:1094500089F81B00652884BF652089F81B00C0B20D
:109460004C3801F08DFB53EC1A2B01F081F901F01F
:1094700043FBC5B280210020F9F790FE4FF47A70CB
:10948000FBF73EFD31210020F9F788FEB9210220CB
:10949000F9F784FE4B211020F9F780FE29460120C0
:1094A000F9F77CFECCE099F80900401CC0B289F8BD
:1094B0000900032884BF032089F8090000F066FB37
:1094C00099F82F00FCF7E2F9F9F70CFDD9E915013D
:1094D00000F070FEB4E099F83600401EC0B289F882
:1094E00036001E283CBF1E2089F83600F9F782FDA1
:1094F000C9F89C0047F23050FBF702FDF9F77AFDFE
:10950000C9F89C009CE099F83000401CC0B289F872
:109510003000022884BF022089F83000C0B2F8F77A
:1095200057F88DE099F82F0002280CD0D9F8740074
:10953000411EC9F87410D9F8A800814238BFC9F893
:1095400074000CD20CE0D9F87800411EC9F87810EC
:10955000D9F8A800814238BFC9F8780000D308467E
:10956000C9F87000F8F754FE6AE099F82F00032854
:1095700009D1D9F80801401CC9F808011428C4BF52
:109580001420C9F80801D9F80801401CC9F80801DD
:10959000B0F5B47FA4BF0020C9F80801F8F79AFE1F
:1095A0004EE00000001000400044014099F81D000A
:1095B000072816D0FBF74CFCAFF6E801FD48F6F79C
:1095C00089FEFC4A1E210320FBF7C2FDC820FBF7E1
:1095D0000FFC4FF4C870F8F711FD00BFFBF738FC23
:1095E0002EE00120F9F73AFD4FF49670FBF700FCEE
:1095F00026E099F83700401CC0B289F837000128EE
:1096000084BF012089F837001AE0022089F806009B
:109610004D2089F827004FF4FA70FBF7E9FBDDE7EE
:1096200099F81F00401CC0B289F81F000F2884BFA2
:109630000F2089F81F00FBF70BFC3220F8F7DEFC47
:1096400099F80A00002808BF40F6C41076D136E227
:10965000D94E306820F00100306099F827000C28BE
:109660006DD009DC0C285CD2DFE800F01F5C6A7664
:109670008894A0BECAD6E4F1122879D008DCA0F103
:109680000D0005284DD2DFE800F0F9F8F7F6F500F7
:1096900015286ED004DC13286CD014286BD007E298
:1096A000162869D04D2868D002E2286810F4805F3F
:1096B00029D11E20F8F7A2FC99F81500401CC0B271
:1096C00089F81500D9F88C10884218D9012089F83A
:1096D0002300316821F00101316099F83B10491CE9
:1096E000C9B289F83B10032988BF89F83B004FF4C1
:1096F000C870FBF77DFB0320C9F89000EBE12868F8
:1097000010F4805FD5D099F8230050B999F8310052
:10971000401E10F0FF0089F8310004BF012089F8D5
:109720003100C5E199F83900401EC0B289F839000E
:10973000FF2804BF002089F83900B9E1C1E19EE0AB
:1097400099F82500401E10F0FF0089F8250004BF9D
:10975000012089F82500ABE199F84800401E40B28D
:1097600089F848000028BCBF002089F848009FE124
:109770000FE176E136E151E17FE189E199F83300CB
:10978000401CC0B289F83300062884BF062089F83F
:1097900033008DE199F83C00401E10F0FF0089F87D
:1097A0003C0004BF012089F83C0081E199F82F00BA
:1097B00001280BD099F83E00401EC0B289F83E0047
:1097C000FF2804BF002089F83E000AE099F83D0018
:1097D000401EC0B289F83D00FF2804BF002089F870
:1097E0003D00F8F76DFE63E199F82C00401EC0B211
:1097F00089F82C0003283CBF032089F82C0057E18E
:1098000099F82D00401EC0B289F82D00FF2804BF32
:10981000002089F82D004BE199F82E00401EC0B2BF
:1098200089F82E00FF2804BF002089F82E00F9F7E0
:1098300059FB3DE199F83400401CC0B289F834006E
:10984000092884BF092089F8340031E1FFE799F83D
:109850003500401EC0B289F83500FF2804BF002043
:1098600089F83500C0B200EBC00101EB001053498C
:1098700048631DE17EE065E04CE018E00BE099F8FC
:109880004500401E10F0FF0089F8450004BF01208C
:1098900089F845000CE199F81E00401EC0B289F815
:1098A0001E0050283CBF502089F81E0000E199F8A6
:1098B0001C00012845D199F81B00401EC0B289F850
:1098C0001B0058289CBF592089F81B00C0B24C3897
:1098D00001F056F953EC1A2B00F04AFF01F00CF995
:1098E000C5B280210020F9F759FC4FF47A70FBF7DC
:1098F00007FB31210020F9F751FCB9210220F9F7CB
:109900004DFC4B211020F9F749FC29460120F9F7BD
:1099100045FCCDE099F80900401EC0B289F8090065
:10992000FF2804BF002089F8090000F02FF999F8FA
:109930002F00FBF7ABFFF9F7D5FAD9E9150100F0D5
:1099400039FCB5E099F83600401CC0B289F8360001
:109950005A2884BF5A2089F83600F9F74BFBC9F81A
:109960009C0047F23050FBF7CBFAF9F743FBC9F8FC
:109970009C009DE099F83000401E10F0FF0089F82F
:10998000300004BF012089F83000C0B2F7F720FE94
:109990008EE099F82F00022812D0D9F87400411CEB
:1099A000C9F87410D9F8A400814288BFC9F87400BE
:1099B00012D912E07402002000100040004401405F
:1099C000D9F87800411CC9F87810D9F8A400814270
:1099D00088BFC9F8780000D80846C9F87000F8F7C1
:1099E00017FC65E099F82F000328D9F80801A0F1C9
:1099F0000100C9F808010AD00028B8BF4FF4B470BC
:109A000002DA00BFC9F80801F8F764FC50E010F171
:109A1000140FB8BF6FF01300F6DAF3E799F81D00E2
:109A2000072816D0FBF714FAAFF658515448F6F74A
:109A300051FC534A1E210320FBF78AFBC820FBF789
:109A4000D7F94FF4C870F8F7D9FA00BFFBF700FA5E
:109A50002EE00120F9F702FB4FF49670FBF7C8F9EE
:109A600026E099F83700401EC0B289F83700FF2879
:109A700004BF002089F837001AE0022089F80600A8
:109A80004D2089F827004FF4FA70FBF7B1F9DDE7B4
:109A900099F81F00401EC0B289F81F000C283CBF77
:109AA0000C2089F81F00FBF7D3F96420F8F7A6FA19
:109AB00099F80A00002808BF4FF4FA6001D1FBF7BB
:109AC00097F94FF49670F8F799FA012089F8210078
:109AD000002089F82300D9F89000401CC9F89000B4
:109AE000B0F5E04F10D30025C9F89050D9F87C00AC
:109AF000B0F57A7F3CBF012089F82100FBF7D4F94B
:109B000089F80E5089F847501E484AF6AA2101608C
:109B1000FDF710B800283CF48BA8401EFDD1FCF7DF
:109B200087B800283CF42CA9401EFDD1FCF728B9C9
:109B30004FF03C0BFCF70ABFEE67FCF794BF002028
:109B4000C9F80001FDF7E2B81720C9F82801FDF7B0
:109B50000DBE00BF40F6E4420B490948F6F7BAFBD8
:109B6000074A0A210320FBF7F3FA4FF47A70FBF758
:109B70003FF9FEF70CBE00BF40F6E442FEF734BEEC
:109B8000740200200030004094880008D249162258
:109B9000487A404202EBC02202F1006202F57042B4
:109BA00092F8002C81F83B20012202EBC02202F146
:109BB000006202F5704292F8002C81F8392081F899
:109BC0003A20022202EBC02202F1006202F570424A
:109BD00092F8002C81F82520032202EBC02202F12A
:109BE000006202F5704292F8002C81F83C200422B9
:109BF00002EBC02202F1006202F5704292F8002CE2
:109C000081F83D20222202EBC02202F1006202F51F
:109C1000704292F8002C81F83E20052202EBC0220F
:109C200002F1006202F5704292F8002C81F83020B7
:109C3000062202EBC02202F1006202F5704292F8A5
:109C4000002C81F82C20252202EBC02202F10062B8
:109C500002F5704292F8002C81F82D20072202EBC9
:109C6000C02202F1006202F5704292F8002C81F8E5
:109C70002E20082202EBC02202F1006202F570429F
:109C800092F8002C81F83320092202EBC02202F165
:109C9000006202F5704292F8002C81F835200A2209
:109CA00002EBC02202F1006202F5704292F8002C31
:109CB00081F845200B2202EBC02202F1006202F57E
:109CC000704292F8002C8A77182202EBC02202F12F
:109CD000006202F5704292F8002C81F834200C22C8
:109CE00002EBC02202F1006202F5704292F8002CF1
:109CF00081F848200D2202EBC02202F1006202F539
:109D0000704292F8002CCA760E2202EBC02202F1B9
:109D1000006202F5704292F8002C81F842200F2276
:109D200002EBC02202F1006202F5704292F8002CB0
:109D300081F83620102202EBC02202F1006202F507
:109D4000704292F8002C81F82F20122202EBC022E0
:109D500002F1006202F5704292F8003C112202EB1F
:109D6000C02202F1006202F5704292F8002C43EA30
:109D700002224A675A2A7CD3212202EBC02202F136
:109D8000006202F5704292F8003C202202EBC022F1
:109D900002F1006202F5704292F8002C43EA0222BE
:109DA0008A675A2A66D3142202EBC02202F10062AB
:109DB00002F5704292F8002C132303EBC02303F149
:109DC000006303F57043C1F80C2193F8003C002BAD
:109DD0001CBF02F58072C1F80C211A2202EBC022CE
:109DE00002F1006202F5704292F8002C192303EB95
:109DF000C02303F1006303F57043C1F8102193F809
:109E0000003C002B1CBF02F58072C1F810212422F7
:109E100002EBC02202F1006202F5704292F8002CBF
:109E2000232303EBC02303F1006303F57043C1F860
:109E3000142193F8003C002B1CBF02F58072C1F87E
:109E40001421152202EBC02202F1006202F57042D9
:109E500092F8002C81F831201F2202EBC02202F17F
:109E6000006202F5704292F8002C81F83720172228
:109E700001E02BE02DE002EBC02000F1006000F5D6
:109E8000704090F8000C0877144890F800040875AA
:109E9000134890F80004C874124890F80004124A5D
:109EA00092F8002440EA0220C1F894000F4890F88C
:109EB00000040F4A92F8002440EA0220C1F89800FA
:109EC0000C4890F8000481F8260070475A224A672F
:109ED00052E75A228A6766E70000002001D0000896
:109EE00002D0000805D0000803D0000806D0000802
:109EF00004D0000807D000082DE9F047644C654DF8
:109F000020462DED028B90F8248090F83A0094F9C9
:109F10000D20614E470017FB08F1002A68DBA07F87
:109F20009042BCBFBDEC028BBDE8F08794F83C00CA
:109F3000012815D0022822D0032842D004280BD1B2
:109F4000C2EB02104000B5FBF0F0C4F8A010F062C4
:109F5000306840F001003060BDEC028BBDE8F08756
:109F60004FF4C860B5FBF0F0C4F8A010F0623068A0
:109F700040F001003060BDEC028BBDE8F087322A72
:109F80000EDA4FF44870B5FBF0F0C4F8A010F062A0
:109F9000306840F001003060BDEC028BBDE8F08716
:109FA0004A2ADDDD40F6FC00B5FBF0F0C4F8A01055
:109FB000F062306840F001003060BDEC028BBDE81B
:109FC000F087672012FB00F08212A2EBE0704FF4E2
:109FD000967210FB02F0B5FBF0F0C4F8A010F0622E
:109FE000306840F001003060BDEC028BBDE8F087C6
:109FF00094F83430D4F800019842CEBF12F1500FDB
:10A00000BDEC028BBDE8F08794F82E00012804BF58
:10A01000BDEC028BBDE8F087022808D194F830002F
:10A020003222A2EB4000D4F8F420904298DC94F85D
:10A030003300F6EE000A00EE100A4FF0BE09B8EE4B
:10A04000400A20EE200A10EE100A01F06DF89FED94
:10A05000141B53EC112B00F0D7FA41EC180B4046BF
:10A0600000F08EFD53EC182B00F082FB00F044FD55
:10A07000C0B217FB00F0C4F8A000B5FBF9F0F06225
:10A08000306840F001003060AEE7000000000000E2
:10A0900000000020007C9200001000400000000042
:10A0A000000000000000E03F002808BF70472DE9D5
:10A0B000F34F0027CD215A3010FB01F0C112A1EB64
:10A0C000E070C0EBC000401C019EDFF8E49000F09F
:10A0D000FF084FF0100A182E2FD200BF16F0070FFE
:10A0E00008BF0027802000EB5700C7B208200124DA
:10A0F000A0EBD600401EC0B200F1B00B4FF40041FF
:10A1000008EB0400C9F82810401EC5B20BF0FF0090
:10A1100000F006F90AEB151000F002F905F00F0047
:10A1200000F0FEF8002000F017F9601CC4B2082C03
:10A13000E4D3701CC6B2182ED0D301980026002894
:10A140009CBF02B0BDE8F08F16F0070F08BF0027D4
:10A15000802000EB5700C7B208200124A0EBD600F6
:10A16000401EC0B200F1B00B4FF4004108EB0400F8
:10A17000C9F82810401EC5B20BF0FF0000F0D0F85F
:10A180000AEB151000F0CCF805F00F0000F0C8F84D
:10A19000384600F0E1F8601CC4B2082CE4D3701C0F
:10A1A000C6B201988642CFD302B0BDE8F08F00005E
:10A1B000000400482DE9F05FDFF8909007462DED90
:10A1C000048B99F80B40002C04BFBDEC048BBDE858
:10A1D000F09F1F4E00254FF4B47A9FED1E9A08465B
:10A1E00000F0B7FC8B46804699F80B00BAFBF0F004
:10A1F00000FB0572B2F5B47FA8BFA2F5B4724BECB8
:10A20000188B00EE102AB8EEC00A20EE090A10EEF4
:10A21000100A00F089FF41EC100BF9F7F1FC53EC48
:10A22000182B51EC100B00F0BFFC53EC182B00F076
:10A23000EBF900F061FC26F8020B641E05F1010544
:10A24000D2D1BDEC048BBDE8F09F000000000020DF
:10A25000A00B00204BFA8E3C2DE9F041264D002644
:10A260002DED0A8BF0EE608AB0EE40CA60279FEDBC
:10A2700024AB9FED259BDFED26CA9FED27BB304623
:10A2800000F067FC884648EC110B044653EC1A2B8F
:10A2900051EC110B00F088FC53EC192B00F068FA1C
:10A2A00000F080F900EE100AF9F70EFDB0EE6C8AAE
:10A2B00053EC1B2B0CEE008A48EC104B51EC100BAE
:10A2C00000F072FC53EC192B00F052FA00F06AF91E
:10A2D00000EE100AF9F7F8FC08EE808A761C7F1E63
:10A2E000BCEEC80A10EE100A25F8020BC7D1BDEC6F
:10A2F0000A8BBDE8F0810000600C00200000000027
:10A30000A7E8482EFF211940000000000000584037
:10A3100000000045000000007DAEB6627FD93240EB
:10A320000C494FF400428A624FF090439A62002237
:10A3300010238B6210F0800F4FF0080314BF8B6165
:10A340008B6210238B614006521C000ED2B2082A89
:10A35000EED37047000400480C494FF400428A6273
:10A360004FF090439A61002210238B6210F0800F0F
:10A370004FF0080314BF8B618B6210238B61400682
:10A38000521C000ED2B2082AEED3704700040048D7
:10A3900010B52DED048BB0EE608AF0EE408A18EE19
:10A3A000100A00F0C1FE224C41EC190B607E00EE59
:10A3B000100AF8EE400A88EE200A30EE280A10EE65
:10A3C000100A00F0B1FE41EC100BB0EE491AF0EEAD
:10A3D000691AF9F7CDF89FED181B51EC100B53ECEF
:10A3E000112B00F0E1FB00F057FB94F82F1003292C
:10A3F00007D1D4F81411084494F83010022908BF8A
:10A40000C01C94F9001008445A305B2805DC10F198
:10A410005A0F06DBBDEC048B10BDBDEC048B5B203A
:10A4200010BDBDEC048B6FF0590010BD00000000A2
:10A4300000000020000000000000006066A64C4004
:10A4400010B5FAF705FD07A10A48F5F743FF094AD9
:10A450000A210320FAF77CFEBDE810404FF4FA70A1
:10A46000FAF7C6BC20504C4541534520574149544A
:10A470000000000074020020384901F2411091F8F8
:10A480003B20827591F83920427081F83A2091F88A
:10A490002520827091F83C20C27091F83D20027115
:10A4A00091F83E2080F8222091F83020427191F8F6
:10A4B0002F20027491F82C20827191F82D2080F8C1
:10A4C000252091F82E20C27191F83320027291F864
:10A4D0003520427291F8452082728A7FC27291F8CB
:10A4E00048200273CA7E427391F84220827391F829
:10A4F0003620C273B1F87420130A43748274B1F821
:10A500007820130A80F8203080F82120B1F80C213F
:10A51000130AC3740275B1F81021130A43768276C8
:10A52000B1F81421130A80F8233080F8242091F820
:10A53000312042750A7FC27591F834200276B1F855
:10A540005420130AC3760277B1F85820130A4377D0
:10A55000827791F83710C177704700000000002023
:10A5600010B500290AD00878002807D0054878449B
:10A57000F6F71CFC002801D0002010BD02487844EA
:10A5800010BD000006280000FE27000081F00041F9
:10A59000704780F00040704721F00041704720F084
:10A5A0000040704721F00042A2F16052B2F5801FD6
:10A5B00001F0004328BFD2F17F6C0BD95FEA001C89
:10A5C00043EAC20242EB507018BF704728BF20F028
:10A5D00001007047B2F5801FBCBF184670474FEAB4
:10A5E000410C1CF5001F02D2084600F013BE70B5E6
:10A5F00000F084FB00000089FFF7F6BF4FF0004039
:10A60000A0F580007047000010B591EA030F48BF25
:10A6100083F0004300F1A684841A71EB030C05D289
:10A62000121943EB0C03001B61EB0C01DFF824E172
:10A630004FEA1154A4EB135C1EEA430F18BF9EEAC5
:10A64000445F73D023EA0E03DCF1200E21EA0451AB
:10A6500043F4801332D322FA0CFE10EB0E0023FADF
:10A660000CFE41EB0E01CCF1200E03FA0EFE10EBB6
:10A670000E0051F10001B1F5801FCCF1200E32D255
:10A6800001EB045112FA0EF2BDE8104058BF7047BA
:10A69000401C38BF5FEA420218BF7047002814BF51
:10A6A00020F0010041F100014FEA410313F5001FC2
:10A6B00038BF7047A1F1C04100F06EBB012A43EBE7
:10A6C0000302ACF1200CDCF11F0E32BF4FF0000E84
:10A6D00023FA0CF310EB030041EB0451B4EB115FD0
:10A6E000D0D0A1EB045101F5801149085FEA300098
:10A6F00001EB04510ED350F1000038BF12FA0EFEE8
:10A7000008D1BDE81040C9E7401C38BF5FEA4202EB
:10A71000CAD1C3E7BDE810404FEA410313F5001F5B
:10A7200038BF7047A1F1C04100F036BB9EEA445FDC
:10A7300008D011EA5E0FBDE8104004BF01F00041EF
:10A7400000207047BDE8104070B500F0D7FA00BF98
:10A7500064FBBE3E0000E0FF491058BFC1F140411C
:10A760005B1058BFC3F140438B42EFF3008070474A
:10A770002DE9C04130B4DFF8A0C23CEA111418BF83
:10A780003CEA131400F0EC8081EA03051CEA111482
:10A7900044EAD57418BF1CEA131500F0C780A4EB77
:10A7A00005044FF0004545EAC12145EAC32341EACB
:10A7B000505143EA525304F17F74994204F5003436
:10A7C0004FEAC0204FEAC22208BF904200F09C80AE
:10A7D0004FEA13650FF24016765D4FEA134506FB0C
:10A7E00005F7C7F1807706FB07F74FEAD737A7FBD6
:10A7F00003687642C8F58038A7FB06CE38BFA8F1BB
:10A80000010807FB08E64FF0000EA6FB028CE6FBF2
:10A8100003CEDCF1000CCEF1004E38BFAEF1010EDC
:10A82000A6FB0C584FF000074FF00005E6FB0E8723
:10A83000A1FB08C6A0FB07CE16EB0E0645F10005EE
:10A84000E1FB076515F1E04E7EBFA4F580345FEAB9
:10A8500046066D4116F1800745F100054FEA1727BE
:10A860004FEA066647EA0567A6F1DE46B6F1805F65
:10A870004FEA15251FD9384624F0010C05EBC471A9
:10A88000BCF1FE6F01EB0C1102D8F0BCBDE80081F9
:10A8900024425CBF01F5801E9EEAC47F02D4F0BC56
:10A8A000BDE80081244238D4F0BCA1F1C041BDE82C
:10A8B000004100F071BA4FEAD22242EA43524FEA15
:10A8C000D323A7FB02864FEAD02040EA415007FB82
:10A8D00003661EEA0E0F4FEAD12105FB026658BF40
:10A8E000A6EB0056B6EB00564FEA520E4EEAC37E78
:10A8F00018EB0E0E56EB530EBDD518EB02085E4159
:10A900007F1C55F10005B6E74FF480154FF00007A6
:10A910004FF000064FF00008ADE7F0BC4FF000002C
:10A9200001F1C04101F00041BDE8008111EA0C1FB6
:10A930000CEA131500D00CE013EA0C1F00F0258080
:10A940004FF00000F0BC81EA030101F00041BDE8D6
:10A950000081F0BCBDE8004181EA030100F01CBAAF
:10A96000F0BCBDE8004170B500F0C8F9097EFC3EBE
:10A9700000F007B881EA03014FF0000001F0004148
:10A98000704781EA030100F007BAF0BCBDE800415E
:10A990004FF0000021497047FFFDFBF9F7F5F4F295
:10A9A000F0EEEDEBE9E8E6E4E3E1E0DEDDDBDAD86A
:10A9B000D7D5D4D3D1D0CFCDCCCBCAC8C7C6C5C4C8
:10A9C000C2C1C0BFBEBDBCBBBAB9B8B7B6B5B4B3DF
:10A9D000B2B1B0AFAEADACABAAA9A8A8A7A6A5A4CA
:10A9E000A3A3A2A1A09F9F9E9D9C9C9B9A9999988E
:10A9F0009797969595949393929191908F8F8E8E31
:10AA00008D8C8C8B8B8A89898888878786858584BD
:10AA100084838382828181800000FF070000F87FA9
:10AA200051EA030C17D41CF5801F58BFBCF5801FDA
:10AA300000F10680994218BF704708BF90427047E6
:10AA400007D711F5801F58BF13F5801F19D49942FD
:10AA50007047894270471CF5801F08D5BCF5801FE0
:10AA6000F7D58B4218BF704708BF824270474FF43A
:10AA7000001C1CEB410F38BF1CEB430F01D28B4273
:10AA8000704770B500F03AF9922449004FF0005138
:10AA90004FF08053FFF760BE4FEA41034FEA535334
:10AAA000A3F58063D3F11E03C8BFD3F1210C0CDDE5
:10AAB0004FF0004242EAC12242EA505232FA03FC0D
:10AAC0008CEAE17CACEBE1707047102BC4BF002036
:10AAD000704703F5787CBCF1FF3F04D06FF0004273
:10AAE00082EA2100704770B500F008F9499224808D
:10AAF00000207047F2E700004FEA1153A3F580638E
:10AB0000D3F11E03A8BFD3F1200C08DB4FF00042A5
:10AB100042EAC12252EA505232FA03F07047094227
:10AB20000BD4102BC4BF0020704703F5787CBCF118
:10AB3000FF3F05D04FF0FF3070474FF000007047E7
:10AB400070B500F0DBF800BF499224800020704708
:10AB5000F0E710F0004248BF4042B0FA80F310FA2C
:10AB600003F10AD0C3F11D0303F580634FEA41509E
:10AB700002EB035202EBD12170474FF00000704707
:10AB8000B0FA80F310FA03F10AD0C3F11D0303F504
:10AB900080634FEA41504FEA035202EBD1217047E4
:10ABA0004FF0000070470000DFF848C170B51CEAA4
:10ABB000111E1EBF1CEA13159EEA0C0F95EA0C0F1E
:10ABC00000F06F8081EA030423EA4C134EEAD47E3E
:10ABD00021EA4C1141F4801143F48013AE44A1FBEF
:10ABE000024CA0FB0365AEF17F7E361955EB0C05D8
:10ABF000A1FB034C4CF10003A0FB021C16EB0C065E
:10AC0000654153F10003094218BF46F0010613F4F1
:10AC1000007F0BD14FEA03314FEA0530340341EA9C
:10AC2000155140EA16506FF003020AE04FEAC321C3
:10AC30004FEAC520F40241EA555140EA56506FF000
:10AC4000020202EB2E4201EB025585EACE710AD0D8
:10AC50005FEA440C18BF24F0004450F1000041F1B9
:10AC6000000120EAD47040F2FE7C624500D270BD43
:10AC7000A84214BF4FF080444FF04044002E08BF5C
:10AC80000024BEF1806FA8BFA1F1C041BDE87040B3
:10AC900080F282804FF0000001F1C04101F00041DC
:10ACA00070479EEA0C0F0CEA131518BF95EA0C0FBB
:10ACB00006D04FF0000081EA030E0EF0004170BD97
:10ACC00000F01CF88900013E00F007B800F009B858
:10ACD0004FEA430C5FEA5C5C08D081EA030100F0B4
:10ACE0005BB84FEA410C5FEA5C5CF6D14FF00000C4
:10ACF000014970470000FF070000F87F0EF1020EC7
:10AD00002EF0030E5EF8046B364205D4012A43EBA5
:10AD1000030515F5001F12D8012841EB010C1CF5A5
:10AD2000001F0CD80ED14FEAD17C15F5001F0CEB9B
:10AD30004C0C0CF1020C08BF4CEBD37C04E04FF040
:10AD4000080C01E04FEAD37C0CEB4C0526FA05F623
:10AD500006F00706B6F1040C06D20EEB860CBDE831
:10AD600070404CF0010C6047DFE80CF0090B020268
:10AD70004FF000414FF00000A1F5002170BD1946D1
:10AD80001046012851EB010418BFD4F5001484BF0C
:10AD9000002001F0004170BD0808A0F500114FEA45
:10ADA0003101704791EA030F10B581F000413FF582
:10ADB00033AC83F0004300F0D5B800002DE9F0413A
:10ADC00001F5801CBCF5001FC0F2A9804FEA115CA0
:10ADD00021EA0C510CF1FD0C41F480115FEA5C0C8E
:10ADE0000CF5C07C01D34000494130A4890241EAFE
:10ADF000905187028E0E0A0CA45D04FB04F602FB40
:10AE000006F6C6F14046A4FB0662F60D46EA422667
:10AE100006FB06F4A4FB01235242C3F1404338BFB2
:10AE20005B1EA6FB02420024E6FB0324D20B42EA8F
:10AE30004446A6FB0623A1FB02E2A3FB07E4E3FBD7
:10AE400061426442C2F1404E38BFAEF1010EA6FB32
:10AE500004234FF00002E6FB0E32A2FB034634004F
:10AE6000E2FB6264A1FB06E6A4FB07E8E4FB616881
:10AE70007642C8F1405838BFA8F10108A2FB06E4A9
:10AE8000A3FB08E5E2FB6854A1FB05E6A7FB04E889
:10AE9000E1FB648618F1200556F10006A809A8F127
:10AEA0001B08B10908F03F08B8F10A0F40EA8660B4
:10AEB0001CD901EB0C51BDE8F08100BFFCF5EEE8B8
:10AEC000E2DDD8D3CFCBC7C3C0BDB9B6B4B1AEAC49
:10AED000A9A7A5A3A19F9D9B9A9896959392908FC1
:10AEE0008D8C8B898887868584838281A0FB00680E
:10AEF00000FB01F208EB4208B8EB872807D53418AD
:10AF000058EB0104D5D5401C51F10001D1E7341AAA
:10AF100078EB0104CDD4401E71F10001C9E75FEA6E
:10AF20004C0C5FEA9C5C0DD105D34FF0000001F0A2
:10AF30000041BDE8F081BDE8F04170B5FFF7DEFEED
:10AF40006DDBFFBEBDE8F0414FF0000000497047E7
:10AF50000000F87F10B591EA030F48BF83F000436B
:10AF60003FF55AAB841A71EB030C07D212198CF01F
:10AF7000004C43EB0C03001B61EB0C01DFF8A4E178
:10AF80004FEA1154A4EB135C1EEA430F18BF9EEA6C
:10AF9000445F00F0B08023EA6E03524221EA04517C
:10AFA000C3EB6E0338BF5B1EDCF1200E25D322FA03
:10AFB0000CFE10EB0E0043FA0CFE41EB0E01CCF13F
:10AFC000200E03FA0EFE10EB0E0051F10001CCF141
:10AFD000200E29D412FA0EF201EB0451BDE8104004
:10AFE00058BF7047401C1CBFB2F1004F704700288B
:10AFF0000CBF491C20F00100704712EB020E43EB1E
:10B00000030218BF4FF0010E4EEA4202ACF1200CD1
:10B01000DCF11E0E54D943FA0CFE10EB0E0051F178
:10B02000FF31CCF11E0ED5D50EF1010E12FA0EFE37
:10B03000404141EB010101EB445C5FEA5C5C10D9EB
:10B0400010EBDE7001EB045138BFBEF1004FBDE8DC
:10B05000104018BF704700280CBF491C20F00100A9
:10B06000704730D24FEAD42C11F5001124F400645B
:10B070001BD0B1FA81F20B3AA41AA41ED2F120031C
:10B08000914030FA03F31943904001EBCC71002C4E
:10B0900001EB0451BDE81040A8BF704701F1C04169
:10B0A0004FF0000001F000417047B0FA80F310FA51
:10B0B00003F100D110BDE41A173C4805C90AE4E7C2
:10B0C00001EB045110BD491001EB0451BDE81040E3
:10B0D0004FEA300002E04FF0000170474A0008BF1D
:10B0E0000042F8D0B2F5001F28BF704701F00041C0
:10B0F0004FF0000070479EEA445F07D011EA5E0FF0
:10B10000BDE8104004BF002100207047BDE810409A
:10B1100070B5FFF7F3FD00BF40DFF63E83F000415E
:10B12000104670470000E0FF43004FEAD30C4FEA9F
:10B130003C0C43401FBF40070CF1605113F0FE4F21
:10B1400070471CF0006F03D100200CF000417047E5
:10B150000CF0004343EA507010B540EACC0000F018
:10B160000EF800BF000000924FEA0001FFF714BE86
:10B170004FF000414FF00000A1F5002170470EF1A3
:10B18000020E2EF0030E5EF8044B244204D44FEA64
:10B190004102B2F17F4F11D84FEA4003B3F17F4F24
:10B1A0000CD80ED14FEAD07CB2F17F4F0CEB4C0C97
:10B1B0000CF1020C08BF4CEBD17C04E04FF0080C02
:10B1C00001E04FEAD17C0CEB4C0324FA03F404F0C9
:10B1D0000704B4F1040C06D20EEB840CBDE8104059
:10B1E0004CF0010C6047DFE80CF0070802024FF05A
:10B1F0000040A0F5800010BD0846420018BFD2F103
:10B20000807288BF00F0004010BD4FF04070E1EE4A
:10B21000100A7047FF2141EAD050C0057047F5F78A
:10B2200029BB000000000404043C3C0000080000AE
:10B23000000800082CF4473B6C48B23B705BD83BDD
:10B24000395CA83B8EBA5F3BB25D47BB777ADFBC07
:10B25000F31C48BDBAF61FBD342CC5BDAC0B68BE8F
:10B26000C1110D3E6CE40F3FC1110D3EAC0B68BE29
:10B27000342CC5BDBAF61FBDF31C48BD777ADFBCC0
:10B28000B25D47BB8EBA5F3B395CA83B705BD83B75
:10B290006C48B23B2CF4473B67A029BD9C5775BD59
:10B2A0006FD1A5BD4AC9D4BDF8C102BEE1D3533F99
:10B2B000F8C102BE4AC9D4BD6FD1A5BD9C5775BDAA
:10B2C00067A029BD84B46FBD5893B5BDDB14FCBD28
:10B2D00017B123BE66BE5D3F17B123BEDB14FCBDB4
:10B2E0005893B5BD84B46FBD00000000000000009D
:10B2F000000000000000000000000000000000004E
:10B30000000000000000000000000000000000003D
:10B31000000000000000000000000000000000002D
:10B32000000000000000000000000000000000001D
:10B33000000000000000000000000000000000000D
:10B3400000000000000000000000000000000000FD
:10B3500000000000000000000000000000000000ED
:10B360000000C0E0F0F8FCFCFCFCFCFCFCFCFCFC7D
:10B37000FCFCF8F0E0C000000000FFFFFFFFFFFF53
:10B380000000000000000000FFFFFFFFFFFF0000C3
:10B390000000FFFFFFFFFFFF0000000000000000B3
:10B3A000FFFFFFFFFFFF00000000FFFFFFFFFFFFA9
:10B3B0000000000000000000FFFFFFFFFFFF000093
:10B3C000000003070F1F3F3F3F3F3F3F3F3F3F3FCF
:10B3D0003F3F1F0F070300000000C0E0F0F8FCFC37
:10B3E000FCFCFCFCFCFCFC00000000000000000079
:10B3F000000000000000000000FFFFFFFFFFFF0053
:10B40000000000000000000000000000000000003C
:10B4100000FFFFFFFFFFFF00000000000000000032
:10B42000000000000000000000FFFFFFFFFFFF0022
:10B43000000000000000000000000000000000000C
:10B44000003F3F3F3F3F3F00000000000000000082
:10B450000000C0E0F0F8FCFCFCFCFCFCFCFCFCFC8C
:10B46000FCFCF8F0E0C0000000000000000000005C
:10B470000000000000000000FFFFFFFFFFFF0000D2
:10B480000000C0E0F0F8FCFE7E7E7E7E7E7E7E7E4A
:10B490007F3F1F0F070300000000FFFFFFFFFFFFBC
:10B4A000000000000000000000000000000000009C
:10B4B000000003070F1F3F3F3F3F3F3F3F3F3F3FDE
:10B4C0003F3F3E3C3830000000000C1C3C7CFCFC44
:10B4D000FCFCFCFCFCFCFCFCFCFCF8F0E0C000000C
:10B4E000000000000000000000000000000000005C
:10B4F000FFFFFFFFFFFF00000000000000007E7E56
:10B500007E7E7E7E7E7E7E7EFFFFFFFFE7C30000A5
:10B51000000000000000000000000000000000002B
:10B52000FFFFFFFFFFFF0000000030383C3E3F3FC1
:10B530003F3F3F3F3F3F3F3F3F3F1F0F070300005D
:10B540000000FCFCF8F0E0C000000000000000007B
:10B55000C0E0F0F8FCFC00000000FFFFFFFFFFFF71
:10B560000000000000000000FFFFFFFFFFFF0000E1
:10B570000000070F1F3F7F7F7E7E7E7E7E7E7E7E69
:10B58000FFFFFFFFFFFF00000000000000000000C1
:10B590000000000000000000FFFFFFFFFFFF0000B1
:10B5A000000000000000000000000000000000009B
:10B5B00003070F1F3F3F00000000C0E0F0F8FCFC55
:10B5C000FCFCFCFCFCFCFCFCFCFC7C3C1C0C0000C3
:10B5D0000000FFFFFFFFFFFF000000000000000071
:10B5E00000000000000000000000070F1F3F7F7FE9
:10B5F0007E7E7E7E7E7E7E7EFEFEFCF8F0E000009B
:10B60000000000000000000000000000000000003A
:10B61000FFFFFFFFFFFF0000000003070F1F3F3F7A
:10B620003F3F3F3F3F3F3F3F3F3F1F0F070300006C
:10B630000000C0E0F0F8FCFCFCFCFCFCFCFCFCFCAA
:10B64000FCFC7C3C1C0C00000000FFFFFFFFFFFF28
:10B6500000000000000000000000000000000000EA
:10B660000000FFFFFFFFFFFF7E7E7E7E7E7E7E7EF0
:10B67000FEFEFCF8F0E000000000FFFFFFFFFFFF10
:10B680000000000000000000FFFFFFFFFFFF0000C0
:10B69000000003070F1F3F3F3F3F3F3F3F3F3F3FFC
:10B6A0003F3F1F0F0703000000000C1C3C7CFCFC0C
:10B6B000FCFCFCFCFCFCFCFCFCFCF8F0E0C000002A
:10B6C000000000000000000000000000000000007A
:10B6D000FFFFFFFFFFFF0000000000000000000070
:10B6E0000000000000000000FFFFFFFFFFFF000060
:10B6F000000000000000000000000000000000004A
:10B70000FFFFFFFFFFFF000000000000000000003F
:10B71000000000000000000003070F1F3F3F000073
:10B720000000C0E0F0F8FCFCFCFCFCFCFCFCFCFCB9
:10B73000FCFCF8F0E0C000000000FFFFFFFFFFFF8F
:10B740000000000000000000FFFFFFFFFFFF0000FF
:10B750000000C3E7FFFFFFFF7E7E7E7E7E7E7E7E53
:10B76000FFFFFFFFE7C300000000FFFFFFFFFFFF39
:10B770000000000000000000FFFFFFFFFFFF0000CF
:10B78000000003070F1F3F3F3F3F3F3F3F3F3F3F0B
:10B790003F3F1F0F070300000000C0E0F0F8FCFC73
:10B7A000FCFCFCFCFCFCFCFCFCFCF8F0E0C0000039
:10B7B0000000FFFFFFFFFFFF00000000000000008F
:10B7C000FFFFFFFFFFFF00000000070F1F3F7F7F0D
:10B7D0007E7E7E7E7E7E7E7EFFFFFFFFFFFF00007F
:10B7E0000000000000000000000000000000000059
:10B7F000FFFFFFFFFFFF0000000030383C3E3F3FEF
:10B800003F3F3F3F3F3F3F3F3F3F1F0F070300008A
:10B810000000000000000000000000000000000028
:10B820000000000000000000000000000000000018
:10B830000000000000000000000000000000000008
:10B8400000000000000000000000000000000000F8
:10B8500000000000000000000000000000000000E8
:10B8600000000000000000000000000000000000D8
:10B8700000000000000000000000000000000000C8
:10B8800000000000000000000000000000000000B8
:10B8900000000000000000000000000000000000A8
:10B8A0000000000000000000000000000000000098
:10B8B0000000000000000000000000000000000088
:10B8C0000000000000000000000000000000000078
:10B8D0000000000000000000000000000000000068
:10B8E0000000000000000000000000000000000058
:10B8F0000000000000000000000000000000000048
:10B900000000000000000000000000000000000037
:10B910000000000000000000000000000000000027
:10B920000000000000000000000000000000000017
:10B930000000000000000000000000000000000007
:10B9400000000000000000000000000000000000F7
:10B9500000000000000000000000000000000000E7
:10B9600000000000000000000000000000000000D7
:10B9700000000000000000000000000000000000C7
:10B980000000000000000000000038FCFC3800004F
:10B990000000000D0D000000000E1E00001E0E0035
:10B9A000000000000000000020F8F820F8F8200057
:10B9B000020F0F020F0F0200387C444747CC98005B
:10B9C000060C0838380F070030300080C0603000A7
:10B9D0000C060301000C0C0080D87CE4BCD84000AD
:10B9E000070F0808070F080000101E0E00000000D7
:10B9F00000000000000000000000F0F80C0400004F
:10BA0000000003070C0800000000040CF8F0000020
:10BA10000000080C0703000080A0E0C0C0E0A08088
:10BA20000002030101030200008080E0E08080004A
:10BA30000000000303000000000000000000000000
:10BA40000000101E0E00000080808080808080003A
:10BA500000000000000000000000000000000000E6
:10BA60000000000C0C00000000000080C0603000EE
:10BA70000C06030100000000F8F80CC40CF8F000FC
:10BA800003070C080C070300001018FCFC00000062
:10BA90000008080F0F080800080C84C4643C180054
:10BAA0000E0F0908080C0C00080C444444FCB800B4
:10BAB000040C0808080F0700C0E0B098FCFC8000E8
:10BAC000000000080F0F08007C7C444444C484003C
:10BAD000040C0808080F0700F0F84C4444C080002C
:10BAE000070F0808080F07000C0C0484C47C3C00F6
:10BAF00000000F0F00000000B8FC444444FCB800F4
:10BB0000070F0808080F0700387C444444FCF8007D
:10BB1000000808080C070300000000303000000097
:10BB200000000006060000000000003030000000A9
:10BB30000000080E060000000080C06030180800F9
:10BB400000000103060C0800002020202020200017
:10BB500000010101010101000008183060C08000EF
:10BB600000080C0603010000181C04C4E43C180083
:10BB70000000000D0D000000F0F008C8C8F8F0004B
:10BB8000070F080B0B0B0100E0F0988C98F0E00019
:10BB90000F0F0000000F0F0004FCFC4444FCB80031
:10BBA000080F0F08080F0700F0F80C04040C180029
:10BBB00003070C08080C060004FCFC040CF8F00059
:10BBC000080F0F080C07030004FCFC44E40C1C00E5
:10BBD000080F0F08080C0E0004FCFC44E40C1C00C9
:10BBE000080F0F0800000000F0F80C84848C980007
:10BBF00003070C0808070F00FCFC404040FCFC0059
:10BC00000F0F0000000F0F00000004FCFC040000F8
:10BC10000000080F0F08000000000004FCFC0400F6
:10BC2000070F08080F07000004FCFCC0E03C1C00E4
:10BC3000080F0F00010F0E0004FCFC0400000000C0
:10BC4000080F0F08080C0E00FCFC387038FCFC00D4
:10BC50000F0F0000000F0F00FCFC3870E0FCFC0030
:10BC60000F0F0000000F0F00F8FC040404FCF800A4
:10BC7000070F0808080F070004FCFC44447C380048
:10BC8000080F0F0800000000F8FC040404FCF80092
:10BC9000070F080E3C3F270004FCFC44C4FC38009E
:10BCA000080F0F00000F0F00183C6444C49C1800DC
:10BCB000060E0808080F0700001C0CFCFC0C1C00FA
:10BCC0000000080F0F080000FCFC000000FCFC0056
:10BCD000070F0808080F0700FCFC000000FCFC0030
:10BCE0000103060C06030100FCFC000000FCFC0044
:10BCF000070F0E030E0F07000C3CF0E0F03C0C00A9
:10BD00000C0F0301030F0C00000C7CC0C07C3C0036
:10BD10000000080F0F0800001C0C84C4643C1C00C9
:10BD20000E0F0908080C0E000000FCFC04040000C3
:10BD300000000F0F080800003870E0C0800000000D
:10BD40000000000103070E0000000404FCFC0000DA
:10BD5000000008080F0F0000080C0603060C08007E
:10BD600000000000000000000000000000000000D3
:10BD700020202020202020200000030704000000B5
:10BD8000000000000000000000A0A0A0E0C0000033
:10BD9000070F0808070F080004FCFC2060C08000A3
:10BDA000000F0F08080F0700C0E0202020604000AF
:10BDB000070F0808080C040080C06024FCFC000089
:10BDC000070F0808070F0800C0E0A0A0A0E0C0000F
:10BDD000070F0808080C040040F8FC440C18000089
:10BDE000080F0F0800000000C0E02020C0E0200085
:10BDF000276F48487F3F000004FCFC4020E0C00063
:10BE0000080F0F00000F0F00000020ECEC000000F6
:10BE10000000080F0F0800000000000020ECEC00FC
:10BE200000307040407F3F0004FCFC80C060200078
:10BE3000080F0F01030E0C00000004FCFC000000C2
:10BE40000000080F0F080000E0E060C060E0C000E4
:10BE50000F0F0007000F0F0020E0C02020E0C000FF
:10BE6000000F0F00000F0F00C0E0202020E0C000F6
:10BE7000070F0808080F070020E0C02020E0C000DE
:10BE8000407F7F48080F0700C0E02020C0E020006E
:10BE9000070F08487F7F400020E0C06020E0C0001E
:10BEA000080F0F080000000040E0A02020604000C4
:10BEB000040C09090B0E04002020F8FC20200000CF
:10BEC0000000070F080C0400E0E00000E0E00000C4
:10BED000070F0808070F080000E0E00000E0E0009E
:10BEE0000003070C0C070300E0E0008000E0E00026
:10BEF000070F0C070C0F07002060C080C0602000F7
:10BF0000080C0703070C0800E0E0000000E0E00078
:10BF1000474F4848683F1F00606020A0E060200055
:10BF20000C0E0B09080C0C00004040F8BC04040087
:10BF3000000000070F080800000000BCBC00000063
:10BF40000000000F0F000000000404BCF840400097
:10BF50000008080F07000000080C040C080C04007F
:10BF60000000000000000000E0F0988C98F0E00075
:10BF70000F0F0000000F0F0004FCFC4444CC8C00A9
:10BF8000080F0F08080F070004FCFC4444FCB8002D
:10BF9000080F0F08080F070004FCFC04040C0C0039
:10BFA000080F0F080000000000F8FC0CFCF800006F
:10BFB0001C0F0F080F0F1C0004FCFC44E40C1C00B9
:10BFC000080F0F08080C0E000C3CE0FCE03C0C00D5
:10BFD0000C0F010F010F0C00080C444444FCB80086
:10BFE000040C0808080F0700FCFC80C060FCFC0083
:10BFF0000F0F0100000F0F00FCFC80C260FCFC0072
:10C000000F0F0100000F0F0004FCFCC0E03C1C00FF
:10C01000080F0F00010F0E0000F0F81C0CFCFC00D4
:10C02000080F0F00000F0F00FCFC387038FCFC00FC
:10C030000F0F0000000F0F00FCFC404040FCFC0014
:10C040000F0F0000000F0F00F8FC040404FCF800C0
:10C05000070F0808080F0700FCFC040404FCFC00A0
:10C060000F0F0000000F0F0004FCFC44447C38005C
:10C07000080F0F0800000000F0F80C04040C180072
:10C0800003070C08080C0600001C0CFCFC0C1C0030
:10C090000000080F0F0800001C3C60C080FCFC0082
:10C0A00000000C0D07030100F0F808FC08F8F00090
:10C0B0000103020F020301000C3CF0E0F03C0C0015
:10C0C0000C0F0301030F0C00FCFC0000FCFC000043
:10C0D0000F0F08080F1F1800387CC08080FCFC0080
:10C0E00000000000000F0F00FC00FCFC00FC000042
:10C0F0000F080F0F080F0000FC00FCFC00FC000004
:10C100000F080F0F081F180004FCFC4040C0C000BF
:10C11000080F0F08080C0F00FCFC40C0C000FC001A
:10C120000F0F080C0F000F0000FCFC4040C0C000C7
:10C13000000F0F08080C0F000C0404C4CCF8F0002A
:10C140000C0808080C070300FCFC80F80404F80045
:10C150000F0F0007080807000078CC8484FCFC005F
:10C16000080C0603010F0F0000A0A0A0E0C0000013
:10C17000070F0808070F0800E0E02020202000003B
:10C180000F0F090909060000E0E0A0A0A040000090
:10C190000F0F080808070000E0E0202020600000E2
:10C1A0000F0F00000000000000E02020E000000071
:10C1B0001C0F0C0C0F1C0000C0E0A0A0A0E0C000F1
:10C1C000070F0808080C040020E080E080E0200051
:10C1D000080F010F010F0800402020A0E0600000C0
:10C1E0000408090906060000E0E0000080E0000005
:10C1F0000F0F0201000F0000E0E0001080E00000DF
:10C200000F0F0201000F000004FCFC80C060200042
:10C21000080F0F01030E0C0000E02020E0E00000FA
:10C22000080700000F0F0000E0C00000C0E00000A1
:10C230000F000101000F0000E0E00000E0E000005E
:10C240000F0F01010F0F0000C0E0202020E0C00010
:10C25000070F0808080F0700E0E02020E0E00000DA
:10C260000F0F00000F0F000020E0C02020E0C000F2
:10C27000407F7F48080F0700C0E02020206040007A
:10C28000070F0808080C04002020E0E02020000030
:10C2900000000F0F0000000060C08000E0E0000020
:10C2A0000C0C070301000000C020F0F020C00000CB
:10C2B00003040F0F040300002060C080C060200052
:10C2C000080C0703070C0800E0E0000000E0000095
:10C2D0000F0F0808080F1800E0E00000E0E0000081
:10C2E000010302020F0F0000E000E0E000E00000A8
:10C2F0000F080F0F080F0000E000E0E000E0000072
:10C300000F080F0F081F10000000000000000000C1
:10C310000000000000000000E080800000E000005D
:10C320000F080807000F0000808080808080800058
:10C33000000000000000000040202020E0C00000BD
:10C34000040808090F070000E000C02020C000001A
:10C350000F01070808070000C0202020E0E00000CF
:10C36000080503010F0F000000000000000000009E
:10C370000000000000000000000000000000002F8E
:10C3800000000007000700147F147F14242A7F2A6E
:10C390001223130864623649552250000503000039
:10C3A000001C2241000041221C0014083E08140811
:10C3B000083E08080000A06000080808080800609F
:10C3C00060000020100804023E5149453E00427FB3
:10C3D000400042615149462141454B311814127FBA
:10C3E0001027454545393C4A494930017109050343
:10C3F0003649494936064949291E003636000000AB
:10C40000563600000814224100141414141400417C
:10C410002214080201510906324959513E7C121179
:10C42000127C7F494949363E414141227F414122A8
:10C430001C7F494949417F090909013E4149497A1F
:10C440007F0808087F00417F41002040413F017F75
:10C45000081422417F404040407F020C027F7F044D
:10C4600008107F3E4141413E7F090909063E415186
:10C47000215E7F09192946464949493101017F0159
:10C48000013F4040403F1F2040201F3F4038403F79
:10C490006314081463070870080761514945430095
:10C4A0007F41410001060830400041417F00040205
:10C4B0000102044040404040000305000020545465
:10C4C00054787F48444438384444442038444448ED
:10C4D0007F3854545418087E09010218A4A4A47C7F
:10C4E0007F0804047800447D40004080847D007F04
:10C4F0001028440000417F40007C041804787C0828
:10C500000404783844444438FC242424181824248F
:10C5100018FC7C080404084854545420043F444048
:10C52000203C4040207C1C2040201C3C4030403CB3
:10C5300044281028441CA0A0A07C4464544C44000F
:10C54000107C82000000FF000000827C10000804C4
:10C550000810087C1211127C7F494949317F4545FA
:10C56000453A7F01010103603F213F607F4949490E
:10C5700041730C7F0C732141494D337F1008047FB8
:10C580007E2011087E7F08142241403F01017F7FF9
:10C590000608067F7F0808087F3E4141413E7F0133
:10C5A00001017F7F090909063E4141412203017FC4
:10C5B000010361261806011C227F221C6314081443
:10C5C000633F20203F60070808087F7F407F407F4F
:10C5D0003F203F207F017F4848307F4878007F7FA1
:10C5E000484830004149492A1C7F103E413E6619A7
:10C5F00009097F20545478403E494545387E4A4ACF
:10C6000034007C04040C00384545493E38545454E9
:10C61000184C307C304C24424A34007C20107C0082
:10C620007C21117C007C10284400403C04047C7C6C
:10C630000810087C7C10107C0038444444387C048A
:10C64000047C00FC18242418384444442804047C46
:10C6500004044C9090907C18247E241844281028C0
:10C66000443C20203C601C10107C007C407C407CC2
:10C670003C203C207C047C5070007C5070007C7C12
:10C6800050700000424252523C7C10384438402CDA
:10C69000127E00000000000030313233343536376E
:10C6A00038394142434445464030580030313233F6
:10C6B00034353637383961626364656640307800F6
:10C6C000040000080000000000000002000100005B
:10C6D000100000000000000004FA97999999D93FD2
:10C6E000AF788E1DC571CC3F9FC678D0099AC33FE5
:10C6F000935555555555E53F599322942449D23FBA
:10C70000DE03CB966446C73F44523EDF12F1C23F80
:10C710004FBB610567ACDD3F182D4454FB21E93F59
:10C720009BF681D20B73EF3F182D4454FB21F93F48
:10C73000E2652F227F2B7A3C075C143326A6813CCE
:10C74000BDCBF07A8807703C075C143326A6913C79
:10C75000C4EB98999999C9BF711623FEC671BCBFE5
:10C760006D9A74AFF2B0B3BF9AFDDE522DDEADBF4D
:10C770002F6C6A2C44B4A2BF0D5555555555D53F65
:10C78000FF8300922449C23F6E204CC5CD45B73F80
:10C79000513DD0A0660DB13FEB0D76244B7BA93FF8
:10C7A00011DA22E33AAD903F4C5555555555A53F0A
:10C7B0007751C1166CC156BF9015CB19A001FA3E36
:10C7C000AD529C804F7E92BEC4B1B4BD9EEE213E60
:10C7D000D43888BEE9FAA8BD0000000000000000BF
:10C7E00000004054FB21F93F3163621A61B4D03D2F
:10C7F0000000601A61B4D03D7370032E8A19A33B08
:10C800000000002E8A19A33BC14920259A837B3959
:10C8100000000000000000006E83F9A22915444EBC
:10C82000D15727FCC0DD34F5999562DB4190433C3C
:10C83000AB6351FE61C5BBDE3A6E24B7E0D24D4218
:10C84000EA2E49061C92D1091CEB1DFE3EA729B118
:10C85000F53582E88444BB2E26709CE9417E5FB4A6
:10C8600039D69139F43953838B5F849C3B28F9BDC9
:10C87000FF97F81F0F9805DE8B112FEF1F6D0A5AD7
:10C88000CF7E366DB709CB27663F464F2DEA5F9EB8
:10C89000C7BA27757BF1E5EBF739073DEA92528A73
:10C8A000B15FFB6B085D8D1F000000006E83F9A275
:10C8B0002915444ED15727FCC0DD34F5999562DB2C
:10C8C0004190433CAB6351FEA6F810111111813F1A
:10C8D000D561C119A0012ABF7DFEB157E31DC73E36
:10C8E000EB9C2B8AE6E55ABE7CD5CF5A3AD9E53D7A
:10C8F0007AFE10111111C13F37D60684F464963FB9
:10C90000280356C9226D6D3F0165F2F2D844433FBA
:10C91000A69237A0887E143F735360DBCB75F3BEBD
:10C92000FE41B31BBAA1AB3F93846EE9E326823F7D
:10C930001583E0FEC8DB573F68108D1AF726303F9D
:10C94000E9A7F0320FB8123FD47ABF74702AFB3EC9
:10C9500002400000000000A00000000005400000B0
:10C96000000000C8000000000C4000000000409CD7
:10C9700000000000194000000020BCBE00000000C4
:10C9800034400000BFC91B8E00000004B540000009
:10C99000504BCFD06607E2CF010000006C41000091
:10C9A0003E8251AADFEEA73401000000D942000008
:10C9B000DCB5A0E23A301F97FFFFFFFFB44500004F
:10C9C000FD25A0C8E9A3C14FFFFFFFFFFF3F000007
:10C9D0000000008000000000FF3F00000000008019
:10C9E00000000000564F4C2E4645202020202000FD
:10C9F000564F4C2E554D4520202020200000000091
:10CA000053454E5320464520202020004449535092
:10CA10004C455920202020004669656C6420202068
:10CA200020000000202042454143482020200000F3
:10CA300020205041524B20202000000046494C54F9
:10CA40004552204C503120200000000046494C54F3
:10CA50004552204C5032202000000000564F4C2EF2
:10CA6000544F4E4520200000484F542053544F4E01
:10CA7000452020004C45442042524947485420203C
:10CA800000000000504F575F202000004E6F2046EE
:10CA90006572756D20200000444953432D2000002D
:10CAA000564F4C2E572E5349472E2000564F4C2E92
:10CAB000534348454D452000205255424249534872
:10CAC00020000000416C6C206D6574616C200000DA
:10CAD0002043752B41672B202A00000057524954F0
:10CAE00045202D206F72202B00000000D093D180B4
:10CAF0002ED0A1D0BB2ED0A1D0B8D0B32E00000034
:10CB00003000000050524F46494C450046455252B5
:10CB1000495445004742562F474246005059432F3B
:10CB2000454E47002053656142454143480000009F
:10CB30004741494E000000004241545445525900BB
:10CB4000465245515F000000D09CD095D094D0ACA7
:10CB5000D18AD0BFD0BBD18ED1810000D0ADD09AC8
:10CB6000D0A0D090D09DD18AD18AD18AD18AD18AC1
:10CB700000000000D0A4D098D09BD0ACD0A2D0A010
:10CB8000D18AD18AD18AD18AD18A0000D18AD18A28
:10CB9000D18AD09FD09ED09BD095D18AD18AD18A7C
:10CBA000D18A0000D0AFD0A0D09AD09ED0A1D0A280
:10CBB000D0ACD18AD18AD18AD18A0000D0A2D09EAD
:10CBC000D09DD18AD097D092D0A3D09AD090D18A3C
:10CBD000D18AD18A00000000D18AD18AD18AD09F1F
:10CBE000D09BD0AFD096D18AD18AD18A00000000E4
:10CBF000D0A2D09ED09AD18AD18AD18A00000000DA
:10CC0000D18AD18AD18AD09FD090D0A0D09AD18A0F
:10CC1000D18AD18A00000000D093D09ED0A0D18AC2
:10CC2000D09AD090D09CD09DD098D18AD18A000043
:10CC3000D0A7D0A3D092D0A1D0A2D18AD096D0959F
:10CC4000D09BD18AD18A0000D18AD18AD18AD09C46
:10CC5000D0A3D0A1D09ED0A0D18AD18A000000005C
:10CC6000D093D0A0D09ED09CD09AD09ED0A1D0A25C
:10CC7000D0ACD18AD18A0000D09CD09ED0A0D0A1C7
:10CC8000D09AD18AD09FD09BD0AFD096D18A0000C5
:10CC9000D090D0A2D090D09AD090D18AD093D0A06A
:10CCA000D09ED09CD18A0000D091D090D09BD090C3
:10CCB000D09DD0A1D18A0000D094D098D0A1D09A94
:10CCC000D18C0000D0A7D0A3D09220D096D095D000
:10CCD0009BD095D097D09000D091D095D097D18A05
:10CCE000D096D095D09BD095D097D09000000000E2
:10CCF000D0A7D090D0A1D0A2D09ED0A2D09000003A
:10CD0000D0A4D095D0A0D0A0D098D0A20000000090
:10CD1000D0A7D090D0A1D0A200000000D092D0A186
:10CD2000D095D18AD09CD095D0A2D090D09BD0ABBA
:10CD300000000000D09FD0A0D09ED0A4D098D09B5F
:10CD4000D0AC0000D091D090D0A2D090D0A0D095FF
:10CD5000D0AF000090CD0008000000207402000059
:10CD6000C401000888CE00087402002004170000E7
:10CD7000200200081C00000043000000F8FFFFFF35
:10CD80000C0000000E0000000F0000002E0000004C
:10CD900032A662015A20080139C5B5E00A47C50A22
:10CDA000D7A3BC0A3E2C6101877F0102040A5A13F3
:10CDB000E616010206010815010501571564015028
:10CDC00001127C14B414017303B4147C06B4D203AE
:10CDD0001304CB140834CD1B0838081A44081A3041
:10CDE0000813F0CC1B0840081A10101A0C0811196F
:10CDF0000813DCCA1B08A8181A14102A1C2412C90C
:10CE00001B0860101AAC181A90081AA0081AEC0433
:10CE10001AE4181A30101A5C0C1ABC281A84081A62
:10CE2000F0081A3C081A74085A4C081A98081AB8DC
:10CE3000281119081AC4081A74081AA4181A0C0818
:10CE40001A5C081A68082A1820190C1AC40C1A1C33
:10CE5000841A8C081AD8141A18081A8C182A241044
:10CE6000290819041A78181AB8101A48081A30082C
:10CE70001119082AD010191C3201821023127A408D
:08CE80000880C0E0F0F8FCFEA0
:040000050800018965
:00000001FF
